################################################################################
#                                                                              #
#      IAR Universal Linker V4.60I/386                                         #
#                                                                              #
#           Link time     =  08/Jun/2010  15:10:26                             #
#           Target CPU    =  ARM                                               #
#           List file     =  F:\SVN\cn\Master\Release_NEWSGOLD\List\Master_NEW #
#                            SGOLD.map                                         #
#           Output file 1 =  F:\SVN\cn\Master\Master_NEWSGOLD.elf              #
#                            Format: elf, variant: -ynpra                      #
#           Command line  =  F:\SVN\cn\Master\Release_NEWSGOLD\Obj\func.r79    #
#                            F:\SVN\cn\Master\Release_NEWSGOLD\Obj\getConfig.r #
#                            79                                                #
#                            F:\SVN\cn\Master\Release_NEWSGOLD\Obj\main.r79    #
#                            F:\SVN\cn\Master\Release_NEWSGOLD\Obj\optionMenu. #
#                            r79                                               #
#                            F:\SVN\cn\Master\Release_NEWSGOLD\Obj\ptcFileWork #
#                            .r79                                              #
#                            F:\SVN\cn\Master\Release_NEWSGOLD\Obj\string.r79  #
#                            F:\SVN\cn\Master\Release_NEWSGOLD\Obj\usedstr.r79 #
#                            F:\SVN\cn\Master\Release_NEWSGOLD\Obj\visual.r79  #
#                            -o F:\SVN\cn\Master\Master_NEWSGOLD.elf -Felf     #
#                            -l                                                #
#                            F:\SVN\cn\Master\Release_NEWSGOLD\List\Master_NEW #
#                            SGOLD.map                                         #
#                            -xmsnio -f F:\SVN\cn\Master/test.xcl (-carm       #
#                            -V(CODE)CODE_AREA,12 -V(DATA)DATA_AREA,12         #
#                            -Z(CODE_AREA)ELFBEGIN,DATA_ID,START,CODE,DATA_C,I #
#                            NITTAB,DATA_Z,DATA_N,CONFIG_C=0-FFFFFFFF          #
#                            -Z(DATA_AREA)DATA_I=0-FFFFFFFF) -ynpra            #
#                            "F:\software\Embedded Workbench 4.0 Evaluation\AR #
#                            M\LIB\dl5tpainl8n.r79"                            #
#                            -s main                                           #
#                                                                              #
#                        Copyright 1987-2007 IAR Systems. All rights reserved. #
################################################################################





                ****************************************
                *                                      *
                *           CROSS REFERENCE            *
                *                                      *
                ****************************************

       Program entry at : CODE_AREA 00003FC8  Relocatable, from module : main




                ****************************************
                *                                      *
                *            RUNTIME MODEL             *
                *                                      *
                ****************************************

  StackAlign4  = USED
  __cpu_mode   = __pcs__interwork
  __data_model = absolute
  __endian     = little
  __rt_version = 6



                ****************************************
                *                                      *
                *              MODULE MAP              *
                *                                      *
                ****************************************


  DEFINED ABSOLUTE ENTRIES
    *************************************************************************

  DEFINED ABSOLUTE ENTRIES
    *************************************************************************

  FILE NAME : F:\SVN\cn\Master\Release_NEWSGOLD\Obj\func.r79
  PROGRAM MODULE, NAME : func

  SEGMENTS IN THE MODULE
  ======================
ELFBEGIN
  Relative segment, address: CODE_AREA 00000000, align: 0
  Segment part 0. ROOT.
           ENTRY                   ADDRESS         REF BY
           =====                   =======         ======
           ELF_BEGIN               00000000        Killer (main)
    -------------------------------------------------------------------------
CODE
  Relative segment, address: CODE_AREA 0000016C - 00000173 (0x8 bytes), align: 2
  Segment part 1. ROOT.
           ENTRY                   ADDRESS         REF BY
           =====                   =======         ======
           kill_data               0000016C        Killer (main)
                                                   method7_2 (visual)
                                                   method7_xy (visual)
           seqkill                 00000170 

    *************************************************************************

  FILE NAME : F:\SVN\cn\Master\Release_NEWSGOLD\Obj\getConfig.r79
  PROGRAM MODULE, NAME : getConfig

  SEGMENTS IN THE MODULE
  ======================
DATA_Z
  Relative segment, address: CODE_AREA 00009B10 - 00015B0F (0xc000 bytes), align: 2
  Segment part 43.            Intra module refs:   Segment part 47
                                                   Segment part 95
           ENTRY                   ADDRESS         REF BY
           =====                   =======         ======
           cfg_buf                 00009B10 
    -------------------------------------------------------------------------
DATA_Z
  Relative segment, address: CODE_AREA 00015B10 - 00015B13 (0x4 bytes), align: 2
  Segment part 44.            Intra module refs:   Segment part 118
                                                   Segment part 60
                                                   Segment part 77
                                                   doItemJob
           ENTRY                   ADDRESS         REF BY
           =====                   =======         ======
           ptcfgtop                00015B10        saveAllConfig (ptcFileWork)
    -------------------------------------------------------------------------
CODE
  Segment part 45. NOT NEEDED.
    -------------------------------------------------------------------------
CODE
  Relative segment, address: CODE_AREA 00000174 - 00000253 (0xe0 bytes), align: 2
  Segment part 46.            Intra module refs:   readConfig
                                                   reloadThisPatch
           ENTRY                   ADDRESS         REF BY
           =====                   =======         ======
           loadConfig              00000174 
               stack 1 = 00000000 ( 000000BC )
    -------------------------------------------------------------------------
CODE
  Relative segment, address: CODE_AREA 00000254 - 00000257 (0x4 bytes), align: 2
  Segment part 47.            Intra module refs:   loadConfig
    -------------------------------------------------------------------------
CODE
  Segment part 48. NOT NEEDED.
    -------------------------------------------------------------------------
CODE
  Relative segment, address: CODE_AREA 00000258 - 000002CF (0x78 bytes), align: 2
  Segment part 49.            Intra module refs:   readConfig
           ENTRY                   ADDRESS         REF BY
           =====                   =======         ======
           addPatchConfigList      00000258 
               stack 1 = 00000000 ( 00000004 )
    -------------------------------------------------------------------------
CODE
  Segment part 50. NOT NEEDED.
    -------------------------------------------------------------------------
CODE
  Relative segment, address: CODE_AREA 000002D0 - 0000049F (0x1d0 bytes), align: 2
  Segment part 51.            Intra module refs:   readConfig
                                                   reloadThisPatch
           ENTRY                   ADDRESS         REF BY
           =====                   =======         ======
           addToPatchInfo          000002D0 
               stack 1 = 00000000 ( 00000018 )
    -------------------------------------------------------------------------
CODE
  Segment part 52. NOT NEEDED.
    -------------------------------------------------------------------------
CODE
  Relative segment, address: CODE_AREA 000004A0 - 000004D7 (0x38 bytes), align: 2
  Segment part 53.            Intra module refs:   addPrepareData
           ENTRY                   ADDRESS         REF BY
           =====                   =======         ======
           addPreItemToData        000004A0 
    -------------------------------------------------------------------------
CODE
  Segment part 54. NOT NEEDED.
    -------------------------------------------------------------------------
CODE
  Relative segment, address: CODE_AREA 000004D8 - 0000058B (0xb4 bytes), align: 2
  Segment part 55.            Intra module refs:   addPrepareData
                                                   doItemJob
                                                   doSubMenuJob
                                                   doTemplateWork
                                                   readConfig
                                                   subMenuCopy
           ENTRY                   ADDRESS         REF BY
           =====                   =======         ======
           addItemToConfig         000004D8 
               stack 1 = 00000000 ( 0000001C )
    -------------------------------------------------------------------------
CODE
  Segment part 56. NOT NEEDED.
    -------------------------------------------------------------------------
CODE
  Relative segment, address: CODE_AREA 0000058C - 000006F3 (0x168 bytes), align: 2
  Segment part 57.            Intra module refs:   readConfig
           ENTRY                   ADDRESS         REF BY
           =====                   =======         ======
           addPrepareData          0000058C 
               stack 1 = 00000000 ( 00000020 )
    -------------------------------------------------------------------------
CODE
  Segment part 58. NOT NEEDED.
    -------------------------------------------------------------------------
CODE
  Relative segment, address: CODE_AREA 000006F4 - 000007D7 (0xe4 bytes), align: 2
  Segment part 59.            Intra module refs:   doItemJob
           ENTRY                   ADDRESS         REF BY
           =====                   =======         ======
           addPreDataToCBoxItem    000006F4 
               stack 1 = 00000000 ( 00000018 )
    -------------------------------------------------------------------------
CODE
  Relative segment, address: CODE_AREA 000007D8 - 000007DB (0x4 bytes), align: 2
  Segment part 60.            Intra module refs:   addPatchConfigList
                                                   addPreDataToCBoxItem
                                                   addPrepareData
                                                   addToPatchInfo
    -------------------------------------------------------------------------
CODE
  Segment part 61. NOT NEEDED.
    -------------------------------------------------------------------------
CODE
  Relative segment, address: CODE_AREA 000007DC - 00000813 (0x38 bytes), align: 2
  Segment part 62.            Intra module refs:   cboxItemColon
           ENTRY                   ADDRESS         REF BY
           =====                   =======         ======
           addItemToCBox           000007DC 
    -------------------------------------------------------------------------
CODE
  Segment part 63. NOT NEEDED.
    -------------------------------------------------------------------------
CODE
  Relative segment, address: CODE_AREA 00000814 - 0000092B (0x118 bytes), align: 2
  Segment part 64.            Intra module refs:   doItemJob
           ENTRY                   ADDRESS         REF BY
           =====                   =======         ======
           cboxItemColon           00000814 
               stack 1 = 00000000 ( 0000001C )
    -------------------------------------------------------------------------
CODE
  Segment part 65. NOT NEEDED.
    -------------------------------------------------------------------------
CODE
  Relative segment, address: CODE_AREA 0000092C - 0000095B (0x30 bytes), align: 2
  Segment part 66.            Intra module refs:   doSubMenuJob
                                                   doTemplateWork
                                                   readConfig
           ENTRY                   ADDRESS         REF BY
           =====                   =======         ======
           isThatItem              0000092C 
    -------------------------------------------------------------------------
CODE
  Segment part 67. NOT NEEDED.
    -------------------------------------------------------------------------
CODE
  Relative segment, address: CODE_AREA 0000095C - 000009BF (0x64 bytes), align: 2
  Segment part 68.            Intra module refs:   doItemJob
           ENTRY                   ADDRESS         REF BY
           =====                   =======         ======
           findTemplate            0000095C 
               stack 1 = 00000000 ( 00000010 )
    -------------------------------------------------------------------------
CODE
  Segment part 69. NOT NEEDED.
    -------------------------------------------------------------------------
CODE
  Relative segment, address: CODE_AREA 000009C0 - 00000A2F (0x70 bytes), align: 2
  Segment part 70.            Intra module refs:   doItemJob
           ENTRY                   ADDRESS         REF BY
           =====                   =======         ======
           isCurrectItem           000009C0 
               stack 1 = 00000000 ( 00000008 )
    -------------------------------------------------------------------------
CODE
  Segment part 71. NOT NEEDED.
    -------------------------------------------------------------------------
CODE
  Relative segment, address: CODE_AREA 00000A30 - 0000283B (0x1e0c bytes), align: 2
  Segment part 72.            Intra module refs:   doSubMenuJob
                                                   doTemplateWork
                                                   readConfig
           ENTRY                   ADDRESS         REF BY
           =====                   =======         ======
           doItemJob               00000A30 
               stack 1 = 00000000 ( 000000B4 )
    -------------------------------------------------------------------------
CODE
  Segment part 73. NOT NEEDED.
    -------------------------------------------------------------------------
CODE
  Relative segment, address: CODE_AREA 0000283C - 00002A7B (0x240 bytes), align: 2
  Segment part 74.            Intra module refs:   doTemplateWork
                                                   readConfig
           ENTRY                   ADDRESS         REF BY
           =====                   =======         ======
           doSubMenuJob            0000283C 
               stack 1 = 00000000 ( 0000001C )
    -------------------------------------------------------------------------
CODE
  Segment part 75. NOT NEEDED.
    -------------------------------------------------------------------------
CODE
  Relative segment, address: CODE_AREA 00002A7C - 00002ACF (0x54 bytes), align: 2
  Segment part 76.            Intra module refs:   readConfig
           ENTRY                   ADDRESS         REF BY
           =====                   =======         ======
           addInfoToPatchInfo      00002A7C 
               stack 1 = 00000000 ( 00000010 )
    -------------------------------------------------------------------------
CODE
  Relative segment, address: CODE_AREA 00002AD0 - 00002AD3 (0x4 bytes), align: 2
  Segment part 77.            Intra module refs:   addInfoToPatchInfo
                                                   doItemJob
    -------------------------------------------------------------------------
CODE
  Segment part 78. NOT NEEDED.
    -------------------------------------------------------------------------
CODE
  Relative segment, address: CODE_AREA 00002AD4 - 00002B27 (0x54 bytes), align: 2
  Segment part 79.            Intra module refs:   readConfig
           ENTRY                   ADDRESS         REF BY
           =====                   =======         ======
           isPrepareItem           00002AD4 
    -------------------------------------------------------------------------
CODE
  Segment part 80. NOT NEEDED.
    -------------------------------------------------------------------------
CODE
  Relative segment, address: CODE_AREA 00002B28 - 00002D6F (0x248 bytes), align: 2
  Segment part 81.            Intra module refs:   readConfig
           ENTRY                   ADDRESS         REF BY
           =====                   =======         ======
           doTemplateWork          00002B28 
               stack 1 = 00000000 ( 00000018 )
    -------------------------------------------------------------------------
CODE
  Segment part 82. NOT NEEDED.
    -------------------------------------------------------------------------
CODE
  Relative segment, address: CODE_AREA 00002D70 - 0000325F (0x4f0 bytes), align: 2
  Segment part 83.            Intra module refs:   doItemJob
           ENTRY                   ADDRESS         REF BY
           =====                   =======         ======
           subMenuCopy             00002D70 
               stack 1 = 00000000 ( 00000028 )
    -------------------------------------------------------------------------
CODE
  Segment part 84. NOT NEEDED.
    -------------------------------------------------------------------------
CODE
  Relative segment, address: CODE_AREA 00003260 - 000035DB (0x37c bytes), align: 2
  Segment part 85.            Intra module refs:   getAllPatchData
                                                   reloadThisPatch
           ENTRY                   ADDRESS         REF BY
           =====                   =======         ======
           readConfig              00003260        deleteAllConfig (optionMenu)
               stack 1 = 00000000 ( 0000001C )
    -------------------------------------------------------------------------
CODE
  Relative segment, address: CODE_AREA 000035DC - 000035DF (0x4 bytes), align: 2
  Segment part 86.            Intra module refs:   readConfig
    -------------------------------------------------------------------------
CODE
  Relative segment, address: CODE_AREA 000035E0 - 000035E3 (0x4 bytes), align: 2
  Segment part 87.            Intra module refs:   doSubMenuJob
                                                   doTemplateWork
                                                   readConfig
    -------------------------------------------------------------------------
CODE
  Relative segment, address: CODE_AREA 000035E4 - 000035E7 (0x4 bytes), align: 2
  Segment part 88.            Intra module refs:   doSubMenuJob
                                                   doTemplateWork
                                                   readConfig
    -------------------------------------------------------------------------
CODE
  Segment part 89. NOT NEEDED.
    -------------------------------------------------------------------------
CODE
  Segment part 90. NOT NEEDED.
           ENTRY                   ADDRESS         REF BY
           =====                   =======         ======
           freeSubMenuItem         
               not allocated function
    -------------------------------------------------------------------------
CODE
  Segment part 91. NOT NEEDED.
    -------------------------------------------------------------------------
CODE
  Relative segment, address: CODE_AREA 000035E8 - 00003697 (0xb0 bytes), align: 2
  Segment part 92.            Intra module refs:   fuckThemAll
                                                   reloadThisPatch
           ENTRY                   ADDRESS         REF BY
           =====                   =======         ======
           freePatchItem           000035E8 
               stack 1 = 00000000 ( 0000000C )
    -------------------------------------------------------------------------
CODE
  Segment part 93. NOT NEEDED.
    -------------------------------------------------------------------------
CODE
  Relative segment, address: CODE_AREA 00003698 - 000037A3 (0x10c bytes), align: 2
  Segment part 94.
           ENTRY                   ADDRESS         REF BY
           =====                   =======         ======
           reloadThisPatch         00003698        deleteThis (optionMenu)
               stack 1 = 00000000 ( 00000018 )
    -------------------------------------------------------------------------
CODE
  Relative segment, address: CODE_AREA 000037A4 - 000037A7 (0x4 bytes), align: 2
  Segment part 95.            Intra module refs:   readConfig
                                                   reloadThisPatch
    -------------------------------------------------------------------------
CODE
  Segment part 96. NOT NEEDED.
    -------------------------------------------------------------------------
CODE
  Relative segment, address: CODE_AREA 000037A8 - 00003837 (0x90 bytes), align: 2
  Segment part 97.            Intra module refs:   sortPatchConfigList
           ENTRY                   ADDRESS         REF BY
           =====                   =======         ======
           swapPatchConfigList     000037A8 
               stack 1 = 00000000 ( 00000020 )
    -------------------------------------------------------------------------
CODE
  Segment part 98. NOT NEEDED.
    -------------------------------------------------------------------------
CODE
  Relative segment, address: CODE_AREA 00003838 - 00003897 (0x60 bytes), align: 2
  Segment part 99.            Intra module refs:   readConfig
           ENTRY                   ADDRESS         REF BY
           =====                   =======         ======
           sortPatchConfigList     00003838 
               stack 1 = 00000000 ( 0000000C )
    -------------------------------------------------------------------------
CODE
  Segment part 100. NOT NEEDED.
    -------------------------------------------------------------------------
CODE
  Relative segment, address: CODE_AREA 00003898 - 00003903 (0x6c bytes), align: 2
  Segment part 101.
           ENTRY                   ADDRESS         REF BY
           =====                   =======         ======
           fuckThemAll             00003898        Killer (main)
                                                   configRestore (optionMenu)
                                                   deleteAllConfig (optionMenu)
               stack 1 = 00000000 ( 0000000C )
    -------------------------------------------------------------------------
CODE
  Segment part 102. NOT NEEDED.
    -------------------------------------------------------------------------
CODE
  Relative segment, address: CODE_AREA 00003904 - 0000393B (0x38 bytes), align: 2
  Segment part 103.
           ENTRY                   ADDRESS         REF BY
           =====                   =======         ======
           getPatchConfigItem      00003904        deleteThis (optionMenu)
                                                   maincsm_onmessage (main)
                                                   menu_iconhndl (main)
                                                   menu_onkey (main)
                                                   profile_menu_iconhndl (optionMenu)
                                                   profile_menu_onkey (optionMenu)
                                                   showPatchInfo (optionMenu)
                                                   show_option_menu (optionMenu)
    -------------------------------------------------------------------------
CODE
  Segment part 104. NOT NEEDED.
    -------------------------------------------------------------------------
CODE
  Relative segment, address: CODE_AREA 0000393C - 0000395F (0x24 bytes), align: 2
  Segment part 105.
           ENTRY                   ADDRESS         REF BY
           =====                   =======         ======
           getMaxCBoxItem          0000393C        createEditGui (main)
    -------------------------------------------------------------------------
CODE
  Segment part 106. NOT NEEDED.
    -------------------------------------------------------------------------
CODE
  Relative segment, address: CODE_AREA 00003960 - 00003983 (0x24 bytes), align: 2
  Segment part 107.
           ENTRY                   ADDRESS         REF BY
           =====                   =======         ======
           getCurCBoxItem          00003960        edGHook (main)
    -------------------------------------------------------------------------
CODE
  Segment part 108. NOT NEEDED.
    -------------------------------------------------------------------------
CODE
  Relative segment, address: CODE_AREA 00003984 - 000039D7 (0x54 bytes), align: 2
  Segment part 109.
           ENTRY                   ADDRESS         REF BY
           =====                   =======         ======
           getInitCBoxItem         00003984        createEditGui (main)
               stack 1 = 00000000 ( 00000004 )
    -------------------------------------------------------------------------
CODE
  Segment part 110. NOT NEEDED.
    -------------------------------------------------------------------------
CODE
  Relative segment, address: CODE_AREA 000039D8 - 00003A1B (0x44 bytes), align: 2
  Segment part 111.
           ENTRY                   ADDRESS         REF BY
           =====                   =======         ======
           getAllPatchData         000039D8        configRestore (optionMenu)
                                                   main (main)
               stack 1 = 00000000 ( 00000008 )
    -------------------------------------------------------------------------
CODE
  Segment part 112. NOT NEEDED.
    -------------------------------------------------------------------------
CODE
  Relative segment, address: CODE_AREA 00003A1C - 00003A57 (0x3c bytes), align: 2
  Segment part 113.
           ENTRY                   ADDRESS         REF BY
           =====                   =======         ======
           setPatchOnOff           00003A1C        maincsm_onmessage (main)
                                                   menu_onkey (main)
                                                   profile_menu_onkey (optionMenu)
               stack 1 = 00000000 ( 00000010 )
    -------------------------------------------------------------------------
CODE
  Segment part 114. NOT NEEDED.
    -------------------------------------------------------------------------
CODE
  Relative segment, address: CODE_AREA 00003A58 - 00003A7F (0x28 bytes), align: 2
  Segment part 115.           Intra module refs:   setPatchOnOff
           ENTRY                   ADDRESS         REF BY
           =====                   =======         ======
           getPatchOnOff           00003A58        maincsm_onmessage (main)
                                                   menu_iconhndl (main)
                                                   menu_onkey (main)
                                                   profile_menu_iconhndl (optionMenu)
                                                   profile_menu_onkey (optionMenu)
                                                   savePatchConfig (ptcFileWork)
    -------------------------------------------------------------------------
CODE
  Segment part 116. NOT NEEDED.
    -------------------------------------------------------------------------
CODE
  Relative segment, address: CODE_AREA 00003A80 - 00003ACB (0x4c bytes), align: 2
  Segment part 117.
           ENTRY                   ADDRESS         REF BY
           =====                   =======         ======
           isPatchExistedByID      00003A80        delUnusedConfig (optionMenu)
               stack 1 = 00000000 ( 0000000C )
    -------------------------------------------------------------------------
CODE
  Relative segment, address: CODE_AREA 00003ACC - 00003ACF (0x4 bytes), align: 2
  Segment part 118.           Intra module refs:   doTemplateWork
                                                   fuckThemAll
                                                   getAllPatchData
                                                   getPatchConfigItem
                                                   isPatchExistedByID
                                                   readConfig
                                                   reloadThisPatch
                                                   sortPatchConfigList
    -------------------------------------------------------------------------
CODE
  Segment part 119. NOT NEEDED.Intra module refs   addInfoToPatchInfo
                                                   addPreDataToCBoxItem
                                                   addPrepareData
                                                   addToPatchInfo
                                                   cboxItemColon
                                                   doItemJob
                                                   doSubMenuJob
                                                   doTemplateWork
    -------------------------------------------------------------------------
CODE
  Segment part 120. NOT NEEDED.Intra module refs   addInfoToPatchInfo
                                                   addPreDataToCBoxItem
                                                   addPrepareData
                                                   addToPatchInfo
                                                   cboxItemColon
                                                   doItemJob
                                                   doSubMenuJob
                                                   doTemplateWork
    -------------------------------------------------------------------------
CODE
  Segment part 121. NOT NEEDED.Intra module refs   addInfoToPatchInfo
                                                   addPrepareData
                                                   addToPatchInfo
                                                   cboxItemColon
                                                   doItemJob
                                                   doSubMenuJob
                                                   doTemplateWork
                                                   readConfig
    -------------------------------------------------------------------------
CODE
  Segment part 122. NOT NEEDED.Intra module refs   addToPatchInfo
                                                   doItemJob
                                                   doSubMenuJob
                                                   doTemplateWork
                                                   readConfig
    -------------------------------------------------------------------------
CODE
  Segment part 123. NOT NEEDED.Intra module refs   addInfoToPatchInfo
                                                   addPreDataToCBoxItem
                                                   addPrepareData
                                                   addToPatchInfo
                                                   cboxItemColon
                                                   doItemJob
                                                   doSubMenuJob
                                                   doTemplateWork
                                                   isCurrectItem
                                                   readConfig
    -------------------------------------------------------------------------
CODE
  Segment part 124. NOT NEEDED.Intra module refs   addToPatchInfo
                                                   doItemJob
                                                   readConfig
    -------------------------------------------------------------------------
CODE
  Segment part 125. NOT NEEDED.Intra module refs   addItemToConfig
                                                   addPrepareData
    -------------------------------------------------------------------------
CODE
  Segment part 126. NOT NEEDED.Intra module refs   addPrepareData
                                                   cboxItemColon
                                                   doSubMenuJob
                                                   doTemplateWork
                                                   readConfig
    -------------------------------------------------------------------------
CODE
  Segment part 127. NOT NEEDED.Intra module refs   addPrepareData
                                                   cboxItemColon
    -------------------------------------------------------------------------
CODE
  Segment part 128. NOT NEEDED.Intra module refs   addPrepareData
                                                   cboxItemColon
                                                   doItemJob
    -------------------------------------------------------------------------
CODE
  Segment part 129. NOT NEEDED.Intra module refs   addPreDataToCBoxItem
                                                   findTemplate
                                                   isPatchExistedByID
                                                   sortPatchConfigList
    -------------------------------------------------------------------------
CODE
  Segment part 130. NOT NEEDED.Intra module refs   isCurrectItem
    -------------------------------------------------------------------------
CODE
  Segment part 131. NOT NEEDED.Intra module refs   doItemJob
    -------------------------------------------------------------------------
CODE
  Segment part 132. NOT NEEDED.Intra module refs   doItemJob
    -------------------------------------------------------------------------
CODE
  Segment part 133. NOT NEEDED.Intra module refs   doItemJob
    -------------------------------------------------------------------------
CODE
  Segment part 134. NOT NEEDED.Intra module refs   doItemJob
    -------------------------------------------------------------------------
CODE
  Segment part 135. NOT NEEDED.Intra module refs   doSubMenuJob
                                                   doTemplateWork
                                                   readConfig
    -------------------------------------------------------------------------
CODE
  Segment part 136. NOT NEEDED.Intra module refs   getAllPatchData
    -------------------------------------------------------------------------
CSTACK
  Segment part 1. NOT NEEDED.
    -------------------------------------------------------------------------
INITTAB
  Relative segment, address: CODE_AREA 00009AF8 - 00009B03 (0xc bytes), align: 2
  Segment part 137. ROOT.
           ENTRY                   ADDRESS         REF BY
           =====                   =======         ======
           ?init?tab?DATA_Z        00009AF8 
    -------------------------------------------------------------------------
DATA_C
  Relative segment, address: CODE_AREA 00008DB0 - 00008DB7 (0x8 bytes), align: 2
  Segment part 2.             Intra module refs:   addToPatchInfo
    -------------------------------------------------------------------------
DATA_C
  Relative segment, address: CODE_AREA 00008DB8 - 00008DBF (0x8 bytes), align: 2
  Segment part 3.             Intra module refs:   readConfig
    -------------------------------------------------------------------------
DATA_C
  Relative segment, address: CODE_AREA 00008DC0 - 00008E3F (0x80 bytes), align: 2
  Segment part 4.             Intra module refs:   loadConfig
    -------------------------------------------------------------------------
DATA_C
  Relative segment, address: CODE_AREA 00008E40 - 00008E47 (0x8 bytes), align: 2
  Segment part 5.             Intra module refs:   loadConfig
    -------------------------------------------------------------------------
DATA_C
  Relative segment, address: CODE_AREA 00008E48 - 00008E53 (0xc bytes), align: 2
  Segment part 6.             Intra module refs:   loadConfig
    -------------------------------------------------------------------------
DATA_C
  Relative segment, address: CODE_AREA 00008E54 - 00008E5B (0x8 bytes), align: 2
  Segment part 7.             Intra module refs:   addToPatchInfo
    -------------------------------------------------------------------------
DATA_C
  Relative segment, address: CODE_AREA 00008E5C - 00008E67 (0xc bytes), align: 2
  Segment part 8.             Intra module refs:   addToPatchInfo
    -------------------------------------------------------------------------
DATA_C
  Segment part 9. NOT NEEDED.
    -------------------------------------------------------------------------
DATA_C
  Relative segment, address: CODE_AREA 00008E68 - 00008E73 (0xc bytes), align: 2
  Segment part 10.            Intra module refs:   addToPatchInfo
    -------------------------------------------------------------------------
DATA_C
  Segment part 11. NOT NEEDED.
    -------------------------------------------------------------------------
DATA_C
  Relative segment, address: CODE_AREA 00008E74 - 00008E7B (0x8 bytes), align: 2
  Segment part 12.            Intra module refs:   readConfig
    -------------------------------------------------------------------------
DATA_C
  Relative segment, address: CODE_AREA 00008E7C - 00008E83 (0x8 bytes), align: 2
  Segment part 13.            Intra module refs:   addToPatchInfo
    -------------------------------------------------------------------------
DATA_C
  Segment part 14. NOT NEEDED.
    -------------------------------------------------------------------------
DATA_C
  Relative segment, address: CODE_AREA 00008E84 - 00008E8B (0x8 bytes), align: 2
  Segment part 15.            Intra module refs:   doItemJob
    -------------------------------------------------------------------------
DATA_C
  Relative segment, address: CODE_AREA 00008E8C - 00008E93 (0x8 bytes), align: 2
  Segment part 16.            Intra module refs:   doItemJob
    -------------------------------------------------------------------------
DATA_C
  Segment part 17. NOT NEEDED.
    -------------------------------------------------------------------------
DATA_C
  Segment part 18. NOT NEEDED.
    -------------------------------------------------------------------------
DATA_C
  Relative segment, address: CODE_AREA 00008E94 - 00008E9F (0xc bytes), align: 2
  Segment part 19.            Intra module refs:   doItemJob
    -------------------------------------------------------------------------
DATA_C
  Relative segment, address: CODE_AREA 00008EA0 - 00008EA7 (0x8 bytes), align: 2
  Segment part 20.            Intra module refs:   doItemJob
    -------------------------------------------------------------------------
DATA_C
  Relative segment, address: CODE_AREA 00008EA8 - 00008EAF (0x8 bytes), align: 2
  Segment part 21.            Intra module refs:   doItemJob
    -------------------------------------------------------------------------
DATA_C
  Segment part 22. NOT NEEDED.
    -------------------------------------------------------------------------
DATA_C
  Relative segment, address: CODE_AREA 00008EB0 - 00008EBB (0xc bytes), align: 2
  Segment part 23.            Intra module refs:   doItemJob
    -------------------------------------------------------------------------
DATA_C
  Relative segment, address: CODE_AREA 00008EBC - 00008EC3 (0x8 bytes), align: 2
  Segment part 24.            Intra module refs:   doItemJob
    -------------------------------------------------------------------------
DATA_C
  Segment part 25. NOT NEEDED.
    -------------------------------------------------------------------------
DATA_C
  Relative segment, address: CODE_AREA 00008EC4 - 00008ECB (0x8 bytes), align: 2
  Segment part 26.            Intra module refs:   doItemJob
    -------------------------------------------------------------------------
DATA_C
  Relative segment, address: CODE_AREA 00008ECC - 00008ED3 (0x8 bytes), align: 2
  Segment part 27.            Intra module refs:   doItemJob
    -------------------------------------------------------------------------
DATA_C
  Relative segment, address: CODE_AREA 00008ED4 - 00008EE3 (0x10 bytes), align: 2
  Segment part 28.            Intra module refs:   doItemJob
    -------------------------------------------------------------------------
DATA_C
  Relative segment, address: CODE_AREA 00008EE4 - 00008EEB (0x8 bytes), align: 2
  Segment part 29.            Intra module refs:   doItemJob
    -------------------------------------------------------------------------
DATA_C
  Relative segment, address: CODE_AREA 00008EEC - 00008EF7 (0xc bytes), align: 2
  Segment part 30.            Intra module refs:   doItemJob
    -------------------------------------------------------------------------
DATA_C
  Segment part 31. NOT NEEDED.
    -------------------------------------------------------------------------
DATA_C
  Relative segment, address: CODE_AREA 00008EF8 - 00008F03 (0xc bytes), align: 2
  Segment part 32.            Intra module refs:   doItemJob
    -------------------------------------------------------------------------
DATA_C
  Segment part 33. NOT NEEDED.
    -------------------------------------------------------------------------
DATA_C
  Relative segment, address: CODE_AREA 00008F04 - 00008F0F (0xc bytes), align: 2
  Segment part 34.            Intra module refs:   doItemJob
    -------------------------------------------------------------------------
DATA_C
  Segment part 35. NOT NEEDED.
    -------------------------------------------------------------------------
DATA_C
  Relative segment, address: CODE_AREA 00008F10 - 00008F17 (0x8 bytes), align: 2
  Segment part 36.            Intra module refs:   doItemJob
    -------------------------------------------------------------------------
DATA_C
  Relative segment, address: CODE_AREA 00008F18 - 00008F1F (0x8 bytes), align: 2
  Segment part 37.            Intra module refs:   doItemJob
    -------------------------------------------------------------------------
DATA_C
  Relative segment, address: CODE_AREA 00008F20 - 00008F27 (0x8 bytes), align: 2
  Segment part 38.            Intra module refs:   readConfig
    -------------------------------------------------------------------------
DATA_C
  Relative segment, address: CODE_AREA 00008F28 - 00008F2F (0x8 bytes), align: 2
  Segment part 39.            Intra module refs:   readConfig
    -------------------------------------------------------------------------
DATA_C
  Segment part 40. NOT NEEDED.
    -------------------------------------------------------------------------
DATA_C
  Segment part 41. NOT NEEDED.
    -------------------------------------------------------------------------
DATA_C
  Segment part 42. NOT NEEDED.

    *************************************************************************

  FILE NAME : F:\SVN\cn\Master\Release_NEWSGOLD\Obj\main.r79
  PROGRAM MODULE, NAME : main

  SEGMENTS IN THE MODULE
  ======================
DATA_Z
  Relative segment, address: CODE_AREA 00015B14 - 00015B17 (0x4 bytes), align: 2
  Segment part 16.            Intra module refs:   Segment part 79
           ENTRY                   ADDRESS         REF BY
           =====                   =======         ======
           ptc_buf                 00015B14        Segment part 25 (ptcFileWork)
    -------------------------------------------------------------------------
DATA_Z
  Relative segment, address: CODE_AREA 00015B18 - 00015B1B (0x4 bytes), align: 2
  Segment part 17.            Intra module refs:   createMainMenu
           ENTRY                   ADDRESS         REF BY
           =====                   =======         ======
           patch_n                 00015B18        Segment part 136 (optionMenu)
                                                   addPatchConfigList (getConfig)
    -------------------------------------------------------------------------
DATA_Z
  Relative segment, address: CODE_AREA 00015B1C - 00015B1F (0x4 bytes), align: 2
  Segment part 18.            Intra module refs:   Segment part 98
           ENTRY                   ADDRESS         REF BY
           =====                   =======         ======
           isSubMenuNeed           00015B1C 
    -------------------------------------------------------------------------
DATA_Z
  Segment part 19. NOT NEEDED.
           ENTRY                   ADDRESS         REF BY
           =====                   =======         ======
           colorEditing            
    -------------------------------------------------------------------------
DATA_Z
  Relative segment, address: CODE_AREA 00015B20 - 00015B23 (0x4 bytes), align: 2
  Segment part 20.            Intra module refs:   Segment part 69
           ENTRY                   ADDRESS         REF BY
           =====                   =======         ======
           PTCFG_CUR               00015B20        Segment part 114 (optionMenu)
    -------------------------------------------------------------------------
DATA_Z
  Relative segment, address: CODE_AREA 00015B24 - 00015B27 (0x4 bytes), align: 2
  Segment part 21.            Intra module refs:   maincsm_oncreate
           ENTRY                   ADDRESS         REF BY
           =====                   =======         ======
           MAIN_GUI_ID             00015B24 
    -------------------------------------------------------------------------
DATA_Z
  Relative segment, address: CODE_AREA 00015B28 - 00015B2B (0x4 bytes), align: 2
  Segment part 22.            Intra module refs:   main
           ENTRY                   ADDRESS         REF BY
           =====                   =======         ======
           MAIN_CSM_ID             00015B28        Segment part 138 (optionMenu)
                                                   Segment part 93 (optionMenu)
    -------------------------------------------------------------------------
DATA_Z
  Segment part 23. NOT NEEDED.
           ENTRY                   ADDRESS         REF BY
           =====                   =======         ======
           MAIN_EDGUI_ID           
    -------------------------------------------------------------------------
DATA_Z
  Relative segment, address: CODE_AREA 00015B2C - 00015B37 (0xc bytes), align: 2
  Segment part 24.            Intra module refs:   Segment part 78
           ENTRY                   ADDRESS         REF BY
           =====                   =======         ======
           S_ICONS                 00015B2C        profile_menu_iconhndl (optionMenu)
    -------------------------------------------------------------------------
DATA_Z
  Relative segment, address: CODE_AREA 00015B38 - 00015B3B (0x4 bytes), align: 2
  Segment part 25.            Intra module refs:   Segment part 103
                                                   Segment part 108
           ENTRY                   ADDRESS         REF BY
           =====                   =======         ======
           ews                     00015B38 
    -------------------------------------------------------------------------
DATA_I
  Relative segment, address: DATA_AREA 00000000 - 00000003 (0x4 bytes), align: 2
  Segment part 26.
           ENTRY                   ADDRESS         REF BY
           =====                   =======         ======
           isRunScanerNeed         00000000        menu_quit_without_rs (optionMenu)
    -------------------------------------------------------------------------
DATA_C
  Relative segment, address: CODE_AREA 00008F30 - 00008F3B (0xc bytes), align: 2
  Segment part 2.             Intra module refs:   on_sdec
    -------------------------------------------------------------------------
DATA_C
  Relative segment, address: CODE_AREA 00008F3C - 00008F43 (0x8 bytes), align: 2
  Segment part 3.             Intra module refs:   menu_sk
    -------------------------------------------------------------------------
DATA_C
  Relative segment, address: CODE_AREA 00008F44 - 00008F4F (0xc bytes), align: 2
  Segment part 4.             Intra module refs:   UpdateCSMname
                                                   menuheader
    -------------------------------------------------------------------------
DATA_C
  Relative segment, address: CODE_AREA 00008F50 - 00008F5F (0x10 bytes), align: 2
  Segment part 5.             Intra module refs:   createEditGui
    -------------------------------------------------------------------------
DATA_C
  Relative segment, address: CODE_AREA 00008F60 - 00008F67 (0x8 bytes), align: 2
  Segment part 6.             Intra module refs:   createEditGui
    -------------------------------------------------------------------------
DATA_C
  Relative segment, address: CODE_AREA 00008F68 - 00008F73 (0xc bytes), align: 2
  Segment part 7.             Intra module refs:   createEditGui
    -------------------------------------------------------------------------
DATA_C
  Relative segment, address: CODE_AREA 00008F74 - 00008F7B (0x8 bytes), align: 2
  Segment part 8.             Intra module refs:   createEditGui
    -------------------------------------------------------------------------
DATA_C
  Relative segment, address: CODE_AREA 00008F7C - 00008F83 (0x8 bytes), align: 2
  Segment part 9.             Intra module refs:   Segment part 113
    -------------------------------------------------------------------------
DATA_C
  Relative segment, address: CODE_AREA 00008F84 - 00008F8F (0xc bytes), align: 2
  Segment part 10.            Intra module refs:   on_sfec
    -------------------------------------------------------------------------
DATA_C
  Relative segment, address: CODE_AREA 00008F90 - 00008F97 (0x8 bytes), align: 2
  Segment part 11.            Intra module refs:   menu_iconhndl
    -------------------------------------------------------------------------
DATA_C
  Relative segment, address: CODE_AREA 00008F98 - 00008F9F (0x8 bytes), align: 2
  Segment part 12.            Intra module refs:   SK_CLOSE
    -------------------------------------------------------------------------
DATA_C
  Relative segment, address: CODE_AREA 00008FA0 - 00008FA7 (0x8 bytes), align: 2
  Segment part 13.            Intra module refs:   SK_BACK
    -------------------------------------------------------------------------
DATA_C
  Relative segment, address: CODE_AREA 00008FA8 - 00008FAF (0x8 bytes), align: 2
  Segment part 14.            Intra module refs:   SK_OK
    -------------------------------------------------------------------------
DATA_C
  Relative segment, address: CODE_AREA 00008FB0 - 00008FB7 (0x8 bytes), align: 2
  Segment part 15.            Intra module refs:   menu_sk
    -------------------------------------------------------------------------
DATA_C
  Relative segment, address: CODE_AREA 00008FB8 - 00008FCB (0x14 bytes), align: 2
  Segment part 28.            Intra module refs:   createMainMenu
           ENTRY                   ADDRESS         REF BY
           =====                   =======         ======
           menuheader              00008FB8 
    -------------------------------------------------------------------------
DATA_C
  Relative segment, address: CODE_AREA 00008FCC - 00008FD7 (0xc bytes), align: 2
  Segment part 29.            Intra module refs:   main_menu
           ENTRY                   ADDRESS         REF BY
           =====                   =======         ======
           menusoftkeys            00008FCC 
    -------------------------------------------------------------------------
DATA_C
  Relative segment, address: CODE_AREA 00008FD8 - 00008FEF (0x18 bytes), align: 2
  Segment part 30.            Intra module refs:   menu_skt
           ENTRY                   ADDRESS         REF BY
           =====                   =======         ======
           menu_sk                 00008FD8 
    -------------------------------------------------------------------------
DATA_C
  Relative segment, address: CODE_AREA 00008FF0 - 00008FF7 (0x8 bytes), align: 2
  Segment part 31.            Intra module refs:   Segment part 46
                                                   main_menu
           ENTRY                   ADDRESS         REF BY
           =====                   =======         ======
           menu_skt                00008FF0 
    -------------------------------------------------------------------------
DATA_Z
  Relative segment, address: CODE_AREA 00015B3C - 00015B3F (0x4 bytes), align: 2
  Segment part 32.            Intra module refs:   Segment part 107
                                                   Segment part 87
           ENTRY                   ADDRESS         REF BY
           =====                   =======         ======
           editItemList            00015B3C 
    -------------------------------------------------------------------------
CODE
  Segment part 47. NOT NEEDED.
    -------------------------------------------------------------------------
CODE
  Relative segment, address: CODE_AREA 00003AD0 - 00003B33 (0x64 bytes), align: 2
  Segment part 48.            Intra module refs:   edOnKey
                                                   menu_onkey
           ENTRY                   ADDRESS         REF BY
           =====                   =======         ======
           pushToItemStack         00003AD0 
               stack 1 = 00000000 ( 00000008 )
    -------------------------------------------------------------------------
CODE
  Segment part 49. NOT NEEDED.
    -------------------------------------------------------------------------
CODE
  Relative segment, address: CODE_AREA 00003B34 - 00003B6B (0x38 bytes), align: 2
  Segment part 50.            Intra module refs:   maincsm_onmessage
           ENTRY                   ADDRESS         REF BY
           =====                   =======         ======
           popItemStack            00003B34 
               stack 1 = 00000000 ( 00000004 )
    -------------------------------------------------------------------------
CODE
  Segment part 51. NOT NEEDED.
    -------------------------------------------------------------------------
CODE
  Relative segment, address: CODE_AREA 00003B6C - 00003B8B (0x20 bytes), align: 2
  Segment part 52.            Intra module refs:   edOnKey
           ENTRY                   ADDRESS         REF BY
           =====                   =======         ======
           updateStackEditCurItem
                                   00003B6C 
    -------------------------------------------------------------------------
CODE
  Segment part 53. NOT NEEDED.
    -------------------------------------------------------------------------
CODE
  Relative segment, address: CODE_AREA 00003B8C - 00003BA3 (0x18 bytes), align: 2
  Segment part 54.            Intra module refs:   menu_onkey
           ENTRY                   ADDRESS         REF BY
           =====                   =======         ======
           updateStackPtcfg        00003B8C 
    -------------------------------------------------------------------------
CODE
  Segment part 55. NOT NEEDED.
    -------------------------------------------------------------------------
CODE
  Relative segment, address: CODE_AREA 00003BA4 - 00003BDB (0x38 bytes), align: 2
  Segment part 56.            Intra module refs:   edGHook
           ENTRY                   ADDRESS         REF BY
           =====                   =======         ======
           isTopSubMenu            00003BA4 
               stack 1 = 00000000 ( 00000004 )
    -------------------------------------------------------------------------
CODE
  Segment part 57. NOT NEEDED.
    -------------------------------------------------------------------------
CODE
  Relative segment, address: CODE_AREA 00003BDC - 00003CC7 (0xec bytes), align: 2
  Segment part 58.            Intra module refs:   main_menu
           ENTRY                   ADDRESS         REF BY
           =====                   =======         ======
           menu_onkey              00003BDC 
               stack 1 = 00000000 ( 00000010 )
    -------------------------------------------------------------------------
CODE
  Segment part 59. NOT NEEDED.
    -------------------------------------------------------------------------
CODE
  Relative segment, address: CODE_AREA 00003CC8 - 00003DA7 (0xe0 bytes), align: 2
  Segment part 60.            Intra module refs:   main_menu
           ENTRY                   ADDRESS         REF BY
           =====                   =======         ======
           menu_iconhndl           00003CC8 
               stack 1 = 00000000 ( 0000001C )
    -------------------------------------------------------------------------
CODE
  Segment part 61. NOT NEEDED.
    -------------------------------------------------------------------------
CODE
  Relative segment, address: CODE_AREA 00003DA8 - 00003DBB (0x14 bytes), align: 2
  Segment part 62.            Intra module refs:   main_menu
           ENTRY                   ADDRESS         REF BY
           =====                   =======         ======
           menu_ghook              00003DA8 
               stack 1 = 00000000 ( 00000004 )
    -------------------------------------------------------------------------
CODE
  Segment part 63. NOT NEEDED.
    -------------------------------------------------------------------------
DATA_C
  Relative segment, address: CODE_AREA 00008FF8 - 00009023 (0x2c bytes), align: 2
  Segment part 33.            Intra module refs:   createMainMenu
           ENTRY                   ADDRESS         REF BY
           =====                   =======         ======
           main_menu               00008FF8 
    -------------------------------------------------------------------------
CODE
  Relative segment, address: CODE_AREA 00003DBC - 00003E2F (0x74 bytes), align: 2
  Segment part 64.            Intra module refs:   maincsm_oncreate
                                                   maincsm_onmessage
           ENTRY                   ADDRESS         REF BY
           =====                   =======         ======
           createMainMenu          00003DBC 
               stack 1 = 00000000 ( 00000018 )
    -------------------------------------------------------------------------
CODE
  Segment part 65. NOT NEEDED.
    -------------------------------------------------------------------------
CODE
  Relative segment, address: CODE_AREA 00003E30 - 00003E4F (0x20 bytes), align: 2
  Segment part 66.            Intra module refs:   MAINCSM
           ENTRY                   ADDRESS         REF BY
           =====                   =======         ======
           maincsm_oncreate        00003E30 
               stack 1 = 00000000 ( 0000000C )
    -------------------------------------------------------------------------
CODE
  Segment part 67. NOT NEEDED.
    -------------------------------------------------------------------------
CODE
  Relative segment, address: CODE_AREA 00003E50 - 00003F5B (0x10c bytes), align: 2
  Segment part 68.            Intra module refs:   MAINCSM
           ENTRY                   ADDRESS         REF BY
           =====                   =======         ======
           maincsm_onmessage       00003E50 
               stack 1 = 00000000 ( 0000000C )
    -------------------------------------------------------------------------
CODE
  Relative segment, address: CODE_AREA 00003F5C - 00003F5F (0x4 bytes), align: 2
  Segment part 69.            Intra module refs:   createMainMenu
                                                   maincsm_onmessage
                                                   menu_onkey
    -------------------------------------------------------------------------
CODE
  Segment part 70. NOT NEEDED.
    -------------------------------------------------------------------------
CODE
  Relative segment, address: CODE_AREA 00003F60 - 00003F9B (0x3c bytes), align: 2
  Segment part 71.            Intra module refs:   Segment part 80
           ENTRY                   ADDRESS         REF BY
           =====                   =======         ======
           Killer                  00003F60 
               stack 1 = 00000000 ( 00000004 )
    -------------------------------------------------------------------------
CODE
  Segment part 72. NOT NEEDED.
    -------------------------------------------------------------------------
CODE
  Relative segment, address: CODE_AREA 00003F9C - 00003FAB (0x10 bytes), align: 2
  Segment part 73.            Intra module refs:   MAINCSM
           ENTRY                   ADDRESS         REF BY
           =====                   =======         ======
           maincsm_onclose         00003F9C 
               stack 1 = 00000000 ( 00000004 )
    -------------------------------------------------------------------------
CODE
  Segment part 74. NOT NEEDED.
    -------------------------------------------------------------------------
DATA_C
  Relative segment, address: CODE_AREA 00009024 - 00009027 (0x4 bytes), align: 2
  Segment part 34.            Intra module refs:   MAINCSM
           ENTRY                   ADDRESS         REF BY
           =====                   =======         ======
           minus11                 00009024 
    -------------------------------------------------------------------------
DATA_C
  Relative segment, address: CODE_AREA 00009028 - 0000913F (0x118 bytes), align: 2
  Segment part 35.            Intra module refs:   MAINCSM
           ENTRY                   ADDRESS         REF BY
           =====                   =======         ======
           maincsm_name_body       00009028 
    -------------------------------------------------------------------------
DATA_C
  Relative segment, address: CODE_AREA 00009140 - 0000917B (0x3c bytes), align: 2
  Segment part 36.            Intra module refs:   UpdateCSMname
                                                   main
           ENTRY                   ADDRESS         REF BY
           =====                   =======         ======
           MAINCSM                 00009140 
    -------------------------------------------------------------------------
CODE
  Relative segment, address: CODE_AREA 00003FAC - 00003FC7 (0x1c bytes), align: 2
  Segment part 75.            Intra module refs:   main
           ENTRY                   ADDRESS         REF BY
           =====                   =======         ======
           UpdateCSMname           00003FAC 
               stack 1 = 00000000 ( 00000004 )
    -------------------------------------------------------------------------
CODE
  Segment part 76. NOT NEEDED.
    -------------------------------------------------------------------------
CODE
  Relative segment, address: CODE_AREA 00003FC8 - 00004073 (0xac bytes), align: 2
  Segment part 77.
           ENTRY                   ADDRESS         REF BY
           =====                   =======         ======
           main                    00003FC8        Absolute parts (?ABS_ENTRY_MOD)
               stack 1 = 00000000 ( 00000034 )
    -------------------------------------------------------------------------
CODE
  Relative segment, address: CODE_AREA 00004074 - 00004077 (0x4 bytes), align: 2
  Segment part 78.            Intra module refs:   main
                                                   menu_iconhndl
    -------------------------------------------------------------------------
CODE
  Relative segment, address: CODE_AREA 00004078 - 0000407B (0x4 bytes), align: 2
  Segment part 79.            Intra module refs:   Killer
                                                   main
    -------------------------------------------------------------------------
CODE
  Relative segment, address: CODE_AREA 0000407C - 0000407F (0x4 bytes), align: 2
  Segment part 80.            Intra module refs:   main
                                                   maincsm_onclose
    -------------------------------------------------------------------------
CODE
  Segment part 81. NOT NEEDED.
    -------------------------------------------------------------------------
DATA_Z
  Relative segment, address: CODE_AREA 00015B40 - 00015BBF (0x80 bytes), align: 2
  Segment part 37.            Intra module refs:   Segment part 39
                                                   updateEdHdr
           ENTRY                   ADDRESS         REF BY
           =====                   =======         ======
           ED_HDR_BODY             00015B40 
    -------------------------------------------------------------------------
DATA_I
  Relative segment, address: DATA_AREA 00000004 - 00000017 (0x14 bytes), align: 2
  Segment part 38.            Intra module refs:   createEditGui
           ENTRY                   ADDRESS         REF BY
           =====                   =======         ======
           ED_HDR                  00000004 
    -------------------------------------------------------------------------
CODE
  Relative segment, address: CODE_AREA 00004080 - 000040EB (0x6c bytes), align: 2
  Segment part 82.            Intra module refs:   edGHook
                                                   edOnKey
           ENTRY                   ADDRESS         REF BY
           =====                   =======         ======
           findPatchItemInED       00004080 
    -------------------------------------------------------------------------
CODE
  Segment part 83. NOT NEEDED.
    -------------------------------------------------------------------------
CODE
  Relative segment, address: CODE_AREA 000040EC - 0000419B (0xb0 bytes), align: 2
  Segment part 84.            Intra module refs:   edOnKey
           ENTRY                   ADDRESS         REF BY
           =====                   =======         ======
           getMaxFocus             000040EC 
    -------------------------------------------------------------------------
CODE
  Segment part 85. NOT NEEDED.
    -------------------------------------------------------------------------
CODE
  Relative segment, address: CODE_AREA 0000419C - 000041F7 (0x5c bytes), align: 2
  Segment part 86.            Intra module refs:   edOnKey
           ENTRY                   ADDRESS         REF BY
           =====                   =======         ======
           getMinFocus             0000419C 
    -------------------------------------------------------------------------
CODE
  Relative segment, address: CODE_AREA 000041F8 - 000041FB (0x4 bytes), align: 2
  Segment part 87.            Intra module refs:   findPatchItemInED
                                                   getMaxFocus
                                                   getMinFocus
                                                   isTopSubMenu
                                                   maincsm_onmessage
                                                   popItemStack
                                                   pushToItemStack
                                                   updateStackEditCurItem
                                                   updateStackPtcfg
    -------------------------------------------------------------------------
CODE
  Segment part 88. NOT NEEDED.
    -------------------------------------------------------------------------
CODE
  Relative segment, address: CODE_AREA 000041FC - 00004257 (0x5c bytes), align: 2
  Segment part 89.            Intra module refs:   createEditGui
           ENTRY                   ADDRESS         REF BY
           =====                   =======         ======
           updateEdHdr             000041FC 
               stack 1 = 00000000 ( 00000010 )
    -------------------------------------------------------------------------
CODE
  Segment part 90. NOT NEEDED.
    -------------------------------------------------------------------------
CODE
  Relative segment, address: CODE_AREA 00004258 - 0000425B (0x4 bytes), align: 2
  Segment part 91.            Intra module refs:   Segment part 46
           ENTRY                   ADDRESS         REF BY
           =====                   =======         ======
           ed_locret               00004258 
    -------------------------------------------------------------------------
CODE
  Segment part 92. NOT NEEDED.
    -------------------------------------------------------------------------
DATA_Z
  Relative segment, address: CODE_AREA 00015BC0 - 00015BC3 (0x4 bytes), align: 2
  Segment part 40.            Intra module refs:   Segment part 99
           ENTRY                   ADDRESS         REF BY
           =====                   =======         ======
           sfItemTemp              00015BC0 
    -------------------------------------------------------------------------
CODE
  Relative segment, address: CODE_AREA 0000425C - 000042DB (0x80 bytes), align: 2
  Segment part 93.            Intra module refs:   edOnKey
           ENTRY                   ADDRESS         REF BY
           =====                   =======         ======
           on_sfec                 0000425C 
               stack 1 = 00000000 ( 00000010 )
    -------------------------------------------------------------------------
CODE
  Segment part 94. NOT NEEDED.
    -------------------------------------------------------------------------
CODE
  Relative segment, address: CODE_AREA 000042DC - 00004333 (0x58 bytes), align: 2
  Segment part 95.            Intra module refs:   edOnKey
           ENTRY                   ADDRESS         REF BY
           =====                   =======         ======
           on_sdec                 000042DC        pathInputOnKey (optionMenu)
               stack 1 = 00000000 ( 00000008 )
    -------------------------------------------------------------------------
CODE
  Segment part 96. NOT NEEDED.
    -------------------------------------------------------------------------
CODE
  Relative segment, address: CODE_AREA 00004334 - 00004743 (0x410 bytes), align: 2
  Segment part 97.            Intra module refs:   Segment part 46
           ENTRY                   ADDRESS         REF BY
           =====                   =======         ======
           edOnKey                 00004334 
               stack 1 = 00000000 ( 00000250 )
    -------------------------------------------------------------------------
CODE
  Relative segment, address: CODE_AREA 00004744 - 00004747 (0x4 bytes), align: 2
  Segment part 98.            Intra module refs:   edOnKey
                                                   maincsm_onmessage
                                                   menu_onkey
    -------------------------------------------------------------------------
CODE
  Relative segment, address: CODE_AREA 00004748 - 0000474B (0x4 bytes), align: 2
  Segment part 99.            Intra module refs:   edOnKey
                                                   on_sfec
    -------------------------------------------------------------------------
CODE
  Relative segment, address: CODE_AREA 0000474C - 0000474F (0x4 bytes), align: 2
  Segment part 100.           Intra module refs:   edOnKey
                                                   menu_iconhndl
                                                   on_sdec
                                                   on_sfec
    -------------------------------------------------------------------------
CODE
  Segment part 101. NOT NEEDED.
    -------------------------------------------------------------------------
DATA_C
  Relative segment, address: CODE_AREA 0000917C - 00009183 (0x8 bytes), align: 2
  Segment part 41.            Intra module refs:   edGHook
           ENTRY                   ADDRESS         REF BY
           =====                   =======         ======
           SK_OK                   0000917C 
    -------------------------------------------------------------------------
DATA_C
  Relative segment, address: CODE_AREA 00009184 - 0000918B (0x8 bytes), align: 2
  Segment part 42.            Intra module refs:   edGHook
           ENTRY                   ADDRESS         REF BY
           =====                   =======         ======
           SK_BACK                 00009184 
    -------------------------------------------------------------------------
DATA_C
  Relative segment, address: CODE_AREA 0000918C - 00009193 (0x8 bytes), align: 2
  Segment part 43.            Intra module refs:   edGHook
           ENTRY                   ADDRESS         REF BY
           =====                   =======         ======
           SK_CLOSE                0000918C 
    -------------------------------------------------------------------------
DATA_C
  Relative segment, address: CODE_AREA 00009194 - 00009197 (0x4 bytes), align: 2
  Segment part 44.            Intra module refs:   Segment part 109
           ENTRY                   ADDRESS         REF BY
           =====                   =======         ======
           PT_PTM_FMT              00009194 
    -------------------------------------------------------------------------
CODE
  Relative segment, address: CODE_AREA 00004750 - 00004C53 (0x504 bytes), align: 2
  Segment part 102.           Intra module refs:   Segment part 46
           ENTRY                   ADDRESS         REF BY
           =====                   =======         ======
           edGHook                 00004750 
               stack 1 = 00000000 ( 000002C4 )
    -------------------------------------------------------------------------
CODE
  Relative segment, address: CODE_AREA 00004C54 - 00004C57 (0x4 bytes), align: 2
  Segment part 103.           Intra module refs:   Killer
                                                   edGHook
                                                   edOnKey
                                                   main
    -------------------------------------------------------------------------
CODE
  Relative segment, address: CODE_AREA 00004C58 - 00004C5B (0x4 bytes), align: 2
  Segment part 104.           Intra module refs:   edGHook
                                                   edOnKey
    -------------------------------------------------------------------------
CODE
  Segment part 105. NOT NEEDED.
    -------------------------------------------------------------------------
DATA_I
  Relative segment, address: DATA_AREA 00000018 - 0000004F (0x38 bytes), align: 2
  Segment part 45.            Intra module refs:   createEditGui
           ENTRY                   ADDRESS         REF BY
           =====                   =======         ======
           ED_DESC                 00000018 
    -------------------------------------------------------------------------
CODE
  Relative segment, address: CODE_AREA 00004C5C - 000054BB (0x860 bytes), align: 2
  Segment part 106.           Intra module refs:   maincsm_onmessage
           ENTRY                   ADDRESS         REF BY
           =====                   =======         ======
           createEditGui           00004C5C 
               stack 1 = 00000000 ( 000002A8 )
    -------------------------------------------------------------------------
CODE
  Relative segment, address: CODE_AREA 000054BC - 000054BF (0x4 bytes), align: 2
  Segment part 107.           Intra module refs:   createEditGui
                                                   edGHook
    -------------------------------------------------------------------------
CODE
  Relative segment, address: CODE_AREA 000054C0 - 000054C3 (0x4 bytes), align: 2
  Segment part 108.           Intra module refs:   createEditGui
    -------------------------------------------------------------------------
CODE
  Relative segment, address: CODE_AREA 000054C4 - 000054C7 (0x4 bytes), align: 2
  Segment part 109.           Intra module refs:   createEditGui
                                                   edGHook
    -------------------------------------------------------------------------
CODE
  Relative segment, address: CODE_AREA 000054C8 - 000054CB (0x4 bytes), align: 2
  Segment part 110.           Intra module refs:   createEditGui
                                                   edGHook
    -------------------------------------------------------------------------
CODE
  Relative segment, address: CODE_AREA 000054CC - 000054CF (0x4 bytes), align: 2
  Segment part 111.           Intra module refs:   createEditGui
                                                   edGHook
    -------------------------------------------------------------------------
CODE
  Relative segment, address: CODE_AREA 000054D0 - 000054D3 (0x4 bytes), align: 2
  Segment part 112.           Intra module refs:   createEditGui
                                                   edGHook
    -------------------------------------------------------------------------
CODE
  Relative segment, address: CODE_AREA 000054D4 - 000054D7 (0x4 bytes), align: 2
  Segment part 113.           Intra module refs:   createEditGui
                                                   edGHook
                                                   edOnKey
    -------------------------------------------------------------------------
CODE
  Relative segment, address: CODE_AREA 000054D8 - 000054DB (0x4 bytes), align: 2
  Segment part 114.           Intra module refs:   createEditGui
    -------------------------------------------------------------------------
CODE
  Segment part 115. NOT NEEDED.Intra module refs   menu_onkey
    -------------------------------------------------------------------------
CODE
  Segment part 116. NOT NEEDED.Intra module refs   maincsm_onmessage
                                                   menu_iconhndl
                                                   menu_onkey
    -------------------------------------------------------------------------
CODE
  Segment part 117. NOT NEEDED.Intra module refs   maincsm_onmessage
                                                   menu_onkey
    -------------------------------------------------------------------------
CODE
  Segment part 118. NOT NEEDED.Intra module refs   maincsm_onmessage
                                                   menu_iconhndl
                                                   menu_onkey
    -------------------------------------------------------------------------
CODE
  Segment part 119. NOT NEEDED.Intra module refs   menu_onkey
    -------------------------------------------------------------------------
CODE
  Segment part 120. NOT NEEDED.Intra module refs   createEditGui
                                                   edGHook
                                                   menu_iconhndl
                                                   updateEdHdr
    -------------------------------------------------------------------------
CODE
  Segment part 121. NOT NEEDED.Intra module refs   createEditGui
                                                   edGHook
                                                   menu_iconhndl
                                                   updateEdHdr
    -------------------------------------------------------------------------
CODE
  Segment part 122. NOT NEEDED.Intra module refs   Killer
    -------------------------------------------------------------------------
CODE
  Segment part 123. NOT NEEDED.Intra module refs   Killer
    -------------------------------------------------------------------------
CODE
  Segment part 124. NOT NEEDED.Intra module refs   Killer
    -------------------------------------------------------------------------
CODE
  Segment part 125. NOT NEEDED.Intra module refs   main
    -------------------------------------------------------------------------
CODE
  Segment part 126. NOT NEEDED.Intra module refs   on_sdec
                                                   on_sfec
    -------------------------------------------------------------------------
CODE
  Segment part 127. NOT NEEDED.Intra module refs   edOnKey
    -------------------------------------------------------------------------
CODE
  Segment part 128. NOT NEEDED.Intra module refs   edOnKey
    -------------------------------------------------------------------------
CODE
  Segment part 129. NOT NEEDED.Intra module refs   edGHook
    -------------------------------------------------------------------------
CODE
  Segment part 130. NOT NEEDED.Intra module refs   edGHook
    -------------------------------------------------------------------------
CODE
  Segment part 131. NOT NEEDED.Intra module refs   edGHook
    -------------------------------------------------------------------------
CODE
  Segment part 132. NOT NEEDED.Intra module refs   edGHook
    -------------------------------------------------------------------------
CODE
  Segment part 133. NOT NEEDED.Intra module refs   edGHook
    -------------------------------------------------------------------------
CODE
  Segment part 134. NOT NEEDED.Intra module refs   edGHook
    -------------------------------------------------------------------------
CODE
  Segment part 135. NOT NEEDED.Intra module refs   edGHook
    -------------------------------------------------------------------------
CODE
  Segment part 136. NOT NEEDED.Intra module refs   createEditGui
    -------------------------------------------------------------------------
CODE
  Segment part 137. NOT NEEDED.Intra module refs   createEditGui
    -------------------------------------------------------------------------
CODE
  Segment part 138. NOT NEEDED.Intra module refs   createEditGui
    -------------------------------------------------------------------------
CODE
  Segment part 139. NOT NEEDED.Intra module refs   createEditGui
    -------------------------------------------------------------------------
CODE
  Segment part 140. NOT NEEDED.Intra module refs   createEditGui
    -------------------------------------------------------------------------
CODE
  Segment part 141. NOT NEEDED.Intra module refs   createEditGui
    -------------------------------------------------------------------------
CODE
  Segment part 142. NOT NEEDED.Intra module refs   createEditGui
    -------------------------------------------------------------------------
CSTACK
  Segment part 1. NOT NEEDED.
    -------------------------------------------------------------------------
DATA_ID
  Relative segment, address: CODE_AREA 00000000 - 00000003 (0x4 bytes), align: 2
  Segment part 27.            Intra module refs:   isRunScanerNeed
    -------------------------------------------------------------------------
DATA_ID
  Relative segment, address: CODE_AREA 00000004 - 00000017 (0x14 bytes), align: 2
  Segment part 39.            Intra module refs:   ED_HDR
    -------------------------------------------------------------------------
DATA_ID
  Relative segment, address: CODE_AREA 00000018 - 0000004F (0x38 bytes), align: 2
  Segment part 46.            Intra module refs:   ED_DESC
    -------------------------------------------------------------------------
DATA_ID
  Segment part 143. NOT NEEDED.
           ENTRY                   ADDRESS         REF BY
           =====                   =======         ======
           ?*?DATA_ID              
    -------------------------------------------------------------------------
INITTAB
  Relative segment, address: CODE_AREA 00009B04 - 00009B0F (0xc bytes), align: 2
  Segment part 144. ROOT.
           ENTRY                   ADDRESS         REF BY
           =====                   =======         ======
           ?init?tab?DATA_I        00009B04 
    -------------------------------------------------------------------------
INITTAB
  Segment part 145. TENTATIVE. Used definition from getConfig
           ENTRY                   ADDRESS         REF BY
           =====                   =======         ======
           ?init?tab?DATA_Z        

    *************************************************************************

  FILE NAME : F:\SVN\cn\Master\Release_NEWSGOLD\Obj\optionMenu.r79
  PROGRAM MODULE, NAME : optionMenu

  SEGMENTS IN THE MODULE
  ======================
DATA_Z
  Relative segment, address: CODE_AREA 00015BC4 - 00015BC7 (0x4 bytes), align: 2
  Segment part 42.            Intra module refs:   Segment part 123
           ENTRY                   ADDRESS         REF BY
           =====                   =======         ======
           PATH_TYPE               00015BC4 
    -------------------------------------------------------------------------
DATA_C
  Relative segment, address: CODE_AREA 00009198 - 0000919F (0x8 bytes), align: 2
  Segment part 2.             Intra module refs:   Segment part 130
    -------------------------------------------------------------------------
DATA_C
  Relative segment, address: CODE_AREA 000091A0 - 000091A7 (0x8 bytes), align: 2
  Segment part 3.             Intra module refs:   Segment part 133
    -------------------------------------------------------------------------
DATA_C
  Relative segment, address: CODE_AREA 000091A8 - 000091BB (0x14 bytes), align: 2
  Segment part 4.             Intra module refs:   Segment part 137
    -------------------------------------------------------------------------
DATA_C
  Relative segment, address: CODE_AREA 000091BC - 000091C7 (0xc bytes), align: 2
  Segment part 5.             Intra module refs:   deleteThis
    -------------------------------------------------------------------------
DATA_C
  Relative segment, address: CODE_AREA 000091C8 - 000091DB (0x14 bytes), align: 2
  Segment part 6.             Intra module refs:   Segment part 125
    -------------------------------------------------------------------------
DATA_C
  Relative segment, address: CODE_AREA 000091DC - 000091E3 (0x8 bytes), align: 2
  Segment part 7.             Intra module refs:   profile_menu_iconhndl
    -------------------------------------------------------------------------
DATA_C
  Relative segment, address: CODE_AREA 000091E4 - 00009263 (0x80 bytes), align: 2
  Segment part 8.             Intra module refs:   delUnusedConfig
    -------------------------------------------------------------------------
DATA_C
  Relative segment, address: CODE_AREA 00009264 - 0000926B (0x8 bytes), align: 2
  Segment part 9.             Intra module refs:   option_menu_ITEMS
                                                   option_menu_ITEMS_1
    -------------------------------------------------------------------------
DATA_C
  Relative segment, address: CODE_AREA 0000926C - 00009273 (0x8 bytes), align: 2
  Segment part 10.            Intra module refs:   showPatchInfo
    -------------------------------------------------------------------------
DATA_C
  Relative segment, address: CODE_AREA 00009274 - 0000927B (0x8 bytes), align: 2
  Segment part 11.            Intra module refs:   showPatchInfo
    -------------------------------------------------------------------------
DATA_C
  Relative segment, address: CODE_AREA 0000927C - 00009283 (0x8 bytes), align: 2
  Segment part 12.            Intra module refs:   showPatchInfo
    -------------------------------------------------------------------------
DATA_C
  Segment part 13. NOT NEEDED.
    -------------------------------------------------------------------------
DATA_C
  Relative segment, address: CODE_AREA 00009284 - 0000928B (0x8 bytes), align: 2
  Segment part 14.            Intra module refs:   showPatchInfo
    -------------------------------------------------------------------------
DATA_C
  Relative segment, address: CODE_AREA 0000928C - 00009297 (0xc bytes), align: 2
  Segment part 15.            Intra module refs:   showPatchInfo
    -------------------------------------------------------------------------
DATA_C
  Relative segment, address: CODE_AREA 00009298 - 000092A7 (0x10 bytes), align: 2
  Segment part 16.            Intra module refs:   pathInputDlg
    -------------------------------------------------------------------------
DATA_C
  Relative segment, address: CODE_AREA 000092A8 - 000092C7 (0x20 bytes), align: 2
  Segment part 17.            Intra module refs:   pathInputDlg
    -------------------------------------------------------------------------
DATA_C
  Relative segment, address: CODE_AREA 000092C8 - 00009347 (0x80 bytes), align: 2
  Segment part 18.            Intra module refs:   configBackUp
    -------------------------------------------------------------------------
DATA_C
  Relative segment, address: CODE_AREA 00009348 - 0000934F (0x8 bytes), align: 2
  Segment part 19.            Intra module refs:   Segment part 135
    -------------------------------------------------------------------------
DATA_C
  Relative segment, address: CODE_AREA 00009350 - 000093CF (0x80 bytes), align: 2
  Segment part 20.            Intra module refs:   configRestore
    -------------------------------------------------------------------------
DATA_C
  Relative segment, address: CODE_AREA 000093D0 - 000093D7 (0x8 bytes), align: 2
  Segment part 21.            Intra module refs:   configRestore
    -------------------------------------------------------------------------
DATA_C
  Relative segment, address: CODE_AREA 000093D8 - 000093E3 (0xc bytes), align: 2
  Segment part 22.            Intra module refs:   configRestore
    -------------------------------------------------------------------------
DATA_C
  Relative segment, address: CODE_AREA 000093E4 - 000093EB (0x8 bytes), align: 2
  Segment part 23.            Intra module refs:   mmenu_sk
    -------------------------------------------------------------------------
DATA_C
  Relative segment, address: CODE_AREA 000093EC - 000093F3 (0x8 bytes), align: 2
  Segment part 24.            Intra module refs:   mmenu_sk
    -------------------------------------------------------------------------
DATA_C
  Relative segment, address: CODE_AREA 000093F4 - 000093FF (0xc bytes), align: 2
  Segment part 25.            Intra module refs:   option_menu_ITEMS
                                                   profile_menu_header
    -------------------------------------------------------------------------
DATA_C
  Relative segment, address: CODE_AREA 00009400 - 0000940B (0xc bytes), align: 2
  Segment part 26.            Intra module refs:   Segment part 58
                                                   option_menu_ITEMS
                                                   option_menu_ITEMS_1
    -------------------------------------------------------------------------
DATA_C
  Relative segment, address: CODE_AREA 0000940C - 0000941B (0x10 bytes), align: 2
  Segment part 27.            Intra module refs:   option_menu_ITEMS
                                                   option_menu_ITEMS_1
    -------------------------------------------------------------------------
DATA_C
  Relative segment, address: CODE_AREA 0000941C - 0000942B (0x10 bytes), align: 2
  Segment part 28.            Intra module refs:   option_menu_ITEMS
                                                   option_menu_ITEMS_1
    -------------------------------------------------------------------------
DATA_C
  Relative segment, address: CODE_AREA 0000942C - 0000943B (0x10 bytes), align: 2
  Segment part 29.            Intra module refs:   option_menu_ITEMS
                                                   option_menu_ITEMS_1
    -------------------------------------------------------------------------
DATA_C
  Relative segment, address: CODE_AREA 0000943C - 00009447 (0xc bytes), align: 2
  Segment part 30.            Intra module refs:   SK_BACKUP
                                                   option_menu_ITEMS
                                                   option_menu_ITEMS_1
    -------------------------------------------------------------------------
DATA_C
  Relative segment, address: CODE_AREA 00009448 - 00009453 (0xc bytes), align: 2
  Segment part 31.            Intra module refs:   SK_RESTORE
                                                   option_menu_ITEMS
                                                   option_menu_ITEMS_1
    -------------------------------------------------------------------------
DATA_C
  Relative segment, address: CODE_AREA 00009454 - 00009463 (0x10 bytes), align: 2
  Segment part 32.            Intra module refs:   pathInputDlg
    -------------------------------------------------------------------------
DATA_C
  Relative segment, address: CODE_AREA 00009464 - 00009473 (0x10 bytes), align: 2
  Segment part 33.            Intra module refs:   option_menu_ITEMS
                                                   option_menu_ITEMS_1
    -------------------------------------------------------------------------
DATA_C
  Relative segment, address: CODE_AREA 00009474 - 0000947B (0x8 bytes), align: 2
  Segment part 34.            Intra module refs:   option_menu_ITEMS
                                                   option_menu_ITEMS_1
    -------------------------------------------------------------------------
DATA_C
  Relative segment, address: CODE_AREA 0000947C - 00009483 (0x8 bytes), align: 2
  Segment part 35.            Intra module refs:   option_menu_header
    -------------------------------------------------------------------------
DATA_C
  Relative segment, address: CODE_AREA 00009484 - 0000948B (0x8 bytes), align: 2
  Segment part 36.            Intra module refs:   profile_menu_sk
    -------------------------------------------------------------------------
DATA_C
  Relative segment, address: CODE_AREA 0000948C - 00009493 (0x8 bytes), align: 2
  Segment part 37.            Intra module refs:   profile_menu_sk
    -------------------------------------------------------------------------
DATA_C
  Relative segment, address: CODE_AREA 00009494 - 000094A3 (0x10 bytes), align: 2
  Segment part 38.            Intra module refs:   Segment part 66
    -------------------------------------------------------------------------
DATA_C
  Relative segment, address: CODE_AREA 000094A4 - 000094E7 (0x44 bytes), align: 2
  Segment part 39.            Intra module refs:   menu_about
    -------------------------------------------------------------------------
DATA_C
  Relative segment, address: CODE_AREA 000094E8 - 00009567 (0x80 bytes), align: 2
  Segment part 40.            Intra module refs:   deleteAllConfig
    -------------------------------------------------------------------------
DATA_C
  Relative segment, address: CODE_AREA 00009568 - 0000956F (0x8 bytes), align: 2
  Segment part 41.            Intra module refs:   Segment part 134
    -------------------------------------------------------------------------
DATA_C
  Relative segment, address: CODE_AREA 00009570 - 0000957B (0xc bytes), align: 2
  Segment part 43.            Intra module refs:   option_menu
                                                   option_menu_1
                                                   profile_menu
           ENTRY                   ADDRESS         REF BY
           =====                   =======         ======
           mmenusoftkeys           00009570 
    -------------------------------------------------------------------------
DATA_C
  Relative segment, address: CODE_AREA 0000957C - 00009593 (0x18 bytes), align: 2
  Segment part 44.            Intra module refs:   mmenu_skt
           ENTRY                   ADDRESS         REF BY
           =====                   =======         ======
           mmenu_sk                0000957C 
    -------------------------------------------------------------------------
DATA_C
  Relative segment, address: CODE_AREA 00009594 - 0000959B (0x8 bytes), align: 2
  Segment part 45.            Intra module refs:   Segment part 60
                                                   Segment part 64
                                                   option_menu
                                                   option_menu_1
           ENTRY                   ADDRESS         REF BY
           =====                   =======         ======
           mmenu_skt               00009594 
    -------------------------------------------------------------------------
CODE
  Segment part 67. NOT NEEDED.
    -------------------------------------------------------------------------
CODE
  Relative segment, address: CODE_AREA 000054DC - 000054EF (0x14 bytes), align: 2
  Segment part 68.            Intra module refs:   option_menu
                                                   option_menu_1
           ENTRY                   ADDRESS         REF BY
           =====                   =======         ======
           option_menu_ghook       000054DC 
               stack 1 = 00000000 ( 00000004 )
    -------------------------------------------------------------------------
CODE
  Segment part 69. NOT NEEDED.
    -------------------------------------------------------------------------
CODE
  Relative segment, address: CODE_AREA 000054F0 - 0000550B (0x1c bytes), align: 2
  Segment part 70.            Intra module refs:   option_menu_HNDLS
                                                   option_menu_HNDLS_1
           ENTRY                   ADDRESS         REF BY
           =====                   =======         ======
           menu_exit               000054F0 
               stack 1 = 00000000 ( 00000004 )
    -------------------------------------------------------------------------
CODE
  Segment part 71. NOT NEEDED.
    -------------------------------------------------------------------------
CODE
  Relative segment, address: CODE_AREA 0000550C - 0000552B (0x20 bytes), align: 2
  Segment part 72.            Intra module refs:   option_menu_HNDLS
                                                   option_menu_HNDLS_1
           ENTRY                   ADDRESS         REF BY
           =====                   =======         ======
           menu_about              0000550C 
               stack 1 = 00000000 ( 00000004 )
    -------------------------------------------------------------------------
CODE
  Segment part 73. NOT NEEDED.
    -------------------------------------------------------------------------
CODE
  Relative segment, address: CODE_AREA 0000552C - 0000553F (0x14 bytes), align: 2
  Segment part 74.            Intra module refs:   option_menu_HNDLS
           ENTRY                   ADDRESS         REF BY
           =====                   =======         ======
           menu_profile            0000552C 
               stack 1 = 00000000 ( 00000004 )
    -------------------------------------------------------------------------
CODE
  Segment part 75. NOT NEEDED.
    -------------------------------------------------------------------------
CODE
  Relative segment, address: CODE_AREA 00005540 - 00005553 (0x14 bytes), align: 2
  Segment part 76.            Intra module refs:   option_menu_HNDLS
                                                   option_menu_HNDLS_1
           ENTRY                   ADDRESS         REF BY
           =====                   =======         ======
           menu_del_all            00005540 
               stack 1 = 00000000 ( 00000004 )
    -------------------------------------------------------------------------
CODE
  Segment part 77. NOT NEEDED.
    -------------------------------------------------------------------------
CODE
  Relative segment, address: CODE_AREA 00005554 - 00005567 (0x14 bytes), align: 2
  Segment part 78.            Intra module refs:   option_menu_HNDLS
                                                   option_menu_HNDLS_1
           ENTRY                   ADDRESS         REF BY
           =====                   =======         ======
           menu_del_this           00005554 
               stack 1 = 00000000 ( 00000004 )
    -------------------------------------------------------------------------
CODE
  Segment part 79. NOT NEEDED.
    -------------------------------------------------------------------------
CODE
  Relative segment, address: CODE_AREA 00005568 - 0000557B (0x14 bytes), align: 2
  Segment part 80.            Intra module refs:   option_menu_HNDLS
                                                   option_menu_HNDLS_1
           ENTRY                   ADDRESS         REF BY
           =====                   =======         ======
           menu_del_unused         00005568 
               stack 1 = 00000000 ( 00000004 )
    -------------------------------------------------------------------------
CODE
  Segment part 81. NOT NEEDED.
    -------------------------------------------------------------------------
CODE
  Relative segment, address: CODE_AREA 0000557C - 0000558F (0x14 bytes), align: 2
  Segment part 82.            Intra module refs:   option_menu_HNDLS
                                                   option_menu_HNDLS_1
           ENTRY                   ADDRESS         REF BY
           =====                   =======         ======
           menu_info               0000557C 
               stack 1 = 00000000 ( 00000004 )
    -------------------------------------------------------------------------
CODE
  Segment part 83. NOT NEEDED.
    -------------------------------------------------------------------------
CODE
  Relative segment, address: CODE_AREA 00005590 - 000055AF (0x20 bytes), align: 2
  Segment part 84.            Intra module refs:   option_menu_HNDLS
                                                   option_menu_HNDLS_1
           ENTRY                   ADDRESS         REF BY
           =====                   =======         ======
           menu_backup             00005590 
               stack 1 = 00000000 ( 00000004 )
    -------------------------------------------------------------------------
CODE
  Segment part 85. NOT NEEDED.
    -------------------------------------------------------------------------
CODE
  Relative segment, address: CODE_AREA 000055B0 - 000055CF (0x20 bytes), align: 2
  Segment part 86.            Intra module refs:   option_menu_HNDLS
                                                   option_menu_HNDLS_1
           ENTRY                   ADDRESS         REF BY
           =====                   =======         ======
           menu_restore            000055B0 
               stack 1 = 00000000 ( 00000004 )
    -------------------------------------------------------------------------
CODE
  Segment part 87. NOT NEEDED.
    -------------------------------------------------------------------------
CODE
  Relative segment, address: CODE_AREA 000055D0 - 000055FB (0x2c bytes), align: 2
  Segment part 88.            Intra module refs:   option_menu_HNDLS
                                                   option_menu_HNDLS_1
           ENTRY                   ADDRESS         REF BY
           =====                   =======         ======
           menu_quit_without_rs    000055D0 
               stack 1 = 00000000 ( 00000004 )
    -------------------------------------------------------------------------
CODE
  Segment part 89. NOT NEEDED.
    -------------------------------------------------------------------------
DATA_C
  Relative segment, address: CODE_AREA 0000959C - 000095C3 (0x28 bytes), align: 2
  Segment part 46.            Intra module refs:   option_menu
           ENTRY                   ADDRESS         REF BY
           =====                   =======         ======
           option_menu_HNDLS       0000959C 
    -------------------------------------------------------------------------
DATA_C
  Relative segment, address: CODE_AREA 000095C4 - 000096DB (0x118 bytes), align: 2
  Segment part 47.            Intra module refs:   option_menu
           ENTRY                   ADDRESS         REF BY
           =====                   =======         ======
           option_menu_ITEMS       000095C4 
    -------------------------------------------------------------------------
DATA_C
  Relative segment, address: CODE_AREA 000096DC - 000096EF (0x14 bytes), align: 2
  Segment part 48.            Intra module refs:   show_option_menu
           ENTRY                   ADDRESS         REF BY
           =====                   =======         ======
           option_menu_header      000096DC 
    -------------------------------------------------------------------------
DATA_C
  Relative segment, address: CODE_AREA 000096F0 - 0000971B (0x2c bytes), align: 2
  Segment part 49.            Intra module refs:   show_option_menu
           ENTRY                   ADDRESS         REF BY
           =====                   =======         ======
           option_menu             000096F0 
    -------------------------------------------------------------------------
DATA_C
  Relative segment, address: CODE_AREA 0000971C - 0000973F (0x24 bytes), align: 2
  Segment part 50.            Intra module refs:   option_menu_1
           ENTRY                   ADDRESS         REF BY
           =====                   =======         ======
           option_menu_HNDLS_1     0000971C 
    -------------------------------------------------------------------------
DATA_C
  Relative segment, address: CODE_AREA 00009740 - 0000983B (0xfc bytes), align: 2
  Segment part 51.            Intra module refs:   option_menu_1
           ENTRY                   ADDRESS         REF BY
           =====                   =======         ======
           option_menu_ITEMS_1     00009740 
    -------------------------------------------------------------------------
DATA_C
  Relative segment, address: CODE_AREA 0000983C - 00009867 (0x2c bytes), align: 2
  Segment part 52.            Intra module refs:   show_option_menu
           ENTRY                   ADDRESS         REF BY
           =====                   =======         ======
           option_menu_1           0000983C 
    -------------------------------------------------------------------------
CODE
  Relative segment, address: CODE_AREA 000055FC - 0000568F (0x94 bytes), align: 2
  Segment part 90.
           ENTRY                   ADDRESS         REF BY
           =====                   =======         ======
           show_option_menu        000055FC        menu_onkey (main)
               stack 1 = 00000000 ( 00000018 )
    -------------------------------------------------------------------------
CODE
  Segment part 91. NOT NEEDED.
    -------------------------------------------------------------------------
CODE
  Relative segment, address: CODE_AREA 00005690 - 0000578B (0xfc bytes), align: 2
  Segment part 92.            Intra module refs:   menu_del_all
           ENTRY                   ADDRESS         REF BY
           =====                   =======         ======
           deleteAllConfig         00005690 
               stack 1 = 00000000 ( 000004CC )
    -------------------------------------------------------------------------
CODE
  Relative segment, address: CODE_AREA 0000578C - 0000578F (0x4 bytes), align: 2
  Segment part 93.            Intra module refs:   deleteAllConfig
                                                   menu_exit
                                                   menu_quit_without_rs
    -------------------------------------------------------------------------
CODE
  Segment part 94. NOT NEEDED.
    -------------------------------------------------------------------------
CODE
  Relative segment, address: CODE_AREA 00005790 - 00005807 (0x78 bytes), align: 2
  Segment part 95.            Intra module refs:   menu_del_this
           ENTRY                   ADDRESS         REF BY
           =====                   =======         ======
           deleteThis              00005790 
               stack 1 = 00000000 ( 000000B8 )
    -------------------------------------------------------------------------
CODE
  Segment part 96. NOT NEEDED.
    -------------------------------------------------------------------------
DATA_C
  Relative segment, address: CODE_AREA 00009868 - 0000987B (0x14 bytes), align: 2
  Segment part 53.            Intra module refs:   createProfileOnoffMenu
           ENTRY                   ADDRESS         REF BY
           =====                   =======         ======
           profile_menu_header     00009868 
    -------------------------------------------------------------------------
CODE
  Relative segment, address: CODE_AREA 00005808 - 000058A7 (0xa0 bytes), align: 2
  Segment part 97.            Intra module refs:   profile_menu
           ENTRY                   ADDRESS         REF BY
           =====                   =======         ======
           profile_menu_onkey      00005808 
               stack 1 = 00000000 ( 00000010 )
    -------------------------------------------------------------------------
CODE
  Segment part 98. NOT NEEDED.
    -------------------------------------------------------------------------
CODE
  Relative segment, address: CODE_AREA 000058A8 - 00005967 (0xc0 bytes), align: 2
  Segment part 99.            Intra module refs:   profile_menu
           ENTRY                   ADDRESS         REF BY
           =====                   =======         ======
           profile_menu_iconhndl   000058A8 
               stack 1 = 00000000 ( 00000018 )
    -------------------------------------------------------------------------
CODE
  Segment part 100. NOT NEEDED.
    -------------------------------------------------------------------------
CODE
  Relative segment, address: CODE_AREA 00005968 - 0000597B (0x14 bytes), align: 2
  Segment part 101.           Intra module refs:   profile_menu
           ENTRY                   ADDRESS         REF BY
           =====                   =======         ======
           profile_menu_ghook      00005968 
               stack 1 = 00000000 ( 00000004 )
    -------------------------------------------------------------------------
CODE
  Segment part 102. NOT NEEDED.
    -------------------------------------------------------------------------
DATA_C
  Relative segment, address: CODE_AREA 0000987C - 00009893 (0x18 bytes), align: 2
  Segment part 54.            Intra module refs:   profile_menu_skt
           ENTRY                   ADDRESS         REF BY
           =====                   =======         ======
           profile_menu_sk         0000987C 
    -------------------------------------------------------------------------
DATA_C
  Relative segment, address: CODE_AREA 00009894 - 0000989B (0x8 bytes), align: 2
  Segment part 55.            Intra module refs:   profile_menu
           ENTRY                   ADDRESS         REF BY
           =====                   =======         ======
           profile_menu_skt        00009894 
    -------------------------------------------------------------------------
DATA_C
  Relative segment, address: CODE_AREA 0000989C - 000098C7 (0x2c bytes), align: 2
  Segment part 56.            Intra module refs:   createProfileOnoffMenu
           ENTRY                   ADDRESS         REF BY
           =====                   =======         ======
           profile_menu            0000989C 
    -------------------------------------------------------------------------
CODE
  Relative segment, address: CODE_AREA 0000597C - 000059DB (0x60 bytes), align: 2
  Segment part 103.           Intra module refs:   menu_profile
           ENTRY                   ADDRESS         REF BY
           =====                   =======         ======
           createProfileOnoffMenu
                                   0000597C        menu_onkey (main)
               stack 1 = 00000000 ( 00000018 )
    -------------------------------------------------------------------------
CODE
  Segment part 104. NOT NEEDED.
    -------------------------------------------------------------------------
CODE
  Relative segment, address: CODE_AREA 000059DC - 00005AC7 (0xec bytes), align: 2
  Segment part 105.           Intra module refs:   menu_del_unused
           ENTRY                   ADDRESS         REF BY
           =====                   =======         ======
           delUnusedConfig         000059DC 
               stack 1 = 00000000 ( 000004DC )
    -------------------------------------------------------------------------
CODE
  Segment part 106. NOT NEEDED.
    -------------------------------------------------------------------------
CODE
  Relative segment, address: CODE_AREA 00005AC8 - 00005AF7 (0x30 bytes), align: 2
  Segment part 107.           Intra module refs:   Segment part 60
           ENTRY                   ADDRESS         REF BY
           =====                   =======         ======
           infoOnKey               00005AC8 
    -------------------------------------------------------------------------
CODE
  Segment part 108. NOT NEEDED.
    -------------------------------------------------------------------------
CODE
  Relative segment, address: CODE_AREA 00005AF8 - 00005B0F (0x18 bytes), align: 2
  Segment part 109.           Intra module refs:   Segment part 60
           ENTRY                   ADDRESS         REF BY
           =====                   =======         ======
           infoGHook               00005AF8 
               stack 1 = 00000000 ( 00000004 )
    -------------------------------------------------------------------------
CODE
  Segment part 110. NOT NEEDED.
    -------------------------------------------------------------------------
CODE
  Relative segment, address: CODE_AREA 00005B10 - 00005B13 (0x4 bytes), align: 2
  Segment part 111.           Intra module refs:   Segment part 60
                                                   Segment part 64
           ENTRY                   ADDRESS         REF BY
           =====                   =======         ======
           info_locret             00005B10 
    -------------------------------------------------------------------------
CODE
  Segment part 112. NOT NEEDED.
    -------------------------------------------------------------------------
DATA_I
  Relative segment, address: DATA_AREA 00000050 - 00000063 (0x14 bytes), align: 2
  Segment part 57.            Intra module refs:   showPatchInfo
           ENTRY                   ADDRESS         REF BY
           =====                   =======         ======
           INFO_HDR                00000050 
    -------------------------------------------------------------------------
DATA_I
  Relative segment, address: DATA_AREA 00000064 - 0000009B (0x38 bytes), align: 2
  Segment part 59.            Intra module refs:   showPatchInfo
           ENTRY                   ADDRESS         REF BY
           =====                   =======         ======
           INFO_DESC               00000064 
    -------------------------------------------------------------------------
CODE
  Relative segment, address: CODE_AREA 00005B14 - 00005E03 (0x2f0 bytes), align: 2
  Segment part 113.           Intra module refs:   menu_info
           ENTRY                   ADDRESS         REF BY
           =====                   =======         ======
           showPatchInfo           00005B14 
               stack 1 = 00000000 ( 0000005C )
    -------------------------------------------------------------------------
CODE
  Relative segment, address: CODE_AREA 00005E04 - 00005E07 (0x4 bytes), align: 2
  Segment part 114.           Intra module refs:   deleteThis
                                                   profile_menu_iconhndl
                                                   profile_menu_onkey
                                                   showPatchInfo
                                                   show_option_menu
    -------------------------------------------------------------------------
CODE
  Segment part 115. NOT NEEDED.
    -------------------------------------------------------------------------
DATA_C
  Relative segment, address: CODE_AREA 000098C8 - 000098CF (0x8 bytes), align: 2
  Segment part 61.            Intra module refs:   pathInputGHook
           ENTRY                   ADDRESS         REF BY
           =====                   =======         ======
           SK_BACKUP               000098C8 
    -------------------------------------------------------------------------
DATA_C
  Relative segment, address: CODE_AREA 000098D0 - 000098D7 (0x8 bytes), align: 2
  Segment part 62.            Intra module refs:   pathInputGHook
           ENTRY                   ADDRESS         REF BY
           =====                   =======         ======
           SK_RESTORE              000098D0 
    -------------------------------------------------------------------------
CODE
  Relative segment, address: CODE_AREA 00005E08 - 00005F6F (0x168 bytes), align: 2
  Segment part 116.           Intra module refs:   configBackUp
                                                   configRestore
           ENTRY                   ADDRESS         REF BY
           =====                   =======         ======
           fcopy                   00005E08 
               stack 1 = 00000000 ( 00000034 )
    -------------------------------------------------------------------------
CODE
  Segment part 117. NOT NEEDED.
    -------------------------------------------------------------------------
CODE
  Relative segment, address: CODE_AREA 00005F70 - 0000601B (0xac bytes), align: 2
  Segment part 118.           Intra module refs:   Segment part 64
           ENTRY                   ADDRESS         REF BY
           =====                   =======         ======
           pathInputOnKey          00005F70 
               stack 1 = 00000000 ( 000000B0 )
    -------------------------------------------------------------------------
CODE
  Segment part 119. NOT NEEDED.
    -------------------------------------------------------------------------
CODE
  Relative segment, address: CODE_AREA 0000601C - 0000605F (0x44 bytes), align: 2
  Segment part 120.           Intra module refs:   Segment part 64
           ENTRY                   ADDRESS         REF BY
           =====                   =======         ======
           pathInputGHook          0000601C 
               stack 1 = 00000000 ( 00000004 )
    -------------------------------------------------------------------------
CODE
  Segment part 121. NOT NEEDED.
    -------------------------------------------------------------------------
DATA_I
  Relative segment, address: DATA_AREA 0000009C - 000000D3 (0x38 bytes), align: 2
  Segment part 63.            Intra module refs:   pathInputDlg
           ENTRY                   ADDRESS         REF BY
           =====                   =======         ======
           PATH_INPUT_DESC         0000009C 
    -------------------------------------------------------------------------
DATA_I
  Relative segment, address: DATA_AREA 000000D4 - 000000E7 (0x14 bytes), align: 2
  Segment part 65.            Intra module refs:   pathInputDlg
           ENTRY                   ADDRESS         REF BY
           =====                   =======         ======
           PATH_INPUT_HDR          000000D4 
    -------------------------------------------------------------------------
CODE
  Relative segment, address: CODE_AREA 00006060 - 000061FF (0x1a0 bytes), align: 2
  Segment part 122.           Intra module refs:   menu_backup
                                                   menu_restore
           ENTRY                   ADDRESS         REF BY
           =====                   =======         ======
           pathInputDlg            00006060 
               stack 1 = 00000000 ( 0000005C )
    -------------------------------------------------------------------------
CODE
  Relative segment, address: CODE_AREA 00006200 - 00006203 (0x4 bytes), align: 2
  Segment part 123.           Intra module refs:   menu_backup
                                                   menu_restore
                                                   pathInputDlg
                                                   pathInputGHook
                                                   pathInputOnKey
    -------------------------------------------------------------------------
CODE
  Relative segment, address: CODE_AREA 00006204 - 00006207 (0x4 bytes), align: 2
  Segment part 124.           Intra module refs:   pathInputDlg
                                                   profile_menu_iconhndl
                                                   showPatchInfo
    -------------------------------------------------------------------------
CODE
  Relative segment, address: CODE_AREA 00006208 - 0000620B (0x4 bytes), align: 2
  Segment part 125.           Intra module refs:   deleteThis
                                                   pathInputDlg
    -------------------------------------------------------------------------
CODE
  Segment part 126. NOT NEEDED.
    -------------------------------------------------------------------------
CODE
  Relative segment, address: CODE_AREA 0000620C - 0000629F (0x94 bytes), align: 2
  Segment part 127.           Intra module refs:   configBackUp
           ENTRY                   ADDRESS         REF BY
           =====                   =======         ======
           mkpath                  0000620C 
               stack 1 = 00000000 ( 00000098 )
    -------------------------------------------------------------------------
CODE
  Segment part 128. NOT NEEDED.
    -------------------------------------------------------------------------
CODE
  Relative segment, address: CODE_AREA 000062A0 - 000063A3 (0x104 bytes), align: 2
  Segment part 129.           Intra module refs:   pathInputOnKey
           ENTRY                   ADDRESS         REF BY
           =====                   =======         ======
           configBackUp            000062A0 
               stack 1 = 00000000 ( 00000558 )
    -------------------------------------------------------------------------
CODE
  Relative segment, address: CODE_AREA 000063A4 - 000063A7 (0x4 bytes), align: 2
  Segment part 130.           Intra module refs:   configBackUp
                                                   delUnusedConfig
                                                   deleteAllConfig
    -------------------------------------------------------------------------
CODE
  Segment part 131. NOT NEEDED.
    -------------------------------------------------------------------------
CODE
  Relative segment, address: CODE_AREA 000063A8 - 000064F7 (0x150 bytes), align: 2
  Segment part 132.           Intra module refs:   pathInputOnKey
           ENTRY                   ADDRESS         REF BY
           =====                   =======         ======
           configRestore           000063A8 
               stack 1 = 00000000 ( 00000558 )
    -------------------------------------------------------------------------
CODE
  Relative segment, address: CODE_AREA 000064F8 - 000064FB (0x4 bytes), align: 2
  Segment part 133.           Intra module refs:   configBackUp
                                                   configRestore
                                                   delUnusedConfig
                                                   deleteAllConfig
    -------------------------------------------------------------------------
CODE
  Relative segment, address: CODE_AREA 000064FC - 000064FF (0x4 bytes), align: 2
  Segment part 134.           Intra module refs:   configBackUp
                                                   configRestore
                                                   delUnusedConfig
                                                   deleteAllConfig
                                                   deleteThis
    -------------------------------------------------------------------------
CODE
  Relative segment, address: CODE_AREA 00006500 - 00006503 (0x4 bytes), align: 2
  Segment part 135.           Intra module refs:   configBackUp
                                                   configRestore
    -------------------------------------------------------------------------
CODE
  Relative segment, address: CODE_AREA 00006504 - 00006507 (0x4 bytes), align: 2
  Segment part 136.           Intra module refs:   configRestore
                                                   deleteAllConfig
    -------------------------------------------------------------------------
CODE
  Relative segment, address: CODE_AREA 00006508 - 0000650B (0x4 bytes), align: 2
  Segment part 137.           Intra module refs:   configRestore
                                                   deleteAllConfig
    -------------------------------------------------------------------------
CODE
  Relative segment, address: CODE_AREA 0000650C - 0000650F (0x4 bytes), align: 2
  Segment part 138.           Intra module refs:   configRestore
    -------------------------------------------------------------------------
CODE
  Segment part 139. NOT NEEDED.Intra module refs   deleteThis
                                                   profile_menu_iconhndl
                                                   profile_menu_onkey
                                                   showPatchInfo
                                                   show_option_menu
    -------------------------------------------------------------------------
CODE
  Segment part 140. NOT NEEDED.Intra module refs   configRestore
                                                   deleteAllConfig
    -------------------------------------------------------------------------
CODE
  Segment part 141. NOT NEEDED.Intra module refs   deleteAllConfig
    -------------------------------------------------------------------------
CODE
  Segment part 142. NOT NEEDED.Intra module refs   deleteThis
    -------------------------------------------------------------------------
CODE
  Segment part 143. NOT NEEDED.Intra module refs   profile_menu_onkey
    -------------------------------------------------------------------------
CODE
  Segment part 144. NOT NEEDED.Intra module refs   profile_menu_iconhndl
                                                   profile_menu_onkey
    -------------------------------------------------------------------------
CODE
  Segment part 145. NOT NEEDED.Intra module refs   delUnusedConfig
    -------------------------------------------------------------------------
CODE
  Segment part 146. NOT NEEDED.Intra module refs   showPatchInfo
    -------------------------------------------------------------------------
CODE
  Segment part 147. NOT NEEDED.Intra module refs   showPatchInfo
    -------------------------------------------------------------------------
CODE
  Segment part 148. NOT NEEDED.Intra module refs   configRestore
    -------------------------------------------------------------------------
CSTACK
  Segment part 1. NOT NEEDED.
    -------------------------------------------------------------------------
DATA_ID
  Relative segment, address: CODE_AREA 00000050 - 00000063 (0x14 bytes), align: 2
  Segment part 58.            Intra module refs:   INFO_HDR
    -------------------------------------------------------------------------
DATA_ID
  Relative segment, address: CODE_AREA 00000064 - 0000009B (0x38 bytes), align: 2
  Segment part 60.            Intra module refs:   INFO_DESC
    -------------------------------------------------------------------------
DATA_ID
  Relative segment, address: CODE_AREA 0000009C - 000000D3 (0x38 bytes), align: 2
  Segment part 64.            Intra module refs:   PATH_INPUT_DESC
    -------------------------------------------------------------------------
DATA_ID
  Relative segment, address: CODE_AREA 000000D4 - 000000E7 (0x14 bytes), align: 2
  Segment part 66.            Intra module refs:   PATH_INPUT_HDR
    -------------------------------------------------------------------------
DATA_ID
  Segment part 149. TENTATIVE. Used definition from main
           ENTRY                   ADDRESS         REF BY
           =====                   =======         ======
           ?*?DATA_ID              
    -------------------------------------------------------------------------
INITTAB
  Segment part 150. TENTATIVE. Used definition from main
           ENTRY                   ADDRESS         REF BY
           =====                   =======         ======
           ?init?tab?DATA_I        
    -------------------------------------------------------------------------
INITTAB
  Segment part 151. TENTATIVE. Used definition from getConfig
           ENTRY                   ADDRESS         REF BY
           =====                   =======         ======
           ?init?tab?DATA_Z        

    *************************************************************************

  FILE NAME : F:\SVN\cn\Master\Release_NEWSGOLD\Obj\ptcFileWork.r79
  PROGRAM MODULE, NAME : ptcFileWork

  SEGMENTS IN THE MODULE
  ======================
DATA_Z
  Relative segment, address: CODE_AREA 00015BC8 - 00015BCB (0x4 bytes), align: 2
  Segment part 6.             Intra module refs:   initPatchConfig
           ENTRY                   ADDRESS         REF BY
           =====                   =======         ======
           ptcfilesize             00015BC8 
    -------------------------------------------------------------------------
CODE
  Segment part 7. NOT NEEDED.
    -------------------------------------------------------------------------
CODE
  Relative segment, address: CODE_AREA 00006510 - 0000676B (0x25c bytes), align: 2
  Segment part 8.             Intra module refs:   initPatchConfig
           ENTRY                   ADDRESS         REF BY
           =====                   =======         ======
           initPatchItem           00006510 
               stack 1 = 00000000 ( 0000000C )
    -------------------------------------------------------------------------
CODE
  Segment part 9. NOT NEEDED.
    -------------------------------------------------------------------------
CODE
  Relative segment, address: CODE_AREA 0000676C - 0000682F (0xc4 bytes), align: 2
  Segment part 10.
           ENTRY                   ADDRESS         REF BY
           =====                   =======         ======
           initPatchConfig         0000676C        getAllPatchData (getConfig)
               stack 1 = 00000000 ( 000000A8 )
    -------------------------------------------------------------------------
CODE
  Segment part 11. NOT NEEDED.
    -------------------------------------------------------------------------
CODE
  Relative segment, address: CODE_AREA 00006830 - 000068E3 (0xb4 bytes), align: 2
  Segment part 12.            Intra module refs:   fillItemDataToBuf
                                                   getPtcSize
           ENTRY                   ADDRESS         REF BY
           =====                   =======         ======
           findNextBposItem        00006830 
               stack 1 = 00000000 ( 00000014 )
    -------------------------------------------------------------------------
CODE
  Segment part 13. NOT NEEDED.
    -------------------------------------------------------------------------
CODE
  Relative segment, address: CODE_AREA 000068E4 - 0000699B (0xb8 bytes), align: 2
  Segment part 14.            Intra module refs:   fillItemDataToBuf
           ENTRY                   ADDRESS         REF BY
           =====                   =======         ======
           getTheSameBPosCheckBox
                                   000068E4 
               stack 1 = 00000000 ( 00000014 )
    -------------------------------------------------------------------------
CODE
  Segment part 15. NOT NEEDED.
    -------------------------------------------------------------------------
CODE
  Relative segment, address: CODE_AREA 0000699C - 00006C57 (0x2bc bytes), align: 2
  Segment part 16.            Intra module refs:   savePatchConfig
           ENTRY                   ADDRESS         REF BY
           =====                   =======         ======
           fillItemDataToBuf       0000699C 
               stack 1 = 00000000 ( 00000010 )
    -------------------------------------------------------------------------
CODE
  Segment part 17. NOT NEEDED.
    -------------------------------------------------------------------------
CODE
  Relative segment, address: CODE_AREA 00006C58 - 00006D6B (0x114 bytes), align: 2
  Segment part 18.            Intra module refs:   savePatchConfig
           ENTRY                   ADDRESS         REF BY
           =====                   =======         ======
           getPtcSize              00006C58 
               stack 1 = 00000000 ( 0000000C )
    -------------------------------------------------------------------------
CODE
  Segment part 19. NOT NEEDED.
    -------------------------------------------------------------------------
CODE
  Relative segment, address: CODE_AREA 00006D6C - 00006EF7 (0x18c bytes), align: 2
  Segment part 20.            Intra module refs:   saveAllConfig
           ENTRY                   ADDRESS         REF BY
           =====                   =======         ======
           savePatchConfig         00006D6C 
               stack 1 = 00000000 ( 000000AC )
    -------------------------------------------------------------------------
CODE
  Relative segment, address: CODE_AREA 00006EF8 - 00006EFB (0x4 bytes), align: 2
  Segment part 21.            Intra module refs:   initPatchConfig
                                                   savePatchConfig
    -------------------------------------------------------------------------
CODE
  Relative segment, address: CODE_AREA 00006EFC - 00006EFF (0x4 bytes), align: 2
  Segment part 22.            Intra module refs:   initPatchConfig
                                                   savePatchConfig
    -------------------------------------------------------------------------
CODE
  Relative segment, address: CODE_AREA 00006F00 - 00006F03 (0x4 bytes), align: 2
  Segment part 23.            Intra module refs:   initPatchConfig
                                                   savePatchConfig
    -------------------------------------------------------------------------
CODE
  Relative segment, address: CODE_AREA 00006F04 - 00006F07 (0x4 bytes), align: 2
  Segment part 24.            Intra module refs:   initPatchConfig
                                                   savePatchConfig
    -------------------------------------------------------------------------
CODE
  Relative segment, address: CODE_AREA 00006F08 - 00006F0B (0x4 bytes), align: 2
  Segment part 25.            Intra module refs:   fillItemDataToBuf
                                                   initPatchConfig
                                                   initPatchItem
                                                   savePatchConfig
    -------------------------------------------------------------------------
CODE
  Segment part 26. NOT NEEDED.
    -------------------------------------------------------------------------
CODE
  Relative segment, address: CODE_AREA 00006F0C - 00006F3B (0x30 bytes), align: 2
  Segment part 27.
           ENTRY                   ADDRESS         REF BY
           =====                   =======         ======
           saveAllConfig           00006F0C        Killer (main)
               stack 1 = 00000000 ( 00000008 )
    -------------------------------------------------------------------------
CODE
  Segment part 28. NOT NEEDED.Intra module refs:   savePatchConfig
    -------------------------------------------------------------------------
CSTACK
  Segment part 1. NOT NEEDED.
    -------------------------------------------------------------------------
INITTAB
  Segment part 29. TENTATIVE. Used definition from getConfig
           ENTRY                   ADDRESS         REF BY
           =====                   =======         ======
           ?init?tab?DATA_Z        
    -------------------------------------------------------------------------
DATA_C
  Relative segment, address: CODE_AREA 000098D8 - 000098EB (0x14 bytes), align: 2
  Segment part 2.             Intra module refs:   Segment part 21
    -------------------------------------------------------------------------
DATA_C
  Relative segment, address: CODE_AREA 000098EC - 000098F3 (0x8 bytes), align: 2
  Segment part 3.             Intra module refs:   Segment part 22
    -------------------------------------------------------------------------
DATA_C
  Relative segment, address: CODE_AREA 000098F4 - 000098FB (0x8 bytes), align: 2
  Segment part 4.             Intra module refs:   Segment part 23
    -------------------------------------------------------------------------
DATA_C
  Relative segment, address: CODE_AREA 000098FC - 00009903 (0x8 bytes), align: 2
  Segment part 5.             Intra module refs:   Segment part 24

    *************************************************************************

  FILE NAME : F:\SVN\cn\Master\Release_NEWSGOLD\Obj\string.r79
  PROGRAM MODULE, NAME : string

  SEGMENTS IN THE MODULE
  ======================
CODE
  Segment part 2. NOT NEEDED.
    -------------------------------------------------------------------------
CODE
  Relative segment, address: CODE_AREA 00006F3C - 00006F6F (0x34 bytes), align: 2
  Segment part 3.
           ENTRY                   ADDRESS         REF BY
           =====                   =======         ======
           getnumwidth             00006F3C        createEditGui (main)
    -------------------------------------------------------------------------
CODE
  Segment part 4. NOT NEEDED.
    -------------------------------------------------------------------------
CODE
  Relative segment, address: CODE_AREA 00006F70 - 00006FD7 (0x68 bytes), align: 2
  Segment part 5.
           ENTRY                   ADDRESS         REF BY
           =====                   =======         ======
           uni2ws                  00006F70        createEditGui (main)
               stack 1 = 00000000 ( 00000008 )
    -------------------------------------------------------------------------
CODE
  Segment part 6. NOT NEEDED.
    -------------------------------------------------------------------------
CODE
  Relative segment, address: CODE_AREA 00006FD8 - 0000703F (0x68 bytes), align: 2
  Segment part 7.
           ENTRY                   ADDRESS         REF BY
           =====                   =======         ======
           ws2uni                  00006FD8        edGHook (main)
               stack 1 = 00000000 ( 00000008 )
    -------------------------------------------------------------------------
CODE
  Segment part 8. NOT NEEDED.
    -------------------------------------------------------------------------
CODE
  Relative segment, address: CODE_AREA 00007040 - 000070AF (0x70 bytes), align: 2
  Segment part 9.
           ENTRY                   ADDRESS         REF BY
           =====                   =======         ======
           hex2ws                  00007040        createEditGui (main)
               stack 1 = 00000000 ( 00000018 )
    -------------------------------------------------------------------------
CODE
  Segment part 10. NOT NEEDED.
    -------------------------------------------------------------------------
CODE
  Relative segment, address: CODE_AREA 000070B0 - 00007157 (0xa8 bytes), align: 2
  Segment part 11.
           ENTRY                   ADDRESS         REF BY
           =====                   =======         ======
           uniFormatString2ws      000070B0        createEditGui (main)
                                                   edGHook (main)
                                                   menu_iconhndl (main)
                                                   showPatchInfo (optionMenu)
                                                   updateEdHdr (main)
               stack 1 = 00000000 ( 00000020 )
    -------------------------------------------------------------------------
CODE
  Segment part 12. NOT NEEDED.
    -------------------------------------------------------------------------
CODE
  Relative segment, address: CODE_AREA 00007158 - 000071B7 (0x60 bytes), align: 2
  Segment part 13.            Intra module refs:   uniFormatString2ws
           ENTRY                   ADDRESS         REF BY
           =====                   =======         ======
           isUniFormat             00007158        createEditGui (main)
                                                   edGHook (main)
                                                   menu_iconhndl (main)
                                                   showPatchInfo (optionMenu)
                                                   updateEdHdr (main)
    -------------------------------------------------------------------------
CODE
  Segment part 14. NOT NEEDED.
    -------------------------------------------------------------------------
CODE
  Relative segment, address: CODE_AREA 000071B8 - 00007297 (0xe0 bytes), align: 2
  Segment part 15.
           ENTRY                   ADDRESS         REF BY
           =====                   =======         ======
           ws2hex                  000071B8        edGHook (main)
               stack 1 = 00000000 ( 00000220 )
    -------------------------------------------------------------------------
CODE
  Segment part 16. NOT NEEDED.
    -------------------------------------------------------------------------
CODE
  Relative segment, address: CODE_AREA 00007298 - 00007323 (0x8c bytes), align: 2
  Segment part 17.
           ENTRY                   ADDRESS         REF BY
           =====                   =======         ======
           bytes_2ws               00007298        createEditGui (main)
               stack 1 = 00000000 ( 00000018 )
    -------------------------------------------------------------------------
CODE
  Segment part 18. NOT NEEDED.
    -------------------------------------------------------------------------
CODE
  Relative segment, address: CODE_AREA 00007324 - 000073AF (0x8c bytes), align: 2
  Segment part 19.
           ENTRY                   ADDRESS         REF BY
           =====                   =======         ======
           ints_2ws                00007324        createEditGui (main)
               stack 1 = 00000000 ( 00000018 )
    -------------------------------------------------------------------------
CODE
  Relative segment, address: CODE_AREA 000073B0 - 000073B3 (0x4 bytes), align: 2
  Segment part 20.            Intra module refs:   bytes_2ws
                                                   ints_2ws
    -------------------------------------------------------------------------
CODE
  Relative segment, address: CODE_AREA 000073B4 - 000073B7 (0x4 bytes), align: 2
  Segment part 21.            Intra module refs:   bytes_2ws
                                                   ints_2ws
    -------------------------------------------------------------------------
CODE
  Segment part 22. NOT NEEDED.
    -------------------------------------------------------------------------
CODE
  Relative segment, address: CODE_AREA 000073B8 - 0000740F (0x58 bytes), align: 2
  Segment part 23.            Intra module refs:   strstrInQuote
           ENTRY                   ADDRESS         REF BY
           =====                   =======         ======
           strncmpNoCase           000073B8        addPreDataToCBoxItem (getConfig)
                                                   findTemplate (getConfig)
                                                   isPatchExistedByID (getConfig)
                                                   sortPatchConfigList (getConfig)
               stack 1 = 00000000 ( 00000004 )
    -------------------------------------------------------------------------
CODE
  Segment part 24. NOT NEEDED.
    -------------------------------------------------------------------------
CODE
  Relative segment, address: CODE_AREA 00007410 - 00007453 (0x44 bytes), align: 2
  Segment part 25.            Intra module refs:   str2num
                                                   str2num_char
                                                   str2num_short
                                                   uniFormatString2ws
                                                   ws2hex
           ENTRY                   ADDRESS         REF BY
           =====                   =======         ======
           chr2num                 00007410        doItemJob (getConfig)
    -------------------------------------------------------------------------
CODE
  Segment part 26. NOT NEEDED.
    -------------------------------------------------------------------------
CODE
  Relative segment, address: CODE_AREA 00007454 - 00007473 (0x20 bytes), align: 2
  Segment part 27.            Intra module refs:   gotoMyStrEnd
                                                   gotoMyStrStart
                                                   str2bytes
                                                   str2ints
           ENTRY                   ADDRESS         REF BY
           =====                   =======         ======
           gotoRealPos             00007454        addInfoToPatchInfo (getConfig)
                                                   addPreDataToCBoxItem (getConfig)
                                                   addPrepareData (getConfig)
                                                   addToPatchInfo (getConfig)
                                                   cboxItemColon (getConfig)
                                                   doItemJob (getConfig)
                                                   doSubMenuJob (getConfig)
                                                   doTemplateWork (getConfig)
                                                   isCurrectItem (getConfig)
                                                   readConfig (getConfig)
    -------------------------------------------------------------------------
CODE
  Segment part 28. NOT NEEDED.
    -------------------------------------------------------------------------
CODE
  Relative segment, address: CODE_AREA 00007474 - 000074CF (0x5c bytes), align: 2
  Segment part 29.
           ENTRY                   ADDRESS         REF BY
           =====                   =======         ======
           strstrInQuote           00007474        addToPatchInfo (getConfig)
                                                   doItemJob (getConfig)
                                                   doSubMenuJob (getConfig)
                                                   doTemplateWork (getConfig)
                                                   readConfig (getConfig)
               stack 1 = 00000000 ( 00000010 )
    -------------------------------------------------------------------------
CODE
  Segment part 30. NOT NEEDED.
    -------------------------------------------------------------------------
CODE
  Relative segment, address: CODE_AREA 000074D0 - 000074FB (0x2c bytes), align: 2
  Segment part 31.            Intra module refs:   str2bytes
                                                   str2ints
           ENTRY                   ADDRESS         REF BY
           =====                   =======         ======
           strchrInQuote           000074D0        isCurrectItem (getConfig)
    -------------------------------------------------------------------------
CODE
  Segment part 32. NOT NEEDED.
    -------------------------------------------------------------------------
CODE
  Relative segment, address: CODE_AREA 000074FC - 00007523 (0x28 bytes), align: 2
  Segment part 33.
           ENTRY                   ADDRESS         REF BY
           =====                   =======         ======
           gotoQuoteStart          000074FC        doSubMenuJob (getConfig)
                                                   doTemplateWork (getConfig)
                                                   readConfig (getConfig)
    -------------------------------------------------------------------------
CODE
  Segment part 34. NOT NEEDED.
    -------------------------------------------------------------------------
CODE
  Relative segment, address: CODE_AREA 00007524 - 0000754B (0x28 bytes), align: 2
  Segment part 35.
           ENTRY                   ADDRESS         REF BY
           =====                   =======         ======
           gotoQuoteEnd            00007524        addPrepareData (getConfig)
                                                   cboxItemColon (getConfig)
                                                   doSubMenuJob (getConfig)
                                                   doTemplateWork (getConfig)
                                                   readConfig (getConfig)
    -------------------------------------------------------------------------
CODE
  Segment part 36. NOT NEEDED.
    -------------------------------------------------------------------------
CODE
  Relative segment, address: CODE_AREA 0000754C - 00007577 (0x2c bytes), align: 2
  Segment part 37.            Intra module refs:   gotoMyStrEnd
           ENTRY                   ADDRESS         REF BY
           =====                   =======         ======
           gotoNextNameQuote       0000754C 
    -------------------------------------------------------------------------
CODE
  Segment part 38. NOT NEEDED.
    -------------------------------------------------------------------------
CODE
  Relative segment, address: CODE_AREA 00007578 - 000075AF (0x38 bytes), align: 2
  Segment part 39.            Intra module refs:   gotoMyStrEnd
           ENTRY                   ADDRESS         REF BY
           =====                   =======         ======
           gotoStringEndByChr      00007578        addPrepareData (getConfig)
                                                   cboxItemColon (getConfig)
    -------------------------------------------------------------------------
CODE
  Segment part 40. NOT NEEDED.
    -------------------------------------------------------------------------
CODE
  Relative segment, address: CODE_AREA 000075B0 - 000075D7 (0x28 bytes), align: 2
  Segment part 41.
           ENTRY                   ADDRESS         REF BY
           =====                   =======         ======
           gotoMyStrStart          000075B0        addInfoToPatchInfo (getConfig)
                                                   addPreDataToCBoxItem (getConfig)
                                                   addPrepareData (getConfig)
                                                   addToPatchInfo (getConfig)
                                                   cboxItemColon (getConfig)
                                                   doItemJob (getConfig)
                                                   doSubMenuJob (getConfig)
                                                   doTemplateWork (getConfig)
               stack 1 = 00000000 ( 00000004 )
    -------------------------------------------------------------------------
CODE
  Segment part 42. NOT NEEDED.
    -------------------------------------------------------------------------
CODE
  Relative segment, address: CODE_AREA 000075D8 - 00007603 (0x2c bytes), align: 2
  Segment part 43.
           ENTRY                   ADDRESS         REF BY
           =====                   =======         ======
           gotoMyStrEnd            000075D8        addInfoToPatchInfo (getConfig)
                                                   addPreDataToCBoxItem (getConfig)
                                                   addPrepareData (getConfig)
                                                   addToPatchInfo (getConfig)
                                                   cboxItemColon (getConfig)
                                                   doItemJob (getConfig)
                                                   doSubMenuJob (getConfig)
                                                   doTemplateWork (getConfig)
               stack 1 = 00000000 ( 00000004 )
    -------------------------------------------------------------------------
CODE
  Segment part 44. NOT NEEDED.
    -------------------------------------------------------------------------
CODE
  Relative segment, address: CODE_AREA 00007604 - 0000761F (0x1c bytes), align: 2
  Segment part 45.
           ENTRY                   ADDRESS         REF BY
           =====                   =======         ======
           strnCopyWithEnd         00007604        addInfoToPatchInfo (getConfig)
                                                   addPrepareData (getConfig)
                                                   addToPatchInfo (getConfig)
                                                   cboxItemColon (getConfig)
                                                   doItemJob (getConfig)
                                                   doSubMenuJob (getConfig)
                                                   doTemplateWork (getConfig)
                                                   readConfig (getConfig)
               stack 1 = 00000000 ( 0000000C )
    -------------------------------------------------------------------------
CODE
  Segment part 46. NOT NEEDED.
    -------------------------------------------------------------------------
CODE
  Relative segment, address: CODE_AREA 00007620 - 00007787 (0x168 bytes), align: 2
  Segment part 47.            Intra module refs:   str2ints
           ENTRY                   ADDRESS         REF BY
           =====                   =======         ======
           str2num                 00007620        addToPatchInfo (getConfig)
                                                   doItemJob (getConfig)
                                                   edGHook (main)
                                                   readConfig (getConfig)
               stack 1 = 00000000 ( 00000020 )
    -------------------------------------------------------------------------
CODE
  Segment part 48. NOT NEEDED.
    -------------------------------------------------------------------------
CODE
  Relative segment, address: CODE_AREA 00007788 - 0000789F (0x118 bytes), align: 2
  Segment part 49.
           ENTRY                   ADDRESS         REF BY
           =====                   =======         ======
           str2num_short           00007788        doItemJob (getConfig)
               stack 1 = 00000000 ( 00000020 )
    -------------------------------------------------------------------------
CODE
  Segment part 50. NOT NEEDED.
    -------------------------------------------------------------------------
CODE
  Relative segment, address: CODE_AREA 000078A0 - 00007A13 (0x174 bytes), align: 2
  Segment part 51.            Intra module refs:   str2bytes
           ENTRY                   ADDRESS         REF BY
           =====                   =======         ======
           str2num_char            000078A0        addPrepareData (getConfig)
                                                   cboxItemColon (getConfig)
                                                   doItemJob (getConfig)
                                                   edGHook (main)
               stack 1 = 00000000 ( 00000024 )
    -------------------------------------------------------------------------
CODE
  Segment part 52. NOT NEEDED.
    -------------------------------------------------------------------------
CODE
  Relative segment, address: CODE_AREA 00007A14 - 00007A5F (0x4c bytes), align: 2
  Segment part 53.
           ENTRY                   ADDRESS         REF BY
           =====                   =======         ======
           cleanStrByChr           00007A14        addItemToConfig (getConfig)
                                                   addPrepareData (getConfig)
    -------------------------------------------------------------------------
CODE
  Segment part 54. NOT NEEDED.
    -------------------------------------------------------------------------
CODE
  Relative segment, address: CODE_AREA 00007A60 - 00007ACB (0x6c bytes), align: 2
  Segment part 55.
           ENTRY                   ADDRESS         REF BY
           =====                   =======         ======
           str2bytes               00007A60        doItemJob (getConfig)
                                                   edGHook (main)
               stack 1 = 00000000 ( 00000018 )
    -------------------------------------------------------------------------
CODE
  Segment part 56. NOT NEEDED.
    -------------------------------------------------------------------------
CODE
  Relative segment, address: CODE_AREA 00007ACC - 00007B37 (0x6c bytes), align: 2
  Segment part 57.
           ENTRY                   ADDRESS         REF BY
           =====                   =======         ======
           str2ints                00007ACC        doItemJob (getConfig)
                                                   edGHook (main)
               stack 1 = 00000000 ( 00000018 )
    -------------------------------------------------------------------------
CSTACK
  Segment part 1. NOT NEEDED.

    *************************************************************************

  FILE NAME : F:\SVN\cn\Master\Release_NEWSGOLD\Obj\usedstr.r79
  PROGRAM MODULE, NAME : usedstr

  SEGMENTS IN THE MODULE
  ======================
DATA_C
  Relative segment, address: CODE_AREA 00009AE0 - 00009AE2 (0x3 bytes), align: 0
  Segment part 2.
           ENTRY                   ADDRESS         REF BY
           =====                   =======         ======
           PERCENT_T               00009AE0        Segment part 100 (main)
                                                   Segment part 110 (main)
                                                   Segment part 124 (optionMenu)
                                                   uniFormatString2ws (string)
    -------------------------------------------------------------------------
DATA_C
  Relative segment, address: CODE_AREA 00009AE3 - 00009AE5 (0x3 bytes), align: 0
  Segment part 3.
           ENTRY                   ADDRESS         REF BY
           =====                   =======         ======
           PERCENT_D               00009AE3        Segment part 111 (main)
                                                   Segment part 20 (string)
    -------------------------------------------------------------------------
DATA_C
  Relative segment, address: CODE_AREA 00009904 - 0000990B (0x8 bytes), align: 2
  Segment part 4.
           ENTRY                   ADDRESS         REF BY
           =====                   =======         ======
           PERCENT_D_D             00009904        Segment part 104 (main)
                                                   Segment part 114 (main)
    -------------------------------------------------------------------------
DATA_C
  Relative segment, address: CODE_AREA 0000990C - 00009913 (0x8 bytes), align: 2
  Segment part 5.
           ENTRY                   ADDRESS         REF BY
           =====                   =======         ======
           PERCENT_08X             0000990C        createEditGui (main)
    -------------------------------------------------------------------------
DATA_C
  Relative segment, address: CODE_AREA 00009914 - 0000991B (0x8 bytes), align: 2
  Segment part 6.
           ENTRY                   ADDRESS         REF BY
           =====                   =======         ======
           PERCENT_02X             00009914        hex2ws (string)
    -------------------------------------------------------------------------
DATA_C
  Relative segment, address: CODE_AREA 0000991C - 0000992F (0x14 bytes), align: 2
  Segment part 7.
           ENTRY                   ADDRESS         REF BY
           =====                   =======         ======
           PERCENT_02X_02X_        0000991C        Segment part 112 (main)
                                                   method0_2 (visual)
    -------------------------------------------------------------------------
DATA_C
  Relative segment, address: CODE_AREA 00009930 - 00009933 (0x4 bytes), align: 2
  Segment part 8.
           ENTRY                   ADDRESS         REF BY
           =====                   =======         ======
           D_PERCENT_D             00009930        Segment part 21 (string)
    -------------------------------------------------------------------------
DATA_C
  Relative segment, address: CODE_AREA 00009934 - 0000993B (0x8 bytes), align: 2
  Segment part 9.
           ENTRY                   ADDRESS         REF BY
           =====                   =======         ======
           STR_CHKBOX1             00009934        doItemJob (getConfig)
    -------------------------------------------------------------------------
DATA_C
  Relative segment, address: CODE_AREA 0000993C - 00009947 (0xc bytes), align: 2
  Segment part 10.
           ENTRY                   ADDRESS         REF BY
           =====                   =======         ======
           STR_CHKBOX2             0000993C        doItemJob (getConfig)
    -------------------------------------------------------------------------
DATA_C
  Relative segment, address: CODE_AREA 00009948 - 0000994B (0x4 bytes), align: 2
  Segment part 11.
           ENTRY                   ADDRESS         REF BY
           =====                   =======         ======
           STR_VL                  00009948        doItemJob (getConfig)
    -------------------------------------------------------------------------
DATA_C
  Relative segment, address: CODE_AREA 0000994C - 00009953 (0x8 bytes), align: 2
  Segment part 12.
           ENTRY                   ADDRESS         REF BY
           =====                   =======         ======
           STR_VL1                 0000994C        doItemJob (getConfig)
    -------------------------------------------------------------------------
DATA_C
  Relative segment, address: CODE_AREA 00009954 - 0000995B (0x8 bytes), align: 2
  Segment part 13.
           ENTRY                   ADDRESS         REF BY
           =====                   =======         ======
           STR_XY1                 00009954        doItemJob (getConfig)
    -------------------------------------------------------------------------
DATA_C
  Relative segment, address: CODE_AREA 0000995C - 00009963 (0x8 bytes), align: 2
  Segment part 14.
           ENTRY                   ADDRESS         REF BY
           =====                   =======         ======
           STR_XY2                 0000995C        doItemJob (getConfig)
    -------------------------------------------------------------------------
DATA_C
  Relative segment, address: CODE_AREA 00009964 - 00009967 (0x4 bytes), align: 2
  Segment part 15.
           ENTRY                   ADDRESS         REF BY
           =====                   =======         ======
           STR_X                   00009964        doItemJob (getConfig)
    -------------------------------------------------------------------------
DATA_C
  Relative segment, address: CODE_AREA 00009968 - 0000996B (0x4 bytes), align: 2
  Segment part 16.
           ENTRY                   ADDRESS         REF BY
           =====                   =======         ======
           STR_Y                   00009968        doItemJob (getConfig)
    -------------------------------------------------------------------------
DATA_C
  Relative segment, address: CODE_AREA 0000996C - 0000996F (0x4 bytes), align: 2
  Segment part 17.
           ENTRY                   ADDRESS         REF BY
           =====                   =======         ======
           STR_WIDTH               0000996C        doItemJob (getConfig)
    -------------------------------------------------------------------------
DATA_C
  Relative segment, address: CODE_AREA 00009970 - 00009973 (0x4 bytes), align: 2
  Segment part 18.
           ENTRY                   ADDRESS         REF BY
           =====                   =======         ======
           STR_HIGHT               00009970        doItemJob (getConfig)
    -------------------------------------------------------------------------
DATA_C
  Relative segment, address: CODE_AREA 00009AE6 - 00009AE8 (0x3 bytes), align: 0
  Segment part 19.
           ENTRY                   ADDRESS         REF BY
           =====                   =======         ======
           STR_CHOICE              00009AE6        Segment part 86 (getConfig)
                                                   doItemJob (getConfig)
    -------------------------------------------------------------------------
DATA_C
  Relative segment, address: CODE_AREA 00009AE9 - 00009AEB (0x3 bytes), align: 0
  Segment part 20.
           ENTRY                   ADDRESS         REF BY
           =====                   =======         ======
           STR_CHOICE1             00009AE9        readConfig (getConfig)
    -------------------------------------------------------------------------
DATA_C
  Relative segment, address: CODE_AREA 00009974 - 0000997B (0x8 bytes), align: 2
  Segment part 21.
           ENTRY                   ADDRESS         REF BY
           =====                   =======         ======
           STR_CHOICE2             00009974        readConfig (getConfig)
    -------------------------------------------------------------------------
DATA_C
  Relative segment, address: CODE_AREA 0000997C - 00009987 (0xc bytes), align: 2
  Segment part 22.
           ENTRY                   ADDRESS         REF BY
           =====                   =======         ======
           STR_SLIDER1             0000997C        doItemJob (getConfig)
    -------------------------------------------------------------------------
DATA_C
  Relative segment, address: CODE_AREA 00009988 - 0000998F (0x8 bytes), align: 2
  Segment part 23.
           ENTRY                   ADDRESS         REF BY
           =====                   =======         ======
           STR_SLIDER2             00009988        doItemJob (getConfig)
    -------------------------------------------------------------------------
DATA_C
  Relative segment, address: CODE_AREA 00009990 - 00009997 (0x8 bytes), align: 2
  Segment part 24.
           ENTRY                   ADDRESS         REF BY
           =====                   =======         ======
           STR_ENDSUBMENU1         00009990        doSubMenuJob (getConfig)
    -------------------------------------------------------------------------
DATA_C
  Relative segment, address: CODE_AREA 00009998 - 000099A3 (0xc bytes), align: 2
  Segment part 25.
           ENTRY                   ADDRESS         REF BY
           =====                   =======         ======
           STR_ENDSUBMENU2         00009998        doSubMenuJob (getConfig)
    -------------------------------------------------------------------------
DATA_C
  Relative segment, address: CODE_AREA 000099A4 - 000099AB (0x8 bytes), align: 2
  Segment part 26.
           ENTRY                   ADDRESS         REF BY
           =====                   =======         ======
           STR_SUBMENU1            000099A4        Segment part 88 (getConfig)
    -------------------------------------------------------------------------
DATA_C
  Relative segment, address: CODE_AREA 00009AEC - 00009AEE (0x3 bytes), align: 0
  Segment part 27.
           ENTRY                   ADDRESS         REF BY
           =====                   =======         ======
           STR_SUBMENU2            00009AEC        Segment part 87 (getConfig)
    -------------------------------------------------------------------------
DATA_C
  Relative segment, address: CODE_AREA 00009AEF - 00009AF1 (0x3 bytes), align: 0
  Segment part 28.
           ENTRY                   ADDRESS         REF BY
           =====                   =======         ======
           STR_TEMPLATE1           00009AEF        readConfig (getConfig)
    -------------------------------------------------------------------------
DATA_C
  Relative segment, address: CODE_AREA 000099AC - 000099B7 (0xc bytes), align: 2
  Segment part 29.
           ENTRY                   ADDRESS         REF BY
           =====                   =======         ======
           STR_TEMPLATE2           000099AC        readConfig (getConfig)
    -------------------------------------------------------------------------
DATA_C
  Relative segment, address: CODE_AREA 000099B8 - 000099BF (0x8 bytes), align: 2
  Segment part 30.
           ENTRY                   ADDRESS         REF BY
           =====                   =======         ======
           STR_ENDTEMPLATE1        000099B8        doTemplateWork (getConfig)
    -------------------------------------------------------------------------
DATA_C
  Relative segment, address: CODE_AREA 000099C0 - 000099CB (0xc bytes), align: 2
  Segment part 31.
           ENTRY                   ADDRESS         REF BY
           =====                   =======         ======
           STR_ENDTEMPLATE2        000099C0        doTemplateWork (getConfig)
    -------------------------------------------------------------------------
DATA_C
  Relative segment, address: CODE_AREA 000099CC - 000099DB (0x10 bytes), align: 2
  Segment part 32.
           ENTRY                   ADDRESS         REF BY
           =====                   =======         ======
           STR_USETEMPLATE1        000099CC        doItemJob (getConfig)
    -------------------------------------------------------------------------
DATA_C
  Relative segment, address: CODE_AREA 000099DC - 000099E3 (0x8 bytes), align: 2
  Segment part 33.
           ENTRY                   ADDRESS         REF BY
           =====                   =======         ======
           STR_USRTEMPLATE2        000099DC        doItemJob (getConfig)
    -------------------------------------------------------------------------
DATA_C
  Relative segment, address: CODE_AREA 000099E4 - 000099EF (0xc bytes), align: 2
  Segment part 34.
           ENTRY                   ADDRESS         REF BY
           =====                   =======         ======
           STR_MS1                 000099E4        doItemJob (getConfig)
    -------------------------------------------------------------------------
DATA_C
  Relative segment, address: CODE_AREA 000099F0 - 000099F7 (0x8 bytes), align: 2
  Segment part 35.
           ENTRY                   ADDRESS         REF BY
           =====                   =======         ======
           STR_MS2                 000099F0        doItemJob (getConfig)
    -------------------------------------------------------------------------
DATA_C
  Relative segment, address: CODE_AREA 000099F8 - 000099FF (0x8 bytes), align: 2
  Segment part 36.
           ENTRY                   ADDRESS         REF BY
           =====                   =======         ======
           STR_DISPF1              000099F8        addToPatchInfo (getConfig)
    -------------------------------------------------------------------------
DATA_C
  Relative segment, address: CODE_AREA 00009A00 - 00009A0B (0xc bytes), align: 2
  Segment part 37.
           ENTRY                   ADDRESS         REF BY
           =====                   =======         ======
           STR_DISPF2              00009A00        addToPatchInfo (getConfig)
    -------------------------------------------------------------------------
DATA_C
  Relative segment, address: CODE_AREA 00009A0C - 00009A0F (0x4 bytes), align: 2
  Segment part 38.
           ENTRY                   ADDRESS         REF BY
           =====                   =======         ======
           STR_RANGE1              00009A0C        doItemJob (getConfig)
    -------------------------------------------------------------------------
DATA_C
  Relative segment, address: CODE_AREA 00009A10 - 00009A17 (0x8 bytes), align: 2
  Segment part 39.
           ENTRY                   ADDRESS         REF BY
           =====                   =======         ======
           STR_RANGE2              00009A10        doItemJob (getConfig)
    -------------------------------------------------------------------------
DATA_C
  Relative segment, address: CODE_AREA 00009A18 - 00009A1B (0x4 bytes), align: 2
  Segment part 40.
           ENTRY                   ADDRESS         REF BY
           =====                   =======         ======
           STR_BYTES1              00009A18        doItemJob (getConfig)
    -------------------------------------------------------------------------
DATA_C
  Relative segment, address: CODE_AREA 00009A1C - 00009A23 (0x8 bytes), align: 2
  Segment part 41.
           ENTRY                   ADDRESS         REF BY
           =====                   =======         ======
           STR_BYTES2              00009A1C        doItemJob (getConfig)
    -------------------------------------------------------------------------
DATA_C
  Relative segment, address: CODE_AREA 00009A24 - 00009A27 (0x4 bytes), align: 2
  Segment part 42.
           ENTRY                   ADDRESS         REF BY
           =====                   =======         ======
           STR_INTS1               00009A24        doItemJob (getConfig)
    -------------------------------------------------------------------------
DATA_C
  Relative segment, address: CODE_AREA 00009A28 - 00009A2F (0x8 bytes), align: 2
  Segment part 43.
           ENTRY                   ADDRESS         REF BY
           =====                   =======         ======
           STR_INTS2               00009A28        doItemJob (getConfig)
    -------------------------------------------------------------------------
DATA_C
  Relative segment, address: CODE_AREA 00009A30 - 00009A37 (0x8 bytes), align: 2
  Segment part 44.
           ENTRY                   ADDRESS         REF BY
           =====                   =======         ======
           STR_CONST               00009A30        doItemJob (getConfig)
    -------------------------------------------------------------------------
CSTACK
  Segment part 1. NOT NEEDED.

    *************************************************************************

  FILE NAME : F:\SVN\cn\Master\Release_NEWSGOLD\Obj\visual.r79
  PROGRAM MODULE, NAME : visual

  SEGMENTS IN THE MODULE
  ======================
DATA_I
  Relative segment, address: DATA_AREA 000000E8 - 000000F7 (0x10 bytes), align: 2
  Segment part 10.            Intra module refs:   Segment part 90
           ENTRY                   ADDRESS         REF BY
           =====                   =======         ======
           colors                  000000E8 
    -------------------------------------------------------------------------
DATA_I
  Relative segment, address: DATA_AREA 000000F8 - 000000FB (0x4 bytes), align: 2
  Segment part 12.            Intra module refs:   Segment part 87
           ENTRY                   ADDRESS         REF BY
           =====                   =======         ======
           black                   000000F8 
    -------------------------------------------------------------------------
DATA_I
  Relative segment, address: DATA_AREA 000000FC - 000000FF (0x4 bytes), align: 2
  Segment part 14.            Intra module refs:   Segment part 89
           ENTRY                   ADDRESS         REF BY
           =====                   =======         ======
           white                   000000FC 
    -------------------------------------------------------------------------
DATA_Z
  Relative segment, address: CODE_AREA 00015BCC - 00015BCF (0x4 bytes), align: 2
  Segment part 16.            Intra module refs:   Segment part 88
           ENTRY                   ADDRESS         REF BY
           =====                   =======         ======
           transparent             00015BCC 
    -------------------------------------------------------------------------
DATA_C
  Relative segment, address: CODE_AREA 00009A38 - 00009A3F (0x8 bytes), align: 2
  Segment part 2.             Intra module refs:   Segment part 34
    -------------------------------------------------------------------------
DATA_C
  Relative segment, address: CODE_AREA 00009A40 - 00009A47 (0x8 bytes), align: 2
  Segment part 3.             Intra module refs:   Segment part 34
    -------------------------------------------------------------------------
DATA_C
  Relative segment, address: CODE_AREA 00009AF2 - 00009AF3 (0x2 bytes), align: 0
  Segment part 4.             Intra module refs:   Segment part 34
    -------------------------------------------------------------------------
DATA_C
  Segment part 5. NOT NEEDED.
    -------------------------------------------------------------------------
DATA_C
  Relative segment, address: CODE_AREA 00009A48 - 00009A4F (0x8 bytes), align: 2
  Segment part 6.             Intra module refs:   Segment part 65
    -------------------------------------------------------------------------
DATA_C
  Relative segment, address: CODE_AREA 00009A50 - 00009A57 (0x8 bytes), align: 2
  Segment part 7.             Intra module refs:   Segment part 135
    -------------------------------------------------------------------------
DATA_C
  Relative segment, address: CODE_AREA 00009A58 - 00009A5F (0x8 bytes), align: 2
  Segment part 8.             Intra module refs:   filelist_menu_iconhndl
    -------------------------------------------------------------------------
DATA_C
  Relative segment, address: CODE_AREA 00009A60 - 00009A67 (0x8 bytes), align: 2
  Segment part 9.             Intra module refs:   CreateRootMenu
    -------------------------------------------------------------------------
DATA_C
  Relative segment, address: CODE_AREA 00009A68 - 00009A6F (0x8 bytes), align: 2
  Segment part 17.            Intra module refs:   imgPointer
           ENTRY                   ADDRESS         REF BY
           =====                   =======         ======
           Pointer                 00009A68 
    -------------------------------------------------------------------------
DATA_C
  Relative segment, address: CODE_AREA 00009A70 - 00009A77 (0x8 bytes), align: 2
  Segment part 18.            Intra module refs:   Segment part 66
           ENTRY                   ADDRESS         REF BY
           =====                   =======         ======
           imgPointer              00009A70 
    -------------------------------------------------------------------------
CODE
  Segment part 41. NOT NEEDED.
    -------------------------------------------------------------------------
CODE
  Relative segment, address: CODE_AREA 00007B38 - 00007B93 (0x5c bytes), align: 2
  Segment part 42.            Intra module refs:   method0_xy
           ENTRY                   ADDRESS         REF BY
           =====                   =======         ======
           DrwImg                  00007B38 
               stack 1 = 00000000 ( 00000040 )
    -------------------------------------------------------------------------
CODE
  Segment part 43. NOT NEEDED.
    -------------------------------------------------------------------------
CODE
  Segment part 44. NOT NEEDED.
           ENTRY                   ADDRESS         REF BY
           =====                   =======         ======
           method0_rect            
               not allocated function
    -------------------------------------------------------------------------
CODE
  Segment part 45. NOT NEEDED.
    -------------------------------------------------------------------------
CODE
  Segment part 46. NOT NEEDED.
           ENTRY                   ADDRESS         REF BY
           =====                   =======         ======
           method1_rect            
               not allocated function
    -------------------------------------------------------------------------
CODE
  Segment part 47. NOT NEEDED.
    -------------------------------------------------------------------------
CODE
  Segment part 48. NOT NEEDED.
           ENTRY                   ADDRESS         REF BY
           =====                   =======         ======
           method2_rect            
               not allocated function
    -------------------------------------------------------------------------
CODE
  Segment part 49. NOT NEEDED.
    -------------------------------------------------------------------------
CODE
  Segment part 50. NOT NEEDED.
           ENTRY                   ADDRESS         REF BY
           =====                   =======         ======
           method3_rect            
               not allocated function
    -------------------------------------------------------------------------
CODE
  Segment part 51. NOT NEEDED.
    -------------------------------------------------------------------------
CODE
  Segment part 52. NOT NEEDED.
           ENTRY                   ADDRESS         REF BY
           =====                   =======         ======
           method4_rect            
               not allocated function
    -------------------------------------------------------------------------
CODE
  Segment part 53. NOT NEEDED.
    -------------------------------------------------------------------------
CODE
  Segment part 54. NOT NEEDED.
           ENTRY                   ADDRESS         REF BY
           =====                   =======         ======
           method5_rect            
               not allocated function
    -------------------------------------------------------------------------
CODE
  Segment part 55. NOT NEEDED.
    -------------------------------------------------------------------------
CODE
  Segment part 56. NOT NEEDED.
           ENTRY                   ADDRESS         REF BY
           =====                   =======         ======
           method7_rect            
               not allocated function
    -------------------------------------------------------------------------
CODE
  Segment part 57. NOT NEEDED.
    -------------------------------------------------------------------------
CODE
  Segment part 58. NOT NEEDED.
           ENTRY                   ADDRESS         REF BY
           =====                   =======         ======
           method8_rect            
               not allocated function
    -------------------------------------------------------------------------
CODE
  Segment part 59. NOT NEEDED.
    -------------------------------------------------------------------------
CODE
  Segment part 60. NOT NEEDED.
           ENTRY                   ADDRESS         REF BY
           =====                   =======         ======
           method9_rect            
               not allocated function
    -------------------------------------------------------------------------
CODE
  Segment part 61. NOT NEEDED.
    -------------------------------------------------------------------------
DATA_C
  Segment part 19. NOT NEEDED.
           ENTRY                   ADDRESS         REF BY
           =====                   =======         ======
           gui_methods_rect        
    -------------------------------------------------------------------------
DATA_C
  Segment part 20. NOT NEEDED.
           ENTRY                   ADDRESS         REF BY
           =====                   =======         ======
           Canvas_1                
    -------------------------------------------------------------------------
CODE
  Segment part 62. NOT NEEDED.
           ENTRY                   ADDRESS         REF BY
           =====                   =======         ======
           EditCoordinates         
               not allocated function
    -------------------------------------------------------------------------
CODE
  Segment part 63. NOT NEEDED.
    -------------------------------------------------------------------------
CODE
  Relative segment, address: CODE_AREA 00007B94 - 00007D37 (0x1a4 bytes), align: 2
  Segment part 64.            Intra module refs:   gui_methods_xy
           ENTRY                   ADDRESS         REF BY
           =====                   =======         ======
           method0_xy              00007B94 
               stack 1 = 00000000 ( 00000038 )
    -------------------------------------------------------------------------
CODE
  Relative segment, address: CODE_AREA 00007D38 - 00007D3B (0x4 bytes), align: 2
  Segment part 65.            Intra module refs:   method0_xy
    -------------------------------------------------------------------------
CODE
  Relative segment, address: CODE_AREA 00007D3C - 00007D3F (0x4 bytes), align: 2
  Segment part 66.            Intra module refs:   method0_xy
    -------------------------------------------------------------------------
CODE
  Segment part 67. NOT NEEDED.
    -------------------------------------------------------------------------
CODE
  Relative segment, address: CODE_AREA 00007D40 - 00007D5F (0x20 bytes), align: 2
  Segment part 68.            Intra module refs:   gui_methods_xy
           ENTRY                   ADDRESS         REF BY
           =====                   =======         ======
           method1_xy              00007D40 
               stack 1 = 00000000 ( 00000008 )
    -------------------------------------------------------------------------
CODE
  Segment part 69. NOT NEEDED.
    -------------------------------------------------------------------------
CODE
  Relative segment, address: CODE_AREA 00007D60 - 00007D7B (0x1c bytes), align: 2
  Segment part 70.            Intra module refs:   gui_methods_xy
           ENTRY                   ADDRESS         REF BY
           =====                   =======         ======
           method2_xy              00007D60 
               stack 1 = 00000000 ( 00000008 )
    -------------------------------------------------------------------------
CODE
  Segment part 71. NOT NEEDED.
    -------------------------------------------------------------------------
CODE
  Relative segment, address: CODE_AREA 00007D7C - 00007D87 (0xc bytes), align: 2
  Segment part 72.            Intra module refs:   gui_methods_xy
           ENTRY                   ADDRESS         REF BY
           =====                   =======         ======
           method3_xy              00007D7C 
    -------------------------------------------------------------------------
CODE
  Segment part 73. NOT NEEDED.
    -------------------------------------------------------------------------
CODE
  Relative segment, address: CODE_AREA 00007D88 - 00007D9B (0x14 bytes), align: 2
  Segment part 74.            Intra module refs:   gui_methods_xy
           ENTRY                   ADDRESS         REF BY
           =====                   =======         ======
           method4_xy              00007D88 
    -------------------------------------------------------------------------
CODE
  Segment part 75. NOT NEEDED.
    -------------------------------------------------------------------------
CODE
  Relative segment, address: CODE_AREA 00007D9C - 00007F9B (0x200 bytes), align: 2
  Segment part 76.            Intra module refs:   gui_methods_xy
           ENTRY                   ADDRESS         REF BY
           =====                   =======         ======
           method5_xy              00007D9C 
               stack 1 = 00000000 ( 00000010 )
    -------------------------------------------------------------------------
CODE
  Segment part 77. NOT NEEDED.
    -------------------------------------------------------------------------
CODE
  Relative segment, address: CODE_AREA 00007F9C - 00007F9F (0x4 bytes), align: 2
  Segment part 78.            Intra module refs:   gui_methods_xy
           ENTRY                   ADDRESS         REF BY
           =====                   =======         ======
           method7_xy              00007F9C 
               stack 1 = 00000000 ( 00000004 )
    -------------------------------------------------------------------------
CODE
  Segment part 79. NOT NEEDED.
    -------------------------------------------------------------------------
CODE
  Relative segment, address: CODE_AREA 00007FA0 - 00007FA7 (0x8 bytes), align: 2
  Segment part 80.            Intra module refs:   gui_methods_xy
           ENTRY                   ADDRESS         REF BY
           =====                   =======         ======
           method8_xy              00007FA0 
    -------------------------------------------------------------------------
CODE
  Segment part 81. NOT NEEDED.
    -------------------------------------------------------------------------
CODE
  Relative segment, address: CODE_AREA 00007FA8 - 00007FAF (0x8 bytes), align: 2
  Segment part 82.            Intra module refs:   gui_methods_xy
           ENTRY                   ADDRESS         REF BY
           =====                   =======         ======
           method9_xy              00007FA8 
    -------------------------------------------------------------------------
CODE
  Segment part 83. NOT NEEDED.
    -------------------------------------------------------------------------
DATA_C
  Relative segment, address: CODE_AREA 00009A78 - 00009AA3 (0x2c bytes), align: 2
  Segment part 21.            Intra module refs:   EditPostionGUI
           ENTRY                   ADDRESS         REF BY
           =====                   =======         ======
           gui_methods_xy          00009A78 
    -------------------------------------------------------------------------
DATA_C
  Relative segment, address: CODE_AREA 00009AA4 - 00009AAB (0x8 bytes), align: 2
  Segment part 22.            Intra module refs:   EditPostionGUI
           ENTRY                   ADDRESS         REF BY
           =====                   =======         ======
           Canvas_xy               00009AA4 
    -------------------------------------------------------------------------
CODE
  Relative segment, address: CODE_AREA 00007FB0 - 00008057 (0xa8 bytes), align: 2
  Segment part 84.
           ENTRY                   ADDRESS         REF BY
           =====                   =======         ======
           EditPostionGUI          00007FB0        edOnKey (main)
               stack 1 = 00000000 ( 00000018 )
    -------------------------------------------------------------------------
CODE
  Segment part 85. NOT NEEDED.
    -------------------------------------------------------------------------
CODE
  Relative segment, address: CODE_AREA 00008058 - 000082FF (0x2a8 bytes), align: 2
  Segment part 86.            Intra module refs:   gui_methods_2
           ENTRY                   ADDRESS         REF BY
           =====                   =======         ======
           method0_2               00008058 
               stack 1 = 00000000 ( 0000005C )
    -------------------------------------------------------------------------
CODE
  Relative segment, address: CODE_AREA 00008300 - 00008303 (0x4 bytes), align: 2
  Segment part 87.            Intra module refs:   method0_2
                                                   method0_xy
    -------------------------------------------------------------------------
CODE
  Relative segment, address: CODE_AREA 00008304 - 00008307 (0x4 bytes), align: 2
  Segment part 88.            Intra module refs:   method0_2
                                                   method0_xy
    -------------------------------------------------------------------------
CODE
  Relative segment, address: CODE_AREA 00008308 - 0000830B (0x4 bytes), align: 2
  Segment part 89.            Intra module refs:   method0_2
                                                   method0_xy
    -------------------------------------------------------------------------
CODE
  Relative segment, address: CODE_AREA 0000830C - 0000830F (0x4 bytes), align: 2
  Segment part 90.            Intra module refs:   method0_2
                                                   method0_xy
    -------------------------------------------------------------------------
CODE
  Segment part 91. NOT NEEDED.
    -------------------------------------------------------------------------
CODE
  Relative segment, address: CODE_AREA 00008310 - 0000832F (0x20 bytes), align: 2
  Segment part 92.            Intra module refs:   gui_methods_2
           ENTRY                   ADDRESS         REF BY
           =====                   =======         ======
           method1_2               00008310 
               stack 1 = 00000000 ( 00000008 )
    -------------------------------------------------------------------------
CODE
  Segment part 93. NOT NEEDED.
    -------------------------------------------------------------------------
CODE
  Relative segment, address: CODE_AREA 00008330 - 0000834B (0x1c bytes), align: 2
  Segment part 94.            Intra module refs:   gui_methods_2
           ENTRY                   ADDRESS         REF BY
           =====                   =======         ======
           method2_2               00008330 
               stack 1 = 00000000 ( 00000008 )
    -------------------------------------------------------------------------
CODE
  Segment part 95. NOT NEEDED.
    -------------------------------------------------------------------------
CODE
  Relative segment, address: CODE_AREA 0000834C - 00008357 (0xc bytes), align: 2
  Segment part 96.            Intra module refs:   gui_methods_2
           ENTRY                   ADDRESS         REF BY
           =====                   =======         ======
           method3_2               0000834C 
    -------------------------------------------------------------------------
CODE
  Segment part 97. NOT NEEDED.
    -------------------------------------------------------------------------
CODE
  Relative segment, address: CODE_AREA 00008358 - 0000836B (0x14 bytes), align: 2
  Segment part 98.            Intra module refs:   gui_methods_2
           ENTRY                   ADDRESS         REF BY
           =====                   =======         ======
           method4_2               00008358 
    -------------------------------------------------------------------------
CODE
  Segment part 99. NOT NEEDED.
    -------------------------------------------------------------------------
CODE
  Relative segment, address: CODE_AREA 0000836C - 0000857B (0x210 bytes), align: 2
  Segment part 100.           Intra module refs:   gui_methods_2
           ENTRY                   ADDRESS         REF BY
           =====                   =======         ======
           method5_2               0000836C 
               stack 1 = 00000000 ( 0000001C )
    -------------------------------------------------------------------------
CODE
  Segment part 101. NOT NEEDED.
    -------------------------------------------------------------------------
CODE
  Relative segment, address: CODE_AREA 0000857C - 0000857F (0x4 bytes), align: 2
  Segment part 102.           Intra module refs:   gui_methods_2
           ENTRY                   ADDRESS         REF BY
           =====                   =======         ======
           method7_2               0000857C 
               stack 1 = 00000000 ( 00000004 )
    -------------------------------------------------------------------------
CODE
  Segment part 103. NOT NEEDED.
    -------------------------------------------------------------------------
CODE
  Relative segment, address: CODE_AREA 00008580 - 00008587 (0x8 bytes), align: 2
  Segment part 104.           Intra module refs:   gui_methods_2
           ENTRY                   ADDRESS         REF BY
           =====                   =======         ======
           method8_2               00008580 
    -------------------------------------------------------------------------
CODE
  Segment part 105. NOT NEEDED.
    -------------------------------------------------------------------------
CODE
  Relative segment, address: CODE_AREA 00008588 - 0000858F (0x8 bytes), align: 2
  Segment part 106.           Intra module refs:   gui_methods_2
           ENTRY                   ADDRESS         REF BY
           =====                   =======         ======
           method9_2               00008588 
    -------------------------------------------------------------------------
CODE
  Segment part 107. NOT NEEDED.
    -------------------------------------------------------------------------
DATA_C
  Relative segment, address: CODE_AREA 00009AAC - 00009AD7 (0x2c bytes), align: 2
  Segment part 23.            Intra module refs:   EditColors
           ENTRY                   ADDRESS         REF BY
           =====                   =======         ======
           gui_methods_2           00009AAC 
    -------------------------------------------------------------------------
DATA_C
  Relative segment, address: CODE_AREA 00009AD8 - 00009ADF (0x8 bytes), align: 2
  Segment part 24.            Intra module refs:   EditColors
           ENTRY                   ADDRESS         REF BY
           =====                   =======         ======
           Canvas_2                00009AD8 
    -------------------------------------------------------------------------
CODE
  Relative segment, address: CODE_AREA 00008590 - 00008627 (0x98 bytes), align: 2
  Segment part 108.
           ENTRY                   ADDRESS         REF BY
           =====                   =======         ======
           EditColors              00008590        edOnKey (main)
               stack 1 = 00000000 ( 0000000C )
    -------------------------------------------------------------------------
CODE
  Segment part 109. NOT NEEDED.
    -------------------------------------------------------------------------
DATA_C
  Segment part 25. NOT NEEDED.
           ENTRY                   ADDRESS         REF BY
           =====                   =======         ======
           col_editor_minus11      
    -------------------------------------------------------------------------
DATA_Z
  Segment part 26. NOT NEEDED.
           ENTRY                   ADDRESS         REF BY
           =====                   =======         ======
           colorForEdit            
    -------------------------------------------------------------------------
DATA_C
  Segment part 27. NOT NEEDED.
           ENTRY                   ADDRESS         REF BY
           =====                   =======         ======
           MAINCSM_2               
    -------------------------------------------------------------------------
CODE
  Segment part 110. NOT NEEDED.
           ENTRY                   ADDRESS         REF BY
           =====                   =======         ======
           col_editor_csm_oncreate
                                   
               not allocated function
    -------------------------------------------------------------------------
CODE
  Segment part 111. NOT NEEDED.
    -------------------------------------------------------------------------
CODE
  Segment part 112. NOT NEEDED.
           ENTRY                   ADDRESS         REF BY
           =====                   =======         ======
           col_editor_csm_onmessage
                                   
               not allocated function
    -------------------------------------------------------------------------
CODE
  Segment part 113. NOT NEEDED.
    -------------------------------------------------------------------------
CODE
  Segment part 114. NOT NEEDED.
           ENTRY                   ADDRESS         REF BY
           =====                   =======         ======
           col_editor_csm_onclose
                                   
               not allocated function
    -------------------------------------------------------------------------
CODE
  Segment part 115. NOT NEEDED.
    -------------------------------------------------------------------------
CODE
  Segment part 116. NOT NEEDED.
           ENTRY                   ADDRESS         REF BY
           =====                   =======         ======
           col_editor_csm          
               not allocated function
    -------------------------------------------------------------------------
CODE
  Segment part 117. NOT NEEDED.
    -------------------------------------------------------------------------
CODE
  Segment part 118. NOT NEEDED.
    -------------------------------------------------------------------------
DATA_Z
  Relative segment, address: CODE_AREA 00015BD0 - 00015BD3 (0x4 bytes), align: 2
  Segment part 28.            Intra module refs:   Segment part 128
           ENTRY                   ADDRESS         REF BY
           =====                   =======         ======
           fltop                   00015BD0 
    -------------------------------------------------------------------------
CODE
  Relative segment, address: CODE_AREA 00008628 - 00008663 (0x3c bytes), align: 2
  Segment part 119.           Intra module refs:   CreateRootMenu
                                                   FindFiles
                                                   filelist_menu_ghook
           ENTRY                   ADDRESS         REF BY
           =====                   =======         ======
           Free_FLIST              00008628 
               stack 1 = 00000000 ( 00000008 )
    -------------------------------------------------------------------------
CODE
  Segment part 120. NOT NEEDED.
    -------------------------------------------------------------------------
DATA_C
  Relative segment, address: CODE_AREA 00009AF4 - 00009AF6 (0x3 bytes), align: 0
  Segment part 29.            Intra module refs:   FindFiles
           ENTRY                   ADDRESS         REF BY
           =====                   =======         ======
           back                    00009AF4 
    -------------------------------------------------------------------------
CODE
  Relative segment, address: CODE_AREA 00008664 - 00008693 (0x30 bytes), align: 2
  Segment part 121.           Intra module refs:   AddToFList
                                                   FindFiles
           ENTRY                   ADDRESS         REF BY
           =====                   =======         ======
           strcmp_nocase           00008664 
    -------------------------------------------------------------------------
CODE
  Segment part 122. NOT NEEDED.
    -------------------------------------------------------------------------
CODE
  Relative segment, address: CODE_AREA 00008694 - 00008743 (0xb0 bytes), align: 2
  Segment part 123.           Intra module refs:   CreateRootMenu
                                                   FindFiles
           ENTRY                   ADDRESS         REF BY
           =====                   =======         ======
           AddToFList              00008694 
               stack 1 = 00000000 ( 00000018 )
    -------------------------------------------------------------------------
CODE
  Segment part 124. NOT NEEDED.
    -------------------------------------------------------------------------
CODE
  Relative segment, address: CODE_AREA 00008744 - 0000891F (0x1dc bytes), align: 2
  Segment part 125.           Intra module refs:   filelist_menu_onkey
                                                   open_select_file_gui
           ENTRY                   ADDRESS         REF BY
           =====                   =======         ======
           FindFiles               00008744 
               stack 1 = 00000000 ( 000004E8 )
    -------------------------------------------------------------------------
CODE
  Segment part 126. NOT NEEDED.
    -------------------------------------------------------------------------
CODE
  Relative segment, address: CODE_AREA 00008920 - 00008963 (0x44 bytes), align: 2
  Segment part 127.           Intra module refs:   FindFLISTtByN
           ENTRY                   ADDRESS         REF BY
           =====                   =======         ======
           FindFLISTtByNS          00008920 
    -------------------------------------------------------------------------
CODE
  Relative segment, address: CODE_AREA 00008964 - 00008967 (0x4 bytes), align: 2
  Segment part 128.           Intra module refs:   AddToFList
                                                   FindFLISTtByNS
                                                   Free_FLIST
    -------------------------------------------------------------------------
CODE
  Segment part 129. NOT NEEDED.
    -------------------------------------------------------------------------
CODE
  Relative segment, address: CODE_AREA 00008968 - 000089BB (0x54 bytes), align: 2
  Segment part 130.           Intra module refs:   filelist_menu_iconhndl
                                                   filelist_menu_onkey
           ENTRY                   ADDRESS         REF BY
           =====                   =======         ======
           FindFLISTtByN           00008968 
               stack 1 = 00000000 ( 00000008 )
    -------------------------------------------------------------------------
CODE
  Segment part 131. NOT NEEDED.
    -------------------------------------------------------------------------
CODE
  Relative segment, address: CODE_AREA 000089BC - 00008A07 (0x4c bytes), align: 2
  Segment part 132.           Intra module refs:   filelist_menu_onkey
           ENTRY                   ADDRESS         REF BY
           =====                   =======         ======
           SavePath                000089BC 
               stack 1 = 00000000 ( 0000003C )
    -------------------------------------------------------------------------
CODE
  Segment part 133. NOT NEEDED.
    -------------------------------------------------------------------------
DATA_Z
  Relative segment, address: CODE_AREA 00015BD4 - 00015C53 (0x80 bytes), align: 2
  Segment part 30.            Intra module refs:   Segment part 144
                                                   Segment part 38
           ENTRY                   ADDRESS         REF BY
           =====                   =======         ======
           header                  00015BD4 
    -------------------------------------------------------------------------
CODE
  Relative segment, address: CODE_AREA 00008A08 - 00008AFF (0xf8 bytes), align: 2
  Segment part 134.           Intra module refs:   Segment part 40
           ENTRY                   ADDRESS         REF BY
           =====                   =======         ======
           filelist_menu_onkey     00008A08 
               stack 1 = 00000000 ( 00000014 )
    -------------------------------------------------------------------------
CODE
  Relative segment, address: CODE_AREA 00008B00 - 00008B03 (0x4 bytes), align: 2
  Segment part 135.           Intra module refs:   FindFiles
                                                   filelist_menu_onkey
    -------------------------------------------------------------------------
CODE
  Segment part 136. NOT NEEDED.
    -------------------------------------------------------------------------
CODE
  Relative segment, address: CODE_AREA 00008B04 - 00008B3B (0x38 bytes), align: 2
  Segment part 137.           Intra module refs:   Segment part 40
           ENTRY                   ADDRESS         REF BY
           =====                   =======         ======
           filelist_menu_ghook     00008B04 
               stack 1 = 00000000 ( 0000000C )
    -------------------------------------------------------------------------
CODE
  Segment part 138. NOT NEEDED.
    -------------------------------------------------------------------------
CODE
  Relative segment, address: CODE_AREA 00008B3C - 00008C0B (0xd0 bytes), align: 2
  Segment part 139.           Intra module refs:   Segment part 40
           ENTRY                   ADDRESS         REF BY
           =====                   =======         ======
           filelist_menu_iconhndl
                                   00008B3C 
               stack 1 = 00000000 ( 0000001C )
    -------------------------------------------------------------------------
CODE
  Segment part 140. NOT NEEDED.
    -------------------------------------------------------------------------
DATA_I
  Relative segment, address: DATA_AREA 00000100 - 0000010B (0xc bytes), align: 2
  Segment part 31.            Intra module refs:   Segment part 40
           ENTRY                   ADDRESS         REF BY
           =====                   =======         ======
           fmenusoftkeys           00000100 
    -------------------------------------------------------------------------
DATA_I
  Relative segment, address: DATA_AREA 0000010C - 00000123 (0x18 bytes), align: 2
  Segment part 33.            Intra module refs:   Segment part 36
           ENTRY                   ADDRESS         REF BY
           =====                   =======         ======
           fmenu_sk                0000010C 
    -------------------------------------------------------------------------
DATA_I
  Relative segment, address: DATA_AREA 00000124 - 0000012B (0x8 bytes), align: 2
  Segment part 35.            Intra module refs:   Segment part 40
           ENTRY                   ADDRESS         REF BY
           =====                   =======         ======
           fmenu_skt               00000124 
    -------------------------------------------------------------------------
DATA_I
  Relative segment, address: DATA_AREA 0000012C - 0000013F (0x14 bytes), align: 2
  Segment part 37.            Intra module refs:   open_select_file_gui
           ENTRY                   ADDRESS         REF BY
           =====                   =======         ======
           filelist_HDR            0000012C 
    -------------------------------------------------------------------------
DATA_I
  Relative segment, address: DATA_AREA 00000140 - 0000016B (0x2c bytes), align: 2
  Segment part 39.            Intra module refs:   open_select_file_gui
           ENTRY                   ADDRESS         REF BY
           =====                   =======         ======
           filelist_STRUCT         00000140 
    -------------------------------------------------------------------------
CODE
  Relative segment, address: CODE_AREA 00008C0C - 00008C8F (0x84 bytes), align: 2
  Segment part 141.           Intra module refs:   filelist_menu_onkey
                                                   open_select_file_gui
           ENTRY                   ADDRESS         REF BY
           =====                   =======         ======
           CreateRootMenu          00008C0C 
               stack 1 = 00000000 ( 00000030 )
    -------------------------------------------------------------------------
CODE
  Segment part 142. NOT NEEDED.
    -------------------------------------------------------------------------
CODE
  Relative segment, address: CODE_AREA 00008C90 - 00008DAB (0x11c bytes), align: 2
  Segment part 143.
           ENTRY                   ADDRESS         REF BY
           =====                   =======         ======
           open_select_file_gui    00008C90        on_sdec (main)
                                                   on_sfec (main)
               stack 1 = 00000000 ( 000000D8 )
    -------------------------------------------------------------------------
CODE
  Relative segment, address: CODE_AREA 00008DAC - 00008DAF (0x4 bytes), align: 2
  Segment part 144.           Intra module refs:   CreateRootMenu
                                                   filelist_menu_onkey
                                                   open_select_file_gui
    -------------------------------------------------------------------------
CODE
  Segment part 145. NOT NEEDED.Intra module refs   method7_2
                                                   method7_xy
    -------------------------------------------------------------------------
CSTACK
  Segment part 1. NOT NEEDED.
    -------------------------------------------------------------------------
DATA_ID
  Relative segment, address: CODE_AREA 000000E8 - 000000F7 (0x10 bytes), align: 2
  Segment part 11.            Intra module refs:   colors
    -------------------------------------------------------------------------
DATA_ID
  Relative segment, address: CODE_AREA 000000F8 - 000000FB (0x4 bytes), align: 2
  Segment part 13.            Intra module refs:   black
    -------------------------------------------------------------------------
DATA_ID
  Relative segment, address: CODE_AREA 000000FC - 000000FF (0x4 bytes), align: 2
  Segment part 15.            Intra module refs:   white
    -------------------------------------------------------------------------
DATA_ID
  Relative segment, address: CODE_AREA 00000100 - 0000010B (0xc bytes), align: 2
  Segment part 32.            Intra module refs:   fmenusoftkeys
    -------------------------------------------------------------------------
DATA_ID
  Relative segment, address: CODE_AREA 0000010C - 00000123 (0x18 bytes), align: 2
  Segment part 34.            Intra module refs:   fmenu_sk
    -------------------------------------------------------------------------
DATA_ID
  Relative segment, address: CODE_AREA 00000124 - 0000012B (0x8 bytes), align: 2
  Segment part 36.            Intra module refs:   fmenu_skt
    -------------------------------------------------------------------------
DATA_ID
  Relative segment, address: CODE_AREA 0000012C - 0000013F (0x14 bytes), align: 2
  Segment part 38.            Intra module refs:   filelist_HDR
    -------------------------------------------------------------------------
DATA_ID
  Relative segment, address: CODE_AREA 00000140 - 0000016B (0x2c bytes), align: 2
  Segment part 40.            Intra module refs:   filelist_STRUCT
    -------------------------------------------------------------------------
INITTAB
  Segment part 146. TENTATIVE. Used definition from getConfig
           ENTRY                   ADDRESS         REF BY
           =====                   =======         ======
           ?init?tab?DATA_Z        
    -------------------------------------------------------------------------
DATA_ID
  Segment part 147. TENTATIVE. Used definition from main
           ENTRY                   ADDRESS         REF BY
           =====                   =======         ======
           ?*?DATA_ID              
    -------------------------------------------------------------------------
INITTAB
  Segment part 148. TENTATIVE. Used definition from main
           ENTRY                   ADDRESS         REF BY
           =====                   =======         ======
           ?init?tab?DATA_I        




                ****************************************
                *                                      *
                *            MODULE SUMMARY            *
                *                                      *
                ****************************************

Module             CODE   DATA
------             ----   ----
                  (Rel)  (Rel)
func                  8
getConfig        64 224
  + shared           12
main              7 540     80
  + shared           12
optionMenu        6 160    152
ptcFileWork       2 652
string            3 068
usedstr             326
visual            5 169    132
N/A (alignment)
------           ------    ---
Total:           89 171    364


                ****************************************
                *                                      *
                *              CALL GRAPH              *
                *                                      *
                ****************************************

  ->Sub-tree of type: Indirectly called function tree that does not make
                    : indirect calls (Is not an interrupt and is not flagged
                    : as not overlayable)
                             CSTACK
    | Stack used (prev) :  00000000
  01  menu_onkey
      | Stack used (prev) :  00000000
      | + function block  :  00000010
  <-Sub-tree of type: Indirectly called function tree that does not make
                    : indirect calls (Is not an interrupt and is not flagged
                    : as not overlayable)
    | Stack used          :  00000010


  ->Sub-tree of type: Indirectly called function tree that does not make
                    : indirect calls (Is not an interrupt and is not flagged
                    : as not overlayable)
                             CSTACK
    | Stack used (prev) :  00000000
  01  menu_iconhndl
      | Stack used (prev) :  00000000
      | + function block  :  0000001C
  <-Sub-tree of type: Indirectly called function tree that does not make
                    : indirect calls (Is not an interrupt and is not flagged
                    : as not overlayable)
    | Stack used          :  0000001C


  ->Sub-tree of type: Indirectly called function tree that does not make
                    : indirect calls (Is not an interrupt and is not flagged
                    : as not overlayable)
                             CSTACK
    | Stack used (prev) :  00000000
  01  menu_ghook
      | Stack used (prev) :  00000000
      | + function block  :  00000004
  <-Sub-tree of type: Indirectly called function tree that does not make
                    : indirect calls (Is not an interrupt and is not flagged
                    : as not overlayable)
    | Stack used          :  00000004


  ->Sub-tree of type: Indirectly called function tree that does not make
                    : indirect calls (Is not an interrupt and is not flagged
                    : as not overlayable)
                             CSTACK
    | Stack used (prev) :  00000000
  01  maincsm_oncreate
      | Stack used (prev) :  00000000
      | + function block  :  0000000C
  <-Sub-tree of type: Indirectly called function tree that does not make
                    : indirect calls (Is not an interrupt and is not flagged
                    : as not overlayable)
    | Stack used          :  0000000C


  ->Sub-tree of type: Indirectly called function tree that does not make
                    : indirect calls (Is not an interrupt and is not flagged
                    : as not overlayable)
                             CSTACK
    | Stack used (prev) :  00000000
  01  maincsm_onmessage
      | Stack used (prev) :  00000000
      | + function block  :  0000000C
  <-Sub-tree of type: Indirectly called function tree that does not make
                    : indirect calls (Is not an interrupt and is not flagged
                    : as not overlayable)
    | Stack used          :  0000000C


  ->Sub-tree of type: Indirectly called function tree that does not make
                    : indirect calls (Is not an interrupt and is not flagged
                    : as not overlayable)
                             CSTACK
    | Stack used (prev) :  00000000
  01  Killer
      | Stack used (prev) :  00000000
      | + function block  :  00000004
  <-Sub-tree of type: Indirectly called function tree that does not make
                    : indirect calls (Is not an interrupt and is not flagged
                    : as not overlayable)
    | Stack used          :  00000004


  ->Sub-tree of type: Indirectly called function tree that does not make
                    : indirect calls (Is not an interrupt and is not flagged
                    : as not overlayable)
                             CSTACK
    | Stack used (prev) :  00000000
  01  maincsm_onclose
      | Stack used (prev) :  00000000
      | + function block  :  00000004
  <-Sub-tree of type: Indirectly called function tree that does not make
                    : indirect calls (Is not an interrupt and is not flagged
                    : as not overlayable)
    | Stack used          :  00000004


  ->Sub-tree of type: Indirectly called function tree that does not make
                    : indirect calls (Is not an interrupt and is not flagged
                    : as not overlayable)
                             CSTACK
    | Stack used (prev) :  00000000
  01  ed_locret
      | Stack used (prev) :  00000000
      | + function block  :  00000000
  <-Sub-tree of type: Indirectly called function tree that does not make
                    : indirect calls (Is not an interrupt and is not flagged
                    : as not overlayable)
    | Stack used          :  00000000


  ->Sub-tree of type: Indirectly called function tree that does not make
                    : indirect calls (Is not an interrupt and is not flagged
                    : as not overlayable)
                             CSTACK
    | Stack used (prev) :  00000000
  01  on_sfec
      | Stack used (prev) :  00000000
      | + function block  :  00000010
  <-Sub-tree of type: Indirectly called function tree that does not make
                    : indirect calls (Is not an interrupt and is not flagged
                    : as not overlayable)
    | Stack used          :  00000010


  ->Sub-tree of type: Indirectly called function tree that does not make
                    : indirect calls (Is not an interrupt and is not flagged
                    : as not overlayable)
                             CSTACK
    | Stack used (prev) :  00000000
  01  on_sdec
      | Stack used (prev) :  00000000
      | + function block  :  00000008
  <-Sub-tree of type: Indirectly called function tree that does not make
                    : indirect calls (Is not an interrupt and is not flagged
                    : as not overlayable)
    | Stack used          :  00000008


  ->Sub-tree of type: Indirectly called function tree that does not make
                    : indirect calls (Is not an interrupt and is not flagged
                    : as not overlayable)
                             CSTACK
    | Stack used (prev) :  00000000
  01  edOnKey
      | Stack used (prev) :  00000000
      | + function block  :  00000250
  <-Sub-tree of type: Indirectly called function tree that does not make
                    : indirect calls (Is not an interrupt and is not flagged
                    : as not overlayable)
    | Stack used          :  00000250


  ->Sub-tree of type: Indirectly called function tree that does not make
                    : indirect calls (Is not an interrupt and is not flagged
                    : as not overlayable)
                             CSTACK
    | Stack used (prev) :  00000000
  01  edGHook
      | Stack used (prev) :  00000000
      | + function block  :  000002C4
  <-Sub-tree of type: Indirectly called function tree that does not make
                    : indirect calls (Is not an interrupt and is not flagged
                    : as not overlayable)
    | Stack used          :  000002C4


  ->Sub-tree of type: Indirectly called function tree that does not make
                    : indirect calls (Is not an interrupt and is not flagged
                    : as not overlayable)
                             CSTACK
    | Stack used (prev) :  00000000
  01  option_menu_ghook
      | Stack used (prev) :  00000000
      | + function block  :  00000004
  <-Sub-tree of type: Indirectly called function tree that does not make
                    : indirect calls (Is not an interrupt and is not flagged
                    : as not overlayable)
    | Stack used          :  00000004


  ->Sub-tree of type: Indirectly called function tree that does not make
                    : indirect calls (Is not an interrupt and is not flagged
                    : as not overlayable)
                             CSTACK
    | Stack used (prev) :  00000000
  01  menu_exit
      | Stack used (prev) :  00000000
      | + function block  :  00000004
  <-Sub-tree of type: Indirectly called function tree that does not make
                    : indirect calls (Is not an interrupt and is not flagged
                    : as not overlayable)
    | Stack used          :  00000004


  ->Sub-tree of type: Indirectly called function tree that does not make
                    : indirect calls (Is not an interrupt and is not flagged
                    : as not overlayable)
                             CSTACK
    | Stack used (prev) :  00000000
  01  menu_about
      | Stack used (prev) :  00000000
      | + function block  :  00000004
  <-Sub-tree of type: Indirectly called function tree that does not make
                    : indirect calls (Is not an interrupt and is not flagged
                    : as not overlayable)
    | Stack used          :  00000004


  ->Sub-tree of type: Indirectly called function tree that does not make
                    : indirect calls (Is not an interrupt and is not flagged
                    : as not overlayable)
                             CSTACK
    | Stack used (prev) :  00000000
  01  menu_profile
      | Stack used (prev) :  00000000
      | + function block  :  00000004
  <-Sub-tree of type: Indirectly called function tree that does not make
                    : indirect calls (Is not an interrupt and is not flagged
                    : as not overlayable)
    | Stack used          :  00000004


  ->Sub-tree of type: Indirectly called function tree that does not make
                    : indirect calls (Is not an interrupt and is not flagged
                    : as not overlayable)
                             CSTACK
    | Stack used (prev) :  00000000
  01  menu_del_all
      | Stack used (prev) :  00000000
      | + function block  :  00000004
  <-Sub-tree of type: Indirectly called function tree that does not make
                    : indirect calls (Is not an interrupt and is not flagged
                    : as not overlayable)
    | Stack used          :  00000004


  ->Sub-tree of type: Indirectly called function tree that does not make
                    : indirect calls (Is not an interrupt and is not flagged
                    : as not overlayable)
                             CSTACK
    | Stack used (prev) :  00000000
  01  menu_del_this
      | Stack used (prev) :  00000000
      | + function block  :  00000004
  <-Sub-tree of type: Indirectly called function tree that does not make
                    : indirect calls (Is not an interrupt and is not flagged
                    : as not overlayable)
    | Stack used          :  00000004


  ->Sub-tree of type: Indirectly called function tree that does not make
                    : indirect calls (Is not an interrupt and is not flagged
                    : as not overlayable)
                             CSTACK
    | Stack used (prev) :  00000000
  01  menu_del_unused
      | Stack used (prev) :  00000000
      | + function block  :  00000004
  <-Sub-tree of type: Indirectly called function tree that does not make
                    : indirect calls (Is not an interrupt and is not flagged
                    : as not overlayable)
    | Stack used          :  00000004


  ->Sub-tree of type: Indirectly called function tree that does not make
                    : indirect calls (Is not an interrupt and is not flagged
                    : as not overlayable)
                             CSTACK
    | Stack used (prev) :  00000000
  01  menu_info
      | Stack used (prev) :  00000000
      | + function block  :  00000004
  <-Sub-tree of type: Indirectly called function tree that does not make
                    : indirect calls (Is not an interrupt and is not flagged
                    : as not overlayable)
    | Stack used          :  00000004


  ->Sub-tree of type: Indirectly called function tree that does not make
                    : indirect calls (Is not an interrupt and is not flagged
                    : as not overlayable)
                             CSTACK
    | Stack used (prev) :  00000000
  01  menu_backup
      | Stack used (prev) :  00000000
      | + function block  :  00000004
  <-Sub-tree of type: Indirectly called function tree that does not make
                    : indirect calls (Is not an interrupt and is not flagged
                    : as not overlayable)
    | Stack used          :  00000004


  ->Sub-tree of type: Indirectly called function tree that does not make
                    : indirect calls (Is not an interrupt and is not flagged
                    : as not overlayable)
                             CSTACK
    | Stack used (prev) :  00000000
  01  menu_restore
      | Stack used (prev) :  00000000
      | + function block  :  00000004
  <-Sub-tree of type: Indirectly called function tree that does not make
                    : indirect calls (Is not an interrupt and is not flagged
                    : as not overlayable)
    | Stack used          :  00000004


  ->Sub-tree of type: Indirectly called function tree that does not make
                    : indirect calls (Is not an interrupt and is not flagged
                    : as not overlayable)
                             CSTACK
    | Stack used (prev) :  00000000
  01  menu_quit_without_rs
      | Stack used (prev) :  00000000
      | + function block  :  00000004
  <-Sub-tree of type: Indirectly called function tree that does not make
                    : indirect calls (Is not an interrupt and is not flagged
                    : as not overlayable)
    | Stack used          :  00000004


  ->Sub-tree of type: Indirectly called function tree that does not make
                    : indirect calls (Is not an interrupt and is not flagged
                    : as not overlayable)
                             CSTACK
    | Stack used (prev) :  00000000
  01  profile_menu_onkey
      | Stack used (prev) :  00000000
      | + function block  :  00000010
  <-Sub-tree of type: Indirectly called function tree that does not make
                    : indirect calls (Is not an interrupt and is not flagged
                    : as not overlayable)
    | Stack used          :  00000010


  ->Sub-tree of type: Indirectly called function tree that does not make
                    : indirect calls (Is not an interrupt and is not flagged
                    : as not overlayable)
                             CSTACK
    | Stack used (prev) :  00000000
  01  profile_menu_iconhndl
      | Stack used (prev) :  00000000
      | + function block  :  00000018
  <-Sub-tree of type: Indirectly called function tree that does not make
                    : indirect calls (Is not an interrupt and is not flagged
                    : as not overlayable)
    | Stack used          :  00000018


  ->Sub-tree of type: Indirectly called function tree that does not make
                    : indirect calls (Is not an interrupt and is not flagged
                    : as not overlayable)
                             CSTACK
    | Stack used (prev) :  00000000
  01  profile_menu_ghook
      | Stack used (prev) :  00000000
      | + function block  :  00000004
  <-Sub-tree of type: Indirectly called function tree that does not make
                    : indirect calls (Is not an interrupt and is not flagged
                    : as not overlayable)
    | Stack used          :  00000004


  ->Sub-tree of type: Indirectly called function tree that does not make
                    : indirect calls (Is not an interrupt and is not flagged
                    : as not overlayable)
                             CSTACK
    | Stack used (prev) :  00000000
  01  infoOnKey
      | Stack used (prev) :  00000000
      | + function block  :  00000000
  <-Sub-tree of type: Indirectly called function tree that does not make
                    : indirect calls (Is not an interrupt and is not flagged
                    : as not overlayable)
    | Stack used          :  00000000


  ->Sub-tree of type: Indirectly called function tree that does not make
                    : indirect calls (Is not an interrupt and is not flagged
                    : as not overlayable)
                             CSTACK
    | Stack used (prev) :  00000000
  01  infoGHook
      | Stack used (prev) :  00000000
      | + function block  :  00000004
  <-Sub-tree of type: Indirectly called function tree that does not make
                    : indirect calls (Is not an interrupt and is not flagged
                    : as not overlayable)
    | Stack used          :  00000004


  ->Sub-tree of type: Indirectly called function tree that does not make
                    : indirect calls (Is not an interrupt and is not flagged
                    : as not overlayable)
                             CSTACK
    | Stack used (prev) :  00000000
  01  info_locret
      | Stack used (prev) :  00000000
      | + function block  :  00000000
  <-Sub-tree of type: Indirectly called function tree that does not make
                    : indirect calls (Is not an interrupt and is not flagged
                    : as not overlayable)
    | Stack used          :  00000000


  ->Sub-tree of type: Indirectly called function tree that does not make
                    : indirect calls (Is not an interrupt and is not flagged
                    : as not overlayable)
                             CSTACK
    | Stack used (prev) :  00000000
  01  pathInputOnKey
      | Stack used (prev) :  00000000
      | + function block  :  000000B0
  <-Sub-tree of type: Indirectly called function tree that does not make
                    : indirect calls (Is not an interrupt and is not flagged
                    : as not overlayable)
    | Stack used          :  000000B0


  ->Sub-tree of type: Indirectly called function tree that does not make
                    : indirect calls (Is not an interrupt and is not flagged
                    : as not overlayable)
                             CSTACK
    | Stack used (prev) :  00000000
  01  pathInputGHook
      | Stack used (prev) :  00000000
      | + function block  :  00000004
  <-Sub-tree of type: Indirectly called function tree that does not make
                    : indirect calls (Is not an interrupt and is not flagged
                    : as not overlayable)
    | Stack used          :  00000004


  ->Sub-tree of type: Indirectly called function tree that does not make
                    : indirect calls (Is not an interrupt and is not flagged
                    : as not overlayable)
                             CSTACK
    | Stack used (prev) :  00000000
  01  method0_xy
      | Stack used (prev) :  00000000
      | + function block  :  00000038
  <-Sub-tree of type: Indirectly called function tree that does not make
                    : indirect calls (Is not an interrupt and is not flagged
                    : as not overlayable)
    | Stack used          :  00000038


  ->Sub-tree of type: Indirectly called function tree that does not make
                    : indirect calls (Is not an interrupt and is not flagged
                    : as not overlayable)
                             CSTACK
    | Stack used (prev) :  00000000
  01  method1_xy
      | Stack used (prev) :  00000000
      | + function block  :  00000008
  <-Sub-tree of type: Indirectly called function tree that does not make
                    : indirect calls (Is not an interrupt and is not flagged
                    : as not overlayable)
    | Stack used          :  00000008


  ->Sub-tree of type: Indirectly called function tree that does not make
                    : indirect calls (Is not an interrupt and is not flagged
                    : as not overlayable)
                             CSTACK
    | Stack used (prev) :  00000000
  01  method2_xy
      | Stack used (prev) :  00000000
      | + function block  :  00000008
  <-Sub-tree of type: Indirectly called function tree that does not make
                    : indirect calls (Is not an interrupt and is not flagged
                    : as not overlayable)
    | Stack used          :  00000008


  ->Sub-tree of type: Indirectly called function tree that does not make
                    : indirect calls (Is not an interrupt and is not flagged
                    : as not overlayable)
                             CSTACK
    | Stack used (prev) :  00000000
  01  method3_xy
      | Stack used (prev) :  00000000
      | + function block  :  00000000
  <-Sub-tree of type: Indirectly called function tree that does not make
                    : indirect calls (Is not an interrupt and is not flagged
                    : as not overlayable)
    | Stack used          :  00000000


  ->Sub-tree of type: Indirectly called function tree that does not make
                    : indirect calls (Is not an interrupt and is not flagged
                    : as not overlayable)
                             CSTACK
    | Stack used (prev) :  00000000
  01  method4_xy
      | Stack used (prev) :  00000000
      | + function block  :  00000000
  <-Sub-tree of type: Indirectly called function tree that does not make
                    : indirect calls (Is not an interrupt and is not flagged
                    : as not overlayable)
    | Stack used          :  00000000


  ->Sub-tree of type: Indirectly called function tree that does not make
                    : indirect calls (Is not an interrupt and is not flagged
                    : as not overlayable)
                             CSTACK
    | Stack used (prev) :  00000000
  01  method5_xy
      | Stack used (prev) :  00000000
      | + function block  :  00000010
  <-Sub-tree of type: Indirectly called function tree that does not make
                    : indirect calls (Is not an interrupt and is not flagged
                    : as not overlayable)
    | Stack used          :  00000010


  ->Sub-tree of type: Indirectly called function tree that does not make
                    : indirect calls (Is not an interrupt and is not flagged
                    : as not overlayable)
                             CSTACK
    | Stack used (prev) :  00000000
  01  method7_xy
      | Stack used (prev) :  00000000
      | + function block  :  00000004
  <-Sub-tree of type: Indirectly called function tree that does not make
                    : indirect calls (Is not an interrupt and is not flagged
                    : as not overlayable)
    | Stack used          :  00000004


  ->Sub-tree of type: Indirectly called function tree that does not make
                    : indirect calls (Is not an interrupt and is not flagged
                    : as not overlayable)
                             CSTACK
    | Stack used (prev) :  00000000
  01  method8_xy
      | Stack used (prev) :  00000000
      | + function block  :  00000000
  <-Sub-tree of type: Indirectly called function tree that does not make
                    : indirect calls (Is not an interrupt and is not flagged
                    : as not overlayable)
    | Stack used          :  00000000


  ->Sub-tree of type: Indirectly called function tree that does not make
                    : indirect calls (Is not an interrupt and is not flagged
                    : as not overlayable)
                             CSTACK
    | Stack used (prev) :  00000000
  01  method9_xy
      | Stack used (prev) :  00000000
      | + function block  :  00000000
  <-Sub-tree of type: Indirectly called function tree that does not make
                    : indirect calls (Is not an interrupt and is not flagged
                    : as not overlayable)
    | Stack used          :  00000000


  ->Sub-tree of type: Indirectly called function tree that does not make
                    : indirect calls (Is not an interrupt and is not flagged
                    : as not overlayable)
                             CSTACK
    | Stack used (prev) :  00000000
  01  method0_2
      | Stack used (prev) :  00000000
      | + function block  :  0000005C
  <-Sub-tree of type: Indirectly called function tree that does not make
                    : indirect calls (Is not an interrupt and is not flagged
                    : as not overlayable)
    | Stack used          :  0000005C


  ->Sub-tree of type: Indirectly called function tree that does not make
                    : indirect calls (Is not an interrupt and is not flagged
                    : as not overlayable)
                             CSTACK
    | Stack used (prev) :  00000000
  01  method1_2
      | Stack used (prev) :  00000000
      | + function block  :  00000008
  <-Sub-tree of type: Indirectly called function tree that does not make
                    : indirect calls (Is not an interrupt and is not flagged
                    : as not overlayable)
    | Stack used          :  00000008


  ->Sub-tree of type: Indirectly called function tree that does not make
                    : indirect calls (Is not an interrupt and is not flagged
                    : as not overlayable)
                             CSTACK
    | Stack used (prev) :  00000000
  01  method2_2
      | Stack used (prev) :  00000000
      | + function block  :  00000008
  <-Sub-tree of type: Indirectly called function tree that does not make
                    : indirect calls (Is not an interrupt and is not flagged
                    : as not overlayable)
    | Stack used          :  00000008


  ->Sub-tree of type: Indirectly called function tree that does not make
                    : indirect calls (Is not an interrupt and is not flagged
                    : as not overlayable)
                             CSTACK
    | Stack used (prev) :  00000000
  01  method3_2
      | Stack used (prev) :  00000000
      | + function block  :  00000000
  <-Sub-tree of type: Indirectly called function tree that does not make
                    : indirect calls (Is not an interrupt and is not flagged
                    : as not overlayable)
    | Stack used          :  00000000


  ->Sub-tree of type: Indirectly called function tree that does not make
                    : indirect calls (Is not an interrupt and is not flagged
                    : as not overlayable)
                             CSTACK
    | Stack used (prev) :  00000000
  01  method4_2
      | Stack used (prev) :  00000000
      | + function block  :  00000000
  <-Sub-tree of type: Indirectly called function tree that does not make
                    : indirect calls (Is not an interrupt and is not flagged
                    : as not overlayable)
    | Stack used          :  00000000


  ->Sub-tree of type: Indirectly called function tree that does not make
                    : indirect calls (Is not an interrupt and is not flagged
                    : as not overlayable)
                             CSTACK
    | Stack used (prev) :  00000000
  01  method5_2
      | Stack used (prev) :  00000000
      | + function block  :  0000001C
  <-Sub-tree of type: Indirectly called function tree that does not make
                    : indirect calls (Is not an interrupt and is not flagged
                    : as not overlayable)
    | Stack used          :  0000001C


  ->Sub-tree of type: Indirectly called function tree that does not make
                    : indirect calls (Is not an interrupt and is not flagged
                    : as not overlayable)
                             CSTACK
    | Stack used (prev) :  00000000
  01  method7_2
      | Stack used (prev) :  00000000
      | + function block  :  00000004
  <-Sub-tree of type: Indirectly called function tree that does not make
                    : indirect calls (Is not an interrupt and is not flagged
                    : as not overlayable)
    | Stack used          :  00000004


  ->Sub-tree of type: Indirectly called function tree that does not make
                    : indirect calls (Is not an interrupt and is not flagged
                    : as not overlayable)
                             CSTACK
    | Stack used (prev) :  00000000
  01  method8_2
      | Stack used (prev) :  00000000
      | + function block  :  00000000
  <-Sub-tree of type: Indirectly called function tree that does not make
                    : indirect calls (Is not an interrupt and is not flagged
                    : as not overlayable)
    | Stack used          :  00000000


  ->Sub-tree of type: Indirectly called function tree that does not make
                    : indirect calls (Is not an interrupt and is not flagged
                    : as not overlayable)
                             CSTACK
    | Stack used (prev) :  00000000
  01  method9_2
      | Stack used (prev) :  00000000
      | + function block  :  00000000
  <-Sub-tree of type: Indirectly called function tree that does not make
                    : indirect calls (Is not an interrupt and is not flagged
                    : as not overlayable)
    | Stack used          :  00000000


  ->Sub-tree of type: Indirectly called function tree that does not make
                    : indirect calls (Is not an interrupt and is not flagged
                    : as not overlayable)
                             CSTACK
    | Stack used (prev) :  00000000
  01  filelist_menu_onkey
      | Stack used (prev) :  00000000
      | + function block  :  00000014
  <-Sub-tree of type: Indirectly called function tree that does not make
                    : indirect calls (Is not an interrupt and is not flagged
                    : as not overlayable)
    | Stack used          :  00000014


  ->Sub-tree of type: Indirectly called function tree that does not make
                    : indirect calls (Is not an interrupt and is not flagged
                    : as not overlayable)
                             CSTACK
    | Stack used (prev) :  00000000
  01  filelist_menu_ghook
      | Stack used (prev) :  00000000
      | + function block  :  0000000C
  <-Sub-tree of type: Indirectly called function tree that does not make
                    : indirect calls (Is not an interrupt and is not flagged
                    : as not overlayable)
    | Stack used          :  0000000C


  ->Sub-tree of type: Indirectly called function tree that does not make
                    : indirect calls (Is not an interrupt and is not flagged
                    : as not overlayable)
                             CSTACK
    | Stack used (prev) :  00000000
  01  filelist_menu_iconhndl
      | Stack used (prev) :  00000000
      | + function block  :  0000001C
  <-Sub-tree of type: Indirectly called function tree that does not make
                    : indirect calls (Is not an interrupt and is not flagged
                    : as not overlayable)
    | Stack used          :  0000001C


  ->Sub-tree of type: Function tree
                             CSTACK
    | Stack used (prev) :  000002C4
  01  loadConfig
      | Stack used (prev) :  000002C4
      | + function block  :  000000BC
  <-Sub-tree of type: Function tree
    | Stack used          :  00000380


  ->Sub-tree of type: Function tree
                             CSTACK
    | Stack used (prev) :  00000380
  01  addPatchConfigList
      | Stack used (prev) :  00000380
      | + function block  :  00000004
  <-Sub-tree of type: Function tree
    | Stack used          :  00000384


  ->Sub-tree of type: Function tree
                             CSTACK
    | Stack used (prev) :  00000384
  01  addToPatchInfo
      | Stack used (prev) :  00000384
      | + function block  :  00000018
  <-Sub-tree of type: Function tree
    | Stack used          :  0000039C


  ->Sub-tree of type: Function tree
                             CSTACK
    | Stack used (prev) :  0000039C
  01  addPreItemToData
      | Stack used (prev) :  0000039C
      | + function block  :  00000000
  <-Sub-tree of type: Function tree
    | Stack used          :  0000039C


  ->Sub-tree of type: Function tree
                             CSTACK
    | Stack used (prev) :  0000039C
  01  addItemToConfig
      | Stack used (prev) :  0000039C
      | + function block  :  0000001C
  <-Sub-tree of type: Function tree
    | Stack used          :  000003B8


  ->Sub-tree of type: Function tree
                             CSTACK
    | Stack used (prev) :  000003B8
  01  addPrepareData
      | Stack used (prev) :  000003B8
      | + function block  :  00000020
  <-Sub-tree of type: Function tree
    | Stack used          :  000003D8


  ->Sub-tree of type: Function tree
                             CSTACK
    | Stack used (prev) :  000003D8
  01  addPreDataToCBoxItem
      | Stack used (prev) :  000003D8
      | + function block  :  00000018
  <-Sub-tree of type: Function tree
    | Stack used          :  000003F0


  ->Sub-tree of type: Function tree
                             CSTACK
    | Stack used (prev) :  000003F0
  01  addItemToCBox
      | Stack used (prev) :  000003F0
      | + function block  :  00000000
  <-Sub-tree of type: Function tree
    | Stack used          :  000003F0


  ->Sub-tree of type: Function tree
                             CSTACK
    | Stack used (prev) :  000003F0
  01  cboxItemColon
      | Stack used (prev) :  000003F0
      | + function block  :  0000001C
  <-Sub-tree of type: Function tree
    | Stack used          :  0000040C


  ->Sub-tree of type: Function tree
                             CSTACK
    | Stack used (prev) :  0000040C
  01  isThatItem
      | Stack used (prev) :  0000040C
      | + function block  :  00000000
  <-Sub-tree of type: Function tree
    | Stack used          :  0000040C


  ->Sub-tree of type: Function tree
                             CSTACK
    | Stack used (prev) :  0000040C
  01  findTemplate
      | Stack used (prev) :  0000040C
      | + function block  :  00000010
  <-Sub-tree of type: Function tree
    | Stack used          :  0000041C


  ->Sub-tree of type: Function tree
                             CSTACK
    | Stack used (prev) :  0000041C
  01  isCurrectItem
      | Stack used (prev) :  0000041C
      | + function block  :  00000008
  <-Sub-tree of type: Function tree
    | Stack used          :  00000424


  ->Sub-tree of type: Function tree
                             CSTACK
    | Stack used (prev) :  00000424
  01  doItemJob
      | Stack used (prev) :  00000424
      | + function block  :  000000B4
  <-Sub-tree of type: Function tree
    | Stack used          :  000004D8


  ->Sub-tree of type: Function tree
                             CSTACK
    | Stack used (prev) :  000004D8
  01  doSubMenuJob
      | Stack used (prev) :  000004D8
      | + function block  :  0000001C
  <-Sub-tree of type: Function tree
    | Stack used          :  000004F4


  ->Sub-tree of type: Function tree
                             CSTACK
    | Stack used (prev) :  000004F4
  01  addInfoToPatchInfo
      | Stack used (prev) :  000004F4
      | + function block  :  00000010
  <-Sub-tree of type: Function tree
    | Stack used          :  00000504


  ->Sub-tree of type: Function tree
                             CSTACK
    | Stack used (prev) :  00000504
  01  isPrepareItem
      | Stack used (prev) :  00000504
      | + function block  :  00000000
  <-Sub-tree of type: Function tree
    | Stack used          :  00000504


  ->Sub-tree of type: Function tree
                             CSTACK
    | Stack used (prev) :  00000504
  01  doTemplateWork
      | Stack used (prev) :  00000504
      | + function block  :  00000018
  <-Sub-tree of type: Function tree
    | Stack used          :  0000051C


  ->Sub-tree of type: Function tree
                             CSTACK
    | Stack used (prev) :  0000051C
  01  subMenuCopy
      | Stack used (prev) :  0000051C
      | + function block  :  00000028
  <-Sub-tree of type: Function tree
    | Stack used          :  00000544


  ->Sub-tree of type: Function tree
                             CSTACK
    | Stack used (prev) :  00000544
  01  readConfig
      | Stack used (prev) :  00000544
      | + function block  :  0000001C
  <-Sub-tree of type: Function tree
    | Stack used          :  00000560


  ->Sub-tree of type: Function tree
                             CSTACK
    | Stack used (prev) :  00000560
  01  freePatchItem
      | Stack used (prev) :  00000560
      | + function block  :  0000000C
  <-Sub-tree of type: Function tree
    | Stack used          :  0000056C


  ->Sub-tree of type: Function tree
                             CSTACK
    | Stack used (prev) :  0000056C
  01  reloadThisPatch
      | Stack used (prev) :  0000056C
      | + function block  :  00000018
  <-Sub-tree of type: Function tree
    | Stack used          :  00000584


  ->Sub-tree of type: Function tree
                             CSTACK
    | Stack used (prev) :  00000584
  01  swapPatchConfigList
      | Stack used (prev) :  00000584
      | + function block  :  00000020
  <-Sub-tree of type: Function tree
    | Stack used          :  000005A4


  ->Sub-tree of type: Function tree
                             CSTACK
    | Stack used (prev) :  000005A4
  01  sortPatchConfigList
      | Stack used (prev) :  000005A4
      | + function block  :  0000000C
  <-Sub-tree of type: Function tree
    | Stack used          :  000005B0


  ->Sub-tree of type: Function tree
                             CSTACK
    | Stack used (prev) :  000005B0
  01  fuckThemAll
      | Stack used (prev) :  000005B0
      | + function block  :  0000000C
  <-Sub-tree of type: Function tree
    | Stack used          :  000005BC


  ->Sub-tree of type: Function tree
                             CSTACK
    | Stack used (prev) :  000005BC
  01  getPatchConfigItem
      | Stack used (prev) :  000005BC
      | + function block  :  00000000
  <-Sub-tree of type: Function tree
    | Stack used          :  000005BC


  ->Sub-tree of type: Function tree
                             CSTACK
    | Stack used (prev) :  000005BC
  01  getMaxCBoxItem
      | Stack used (prev) :  000005BC
      | + function block  :  00000000
  <-Sub-tree of type: Function tree
    | Stack used          :  000005BC


  ->Sub-tree of type: Function tree
                             CSTACK
    | Stack used (prev) :  000005BC
  01  getCurCBoxItem
      | Stack used (prev) :  000005BC
      | + function block  :  00000000
  <-Sub-tree of type: Function tree
    | Stack used          :  000005BC


  ->Sub-tree of type: Function tree
                             CSTACK
    | Stack used (prev) :  000005BC
  01  getInitCBoxItem
      | Stack used (prev) :  000005BC
      | + function block  :  00000004
  <-Sub-tree of type: Function tree
    | Stack used          :  000005C0


  ->Sub-tree of type: Function tree
                             CSTACK
    | Stack used (prev) :  000005C0
  01  getAllPatchData
      | Stack used (prev) :  000005C0
      | + function block  :  00000008
  <-Sub-tree of type: Function tree
    | Stack used          :  000005C8


  ->Sub-tree of type: Function tree
                             CSTACK
    | Stack used (prev) :  000005C8
  01  setPatchOnOff
      | Stack used (prev) :  000005C8
      | + function block  :  00000010
  <-Sub-tree of type: Function tree
    | Stack used          :  000005D8


  ->Sub-tree of type: Function tree
                             CSTACK
    | Stack used (prev) :  000005D8
  01  getPatchOnOff
      | Stack used (prev) :  000005D8
      | + function block  :  00000000
  <-Sub-tree of type: Function tree
    | Stack used          :  000005D8


  ->Sub-tree of type: Function tree
                             CSTACK
    | Stack used (prev) :  000005D8
  01  isPatchExistedByID
      | Stack used (prev) :  000005D8
      | + function block  :  0000000C
  <-Sub-tree of type: Function tree
    | Stack used          :  000005E4


  ->Sub-tree of type: Function tree
                             CSTACK
    | Stack used (prev) :  000005E4
  01  pushToItemStack
      | Stack used (prev) :  000005E4
      | + function block  :  00000008
  <-Sub-tree of type: Function tree
    | Stack used          :  000005EC


  ->Sub-tree of type: Function tree
                             CSTACK
    | Stack used (prev) :  000005EC
  01  popItemStack
      | Stack used (prev) :  000005EC
      | + function block  :  00000004
  <-Sub-tree of type: Function tree
    | Stack used          :  000005F0


  ->Sub-tree of type: Function tree
                             CSTACK
    | Stack used (prev) :  000005F0
  01  updateStackEditCurItem
      | Stack used (prev) :  000005F0
      | + function block  :  00000000
  <-Sub-tree of type: Function tree
    | Stack used          :  000005F0


  ->Sub-tree of type: Function tree
                             CSTACK
    | Stack used (prev) :  000005F0
  01  updateStackPtcfg
      | Stack used (prev) :  000005F0
      | + function block  :  00000000
  <-Sub-tree of type: Function tree
    | Stack used          :  000005F0


  ->Sub-tree of type: Function tree
                             CSTACK
    | Stack used (prev) :  000005F0
  01  isTopSubMenu
      | Stack used (prev) :  000005F0
      | + function block  :  00000004
  <-Sub-tree of type: Function tree
    | Stack used          :  000005F4


  ->Sub-tree of type: Function tree
                             CSTACK
    | Stack used (prev) :  000005F4
  01  createMainMenu
      | Stack used (prev) :  000005F4
      | + function block  :  00000018
  <-Sub-tree of type: Function tree
    | Stack used          :  0000060C


  ->Sub-tree of type: Function tree
                             CSTACK
    | Stack used (prev) :  0000060C
  01  UpdateCSMname
      | Stack used (prev) :  0000060C
      | + function block  :  00000004
  <-Sub-tree of type: Function tree
    | Stack used          :  00000610


  ->Sub-tree of type: Function tree
                             CSTACK
    | Stack used (prev) :  00000610
  01  main
      | Stack used (prev) :  00000610
      | + function block  :  00000034
  <-Sub-tree of type: Function tree
    | Stack used          :  00000644


  ->Sub-tree of type: Function tree
                             CSTACK
    | Stack used (prev) :  00000644
  01  findPatchItemInED
      | Stack used (prev) :  00000644
      | + function block  :  00000000
  <-Sub-tree of type: Function tree
    | Stack used          :  00000644


  ->Sub-tree of type: Function tree
                             CSTACK
    | Stack used (prev) :  00000644
  01  getMaxFocus
      | Stack used (prev) :  00000644
      | + function block  :  00000000
  <-Sub-tree of type: Function tree
    | Stack used          :  00000644


  ->Sub-tree of type: Function tree
                             CSTACK
    | Stack used (prev) :  00000644
  01  getMinFocus
      | Stack used (prev) :  00000644
      | + function block  :  00000000
  <-Sub-tree of type: Function tree
    | Stack used          :  00000644


  ->Sub-tree of type: Function tree
                             CSTACK
    | Stack used (prev) :  00000644
  01  updateEdHdr
      | Stack used (prev) :  00000644
      | + function block  :  00000010
  <-Sub-tree of type: Function tree
    | Stack used          :  00000654


  ->Sub-tree of type: Function tree
                             CSTACK
    | Stack used (prev) :  00000654
  01  createEditGui
      | Stack used (prev) :  00000654
      | + function block  :  000002A8
  <-Sub-tree of type: Function tree
    | Stack used          :  000008FC


  ->Sub-tree of type: Function tree
                             CSTACK
    | Stack used (prev) :  000008FC
  01  show_option_menu
      | Stack used (prev) :  000008FC
      | + function block  :  00000018
  <-Sub-tree of type: Function tree
    | Stack used          :  00000914


  ->Sub-tree of type: Function tree
                             CSTACK
    | Stack used (prev) :  00000914
  01  deleteAllConfig
      | Stack used (prev) :  00000914
      | + function block  :  000004CC
  <-Sub-tree of type: Function tree
    | Stack used          :  00000DE0


  ->Sub-tree of type: Function tree
                             CSTACK
    | Stack used (prev) :  00000DE0
  01  deleteThis
      | Stack used (prev) :  00000DE0
      | + function block  :  000000B8
  <-Sub-tree of type: Function tree
    | Stack used          :  00000E98


  ->Sub-tree of type: Function tree
                             CSTACK
    | Stack used (prev) :  00000E98
  01  createProfileOnoffMenu
      | Stack used (prev) :  00000E98
      | + function block  :  00000018
  <-Sub-tree of type: Function tree
    | Stack used          :  00000EB0


  ->Sub-tree of type: Function tree
                             CSTACK
    | Stack used (prev) :  00000EB0
  01  delUnusedConfig
      | Stack used (prev) :  00000EB0
      | + function block  :  000004DC
  <-Sub-tree of type: Function tree
    | Stack used          :  0000138C


  ->Sub-tree of type: Function tree
                             CSTACK
    | Stack used (prev) :  0000138C
  01  showPatchInfo
      | Stack used (prev) :  0000138C
      | + function block  :  0000005C
  <-Sub-tree of type: Function tree
    | Stack used          :  000013E8


  ->Sub-tree of type: Function tree
                             CSTACK
    | Stack used (prev) :  000013E8
  01  fcopy
      | Stack used (prev) :  000013E8
      | + function block  :  00000034
  <-Sub-tree of type: Function tree
    | Stack used          :  0000141C


  ->Sub-tree of type: Function tree
                             CSTACK
    | Stack used (prev) :  0000141C
  01  pathInputDlg
      | Stack used (prev) :  0000141C
      | + function block  :  0000005C
  <-Sub-tree of type: Function tree
    | Stack used          :  00001478


  ->Sub-tree of type: Function tree
                             CSTACK
    | Stack used (prev) :  00001478
  01  mkpath
      | Stack used (prev) :  00001478
      | + function block  :  00000098
  <-Sub-tree of type: Function tree
    | Stack used          :  00001510


  ->Sub-tree of type: Function tree
                             CSTACK
    | Stack used (prev) :  00001510
  01  configBackUp
      | Stack used (prev) :  00001510
      | + function block  :  00000558
  <-Sub-tree of type: Function tree
    | Stack used          :  00001A68


  ->Sub-tree of type: Function tree
                             CSTACK
    | Stack used (prev) :  00001A68
  01  configRestore
      | Stack used (prev) :  00001A68
      | + function block  :  00000558
  <-Sub-tree of type: Function tree
    | Stack used          :  00001FC0


  ->Sub-tree of type: Function tree
                             CSTACK
    | Stack used (prev) :  00001FC0
  01  initPatchItem
      | Stack used (prev) :  00001FC0
      | + function block  :  0000000C
  <-Sub-tree of type: Function tree
    | Stack used          :  00001FCC


  ->Sub-tree of type: Function tree
                             CSTACK
    | Stack used (prev) :  00001FCC
  01  initPatchConfig
      | Stack used (prev) :  00001FCC
      | + function block  :  000000A8
  <-Sub-tree of type: Function tree
    | Stack used          :  00002074


  ->Sub-tree of type: Function tree
                             CSTACK
    | Stack used (prev) :  00002074
  01  findNextBposItem
      | Stack used (prev) :  00002074
      | + function block  :  00000014
  <-Sub-tree of type: Function tree
    | Stack used          :  00002088


  ->Sub-tree of type: Function tree
                             CSTACK
    | Stack used (prev) :  00002088
  01  getTheSameBPosCheckBox
      | Stack used (prev) :  00002088
      | + function block  :  00000014
  <-Sub-tree of type: Function tree
    | Stack used          :  0000209C


  ->Sub-tree of type: Function tree
                             CSTACK
    | Stack used (prev) :  0000209C
  01  fillItemDataToBuf
      | Stack used (prev) :  0000209C
      | + function block  :  00000010
  <-Sub-tree of type: Function tree
    | Stack used          :  000020AC


  ->Sub-tree of type: Function tree
                             CSTACK
    | Stack used (prev) :  000020AC
  01  getPtcSize
      | Stack used (prev) :  000020AC
      | + function block  :  0000000C
  <-Sub-tree of type: Function tree
    | Stack used          :  000020B8


  ->Sub-tree of type: Function tree
                             CSTACK
    | Stack used (prev) :  000020B8
  01  savePatchConfig
      | Stack used (prev) :  000020B8
      | + function block  :  000000AC
  <-Sub-tree of type: Function tree
    | Stack used          :  00002164


  ->Sub-tree of type: Function tree
                             CSTACK
    | Stack used (prev) :  00002164
  01  saveAllConfig
      | Stack used (prev) :  00002164
      | + function block  :  00000008
  <-Sub-tree of type: Function tree
    | Stack used          :  0000216C


  ->Sub-tree of type: Function tree
                             CSTACK
    | Stack used (prev) :  0000216C
  01  getnumwidth
      | Stack used (prev) :  0000216C
      | + function block  :  00000000
  <-Sub-tree of type: Function tree
    | Stack used          :  0000216C


  ->Sub-tree of type: Function tree
                             CSTACK
    | Stack used (prev) :  0000216C
  01  uni2ws
      | Stack used (prev) :  0000216C
      | + function block  :  00000008
  <-Sub-tree of type: Function tree
    | Stack used          :  00002174


  ->Sub-tree of type: Function tree
                             CSTACK
    | Stack used (prev) :  00002174
  01  ws2uni
      | Stack used (prev) :  00002174
      | + function block  :  00000008
  <-Sub-tree of type: Function tree
    | Stack used          :  0000217C


  ->Sub-tree of type: Function tree
                             CSTACK
    | Stack used (prev) :  0000217C
  01  hex2ws
      | Stack used (prev) :  0000217C
      | + function block  :  00000018
  <-Sub-tree of type: Function tree
    | Stack used          :  00002194


  ->Sub-tree of type: Function tree
                             CSTACK
    | Stack used (prev) :  00002194
  01  uniFormatString2ws
      | Stack used (prev) :  00002194
      | + function block  :  00000020
  <-Sub-tree of type: Function tree
    | Stack used          :  000021B4


  ->Sub-tree of type: Function tree
                             CSTACK
    | Stack used (prev) :  000021B4
  01  isUniFormat
      | Stack used (prev) :  000021B4
      | + function block  :  00000000
  <-Sub-tree of type: Function tree
    | Stack used          :  000021B4


  ->Sub-tree of type: Function tree
                             CSTACK
    | Stack used (prev) :  000021B4
  01  ws2hex
      | Stack used (prev) :  000021B4
      | + function block  :  00000220
  <-Sub-tree of type: Function tree
    | Stack used          :  000023D4


  ->Sub-tree of type: Function tree
                             CSTACK
    | Stack used (prev) :  000023D4
  01  bytes_2ws
      | Stack used (prev) :  000023D4
      | + function block  :  00000018
  <-Sub-tree of type: Function tree
    | Stack used          :  000023EC


  ->Sub-tree of type: Function tree
                             CSTACK
    | Stack used (prev) :  000023EC
  01  ints_2ws
      | Stack used (prev) :  000023EC
      | + function block  :  00000018
  <-Sub-tree of type: Function tree
    | Stack used          :  00002404


  ->Sub-tree of type: Function tree
                             CSTACK
    | Stack used (prev) :  00002404
  01  strncmpNoCase
      | Stack used (prev) :  00002404
      | + function block  :  00000004
  <-Sub-tree of type: Function tree
    | Stack used          :  00002408


  ->Sub-tree of type: Function tree
                             CSTACK
    | Stack used (prev) :  00002408
  01  chr2num
      | Stack used (prev) :  00002408
      | + function block  :  00000000
  <-Sub-tree of type: Function tree
    | Stack used          :  00002408


  ->Sub-tree of type: Function tree
                             CSTACK
    | Stack used (prev) :  00002408
  01  gotoRealPos
      | Stack used (prev) :  00002408
      | + function block  :  00000000
  <-Sub-tree of type: Function tree
    | Stack used          :  00002408


  ->Sub-tree of type: Function tree
                             CSTACK
    | Stack used (prev) :  00002408
  01  strstrInQuote
      | Stack used (prev) :  00002408
      | + function block  :  00000010
  <-Sub-tree of type: Function tree
    | Stack used          :  00002418


  ->Sub-tree of type: Function tree
                             CSTACK
    | Stack used (prev) :  00002418
  01  strchrInQuote
      | Stack used (prev) :  00002418
      | + function block  :  00000000
  <-Sub-tree of type: Function tree
    | Stack used          :  00002418


  ->Sub-tree of type: Function tree
                             CSTACK
    | Stack used (prev) :  00002418
  01  gotoQuoteStart
      | Stack used (prev) :  00002418
      | + function block  :  00000000
  <-Sub-tree of type: Function tree
    | Stack used          :  00002418


  ->Sub-tree of type: Function tree
                             CSTACK
    | Stack used (prev) :  00002418
  01  gotoQuoteEnd
      | Stack used (prev) :  00002418
      | + function block  :  00000000
  <-Sub-tree of type: Function tree
    | Stack used          :  00002418


  ->Sub-tree of type: Function tree
                             CSTACK
    | Stack used (prev) :  00002418
  01  gotoNextNameQuote
      | Stack used (prev) :  00002418
      | + function block  :  00000000
  <-Sub-tree of type: Function tree
    | Stack used          :  00002418


  ->Sub-tree of type: Function tree
                             CSTACK
    | Stack used (prev) :  00002418
  01  gotoStringEndByChr
      | Stack used (prev) :  00002418
      | + function block  :  00000000
  <-Sub-tree of type: Function tree
    | Stack used          :  00002418


  ->Sub-tree of type: Function tree
                             CSTACK
    | Stack used (prev) :  00002418
  01  gotoMyStrStart
      | Stack used (prev) :  00002418
      | + function block  :  00000004
  <-Sub-tree of type: Function tree
    | Stack used          :  0000241C


  ->Sub-tree of type: Function tree
                             CSTACK
    | Stack used (prev) :  0000241C
  01  gotoMyStrEnd
      | Stack used (prev) :  0000241C
      | + function block  :  00000004
  <-Sub-tree of type: Function tree
    | Stack used          :  00002420


  ->Sub-tree of type: Function tree
                             CSTACK
    | Stack used (prev) :  00002420
  01  strnCopyWithEnd
      | Stack used (prev) :  00002420
      | + function block  :  0000000C
  <-Sub-tree of type: Function tree
    | Stack used          :  0000242C


  ->Sub-tree of type: Function tree
                             CSTACK
    | Stack used (prev) :  0000242C
  01  str2num
      | Stack used (prev) :  0000242C
      | + function block  :  00000020
  <-Sub-tree of type: Function tree
    | Stack used          :  0000244C


  ->Sub-tree of type: Function tree
                             CSTACK
    | Stack used (prev) :  0000244C
  01  str2num_short
      | Stack used (prev) :  0000244C
      | + function block  :  00000020
  <-Sub-tree of type: Function tree
    | Stack used          :  0000246C


  ->Sub-tree of type: Function tree
                             CSTACK
    | Stack used (prev) :  0000246C
  01  str2num_char
      | Stack used (prev) :  0000246C
      | + function block  :  00000024
  <-Sub-tree of type: Function tree
    | Stack used          :  00002490


  ->Sub-tree of type: Function tree
                             CSTACK
    | Stack used (prev) :  00002490
  01  cleanStrByChr
      | Stack used (prev) :  00002490
      | + function block  :  00000000
  <-Sub-tree of type: Function tree
    | Stack used          :  00002490


  ->Sub-tree of type: Function tree
                             CSTACK
    | Stack used (prev) :  00002490
  01  str2bytes
      | Stack used (prev) :  00002490
      | + function block  :  00000018
  <-Sub-tree of type: Function tree
    | Stack used          :  000024A8


  ->Sub-tree of type: Function tree
                             CSTACK
    | Stack used (prev) :  000024A8
  01  str2ints
      | Stack used (prev) :  000024A8
      | + function block  :  00000018
  <-Sub-tree of type: Function tree
    | Stack used          :  000024C0


  ->Sub-tree of type: Function tree
                             CSTACK
    | Stack used (prev) :  000024C0
  01  DrwImg
      | Stack used (prev) :  000024C0
      | + function block  :  00000040
  <-Sub-tree of type: Function tree
    | Stack used          :  00002500


  ->Sub-tree of type: Function tree
                             CSTACK
    | Stack used (prev) :  00002500
  01  EditPostionGUI
      | Stack used (prev) :  00002500
      | + function block  :  00000018
  <-Sub-tree of type: Function tree
    | Stack used          :  00002518


  ->Sub-tree of type: Function tree
                             CSTACK
    | Stack used (prev) :  00002518
  01  EditColors
      | Stack used (prev) :  00002518
      | + function block  :  0000000C
  <-Sub-tree of type: Function tree
    | Stack used          :  00002524


  ->Sub-tree of type: Function tree
                             CSTACK
    | Stack used (prev) :  00002524
  01  Free_FLIST
      | Stack used (prev) :  00002524
      | + function block  :  00000008
  <-Sub-tree of type: Function tree
    | Stack used          :  0000252C


  ->Sub-tree of type: Function tree
                             CSTACK
    | Stack used (prev) :  0000252C
  01  strcmp_nocase
      | Stack used (prev) :  0000252C
      | + function block  :  00000000
  <-Sub-tree of type: Function tree
    | Stack used          :  0000252C


  ->Sub-tree of type: Function tree
                             CSTACK
    | Stack used (prev) :  0000252C
  01  AddToFList
      | Stack used (prev) :  0000252C
      | + function block  :  00000018
  <-Sub-tree of type: Function tree
    | Stack used          :  00002544


  ->Sub-tree of type: Function tree
                             CSTACK
    | Stack used (prev) :  00002544
  01  FindFiles
      | Stack used (prev) :  00002544
      | + function block  :  000004E8
  <-Sub-tree of type: Function tree
    | Stack used          :  00002A2C


  ->Sub-tree of type: Function tree
                             CSTACK
    | Stack used (prev) :  00002A2C
  01  FindFLISTtByNS
      | Stack used (prev) :  00002A2C
      | + function block  :  00000000
  <-Sub-tree of type: Function tree
    | Stack used          :  00002A2C


  ->Sub-tree of type: Function tree
                             CSTACK
    | Stack used (prev) :  00002A2C
  01  FindFLISTtByN
      | Stack used (prev) :  00002A2C
      | + function block  :  00000008
  <-Sub-tree of type: Function tree
    | Stack used          :  00002A34


  ->Sub-tree of type: Function tree
                             CSTACK
    | Stack used (prev) :  00002A34
  01  SavePath
      | Stack used (prev) :  00002A34
      | + function block  :  0000003C
  <-Sub-tree of type: Function tree
    | Stack used          :  00002A70


  ->Sub-tree of type: Function tree
                             CSTACK
    | Stack used (prev) :  00002A70
  01  CreateRootMenu
      | Stack used (prev) :  00002A70
      | + function block  :  00000030
  <-Sub-tree of type: Function tree
    | Stack used          :  00002AA0


  ->Sub-tree of type: Function tree
                             CSTACK
    | Stack used (prev) :  00002AA0
  01  open_select_file_gui
      | Stack used (prev) :  00002AA0
      | + function block  :  000000D8
  <-Sub-tree of type: Function tree
    | Stack used          :  00002B78




                ****************************************
                *                                      *
                *      SEGMENTS IN ADDRESS ORDER       *
                *                                      *
                ****************************************


SEGMENT              SPACE    START ADDRESS   END ADDRESS     SIZE  TYPE  ALIGN
=======              =====    =============   ===========     ====  ====  =====
ELFBEGIN             CODE_AREA           00000000                     rel    0
DATA_ID              CODE_AREA      00000000 - 0000016B         16C   rel    2
START                CODE_AREA           0000016C                     dse    0
CODE                 CODE_AREA      0000016C - 00008DAF        8C44   rel    2
DATA_C               CODE_AREA      00008DB0 - 00009AF6         D47   rel    2
INITTAB              CODE_AREA      00009AF8 - 00009B0F          18   rel    2
DATA_Z               CODE_AREA      00009B10 - 00015C53        C144   rel    2
DATA_I               DATA_AREA      00000000 - 0000016B         16C   rel    2

                ****************************************
                *                                      *
                *        END OF CROSS REFERENCE        *
                *                                      *
                ****************************************

 89 171 bytes of CODE memory
    364 bytes of DATA memory

Errors: none
Warnings: none

